:020000040800F2
:1000000000800020152E0008A11A0008A31A00087D
:10001000A51A0008A71A0008A91A00080000000085
:10002000000000000000000000000000AB1A000803
:10003000AD1A000800000000AF1A0008B11A00084D
:10004000652E0008652E0008B51A0008652E000808
:10005000652E0008652E0008C11A0008C71A00089E
:10006000652E0008652E0008652E0008652E000824
:10007000652E0008652E0008652E0008CD1A0008C0
:10008000652E0008652E0008652E0008652E000804
:10009000652E0008652E0008D91A0008652E000894
:1000A000652E0008652E0008652E0008652E0008E4
:1000B000652E0008652E0008652E0008652E0008D4
:1000C000652E0008652E0008652E0008652E0008C4
:1000D000652E0008E11A0008652E0008652E00084C
:1000E000652E0008652E0008ED1A0008652E000830
:1000F000652E0008652E0008652E0008652E000894
:10010000652E0008652E0008F91A0008652E000803
:10011000652E0008652E0008652E0008652E000873
:10012000652E0008652E0008652E0008652E000863
:08013000652E0008652E000891
:1001380010B5054C237833B9044B13B10448AFF319
:1001480000800123237010BD100100200000000072
:10015800900B010808B5034B1BB103490348AFF3E3
:10016800008008BD0000000014010020900B010869
:10017800034613F8012B002AFBD1181A01387047DF
:1001880081F0004102E000BF83F0004330B54FEA40
:1001980041044FEA430594EA050F08BF90EA020FAD
:1001A8001FBF54EA000C55EA020C7FEA645C7FEA40
:1001B800655C00F0E2804FEA5454D4EB5555B8BF63
:1001C8006D420CDD2C4480EA020281EA030382EAD4
:1001D800000083EA010180EA020281EA0303362D66
:1001E80088BF30BD11F0004F4FEA01314FF4801C39
:1001F8004CEA113102D0404261EB410113F0004F4B
:100208004FEA03334CEA133302D0524263EB430301
:1002180094EA050F00F0A780A4F10104D5F1200E9F
:100228000DDB02FA0EFC22FA05F2801841F10001FA
:1002380003FA0EF2801843FA05F359410EE0A5F1CE
:1002480020050EF1200E012A03FA0EFC28BF4CF0FF
:10025800020C43FA05F3C01851EBE37101F00045B5
:1002680007D54FF0000EDCF1000C7EEB00006EEBC2
:100278000101B1F5801F1BD3B1F5001F0CD349084C
:100288005FEA30004FEA3C0C04F101044FEA4452A3
:1002980012F5800F80F09A80BCF1004F08BF5FEA2A
:1002A800500C50F1000041EB045141EA050130BD0A
:1002B8005FEA4C0C404141EB0101013C28BFB1F51C
:1002C800801FE9D291F0000F04BF01460020B1FA67
:1002D80081F308BF2033A3F10B03B3F120020CDA3A
:1002E8000C3208DD02F1140CC2F10C0201FA0CF018
:1002F80021FA02F10CE002F11402D8BFC2F1200C7D
:1003080001FA02F120FA0CFCDCBF41EA0C01904032
:10031800E41AA2BF01EB0451294330BD6FEA04047B
:100328001F3C1CDA0C340EDC04F11404C4F1200266
:1003380020FA04F001FA02F340EA030021FA04F378
:1003480045EA030130BDC4F10C04C4F1200220FACF
:1003580002F001FA04F340EA0300294630BD21FA0D
:1003680004F0294630BD94F0000F83F4801306BFD3
:1003780081F480110134013D4EE77FEA645C18BFC7
:100388007FEA655C29D094EA050F08BF90EA020F5E
:1003980005D054EA000C04BF1946104630BD91EA56
:1003A800030F1EBF0021002030BD5FEA545C05D159
:1003B8004000494128BF41F0004130BD14F5800498
:1003C8003CBF01F5801130BD01F0004545F0FE410C
:1003D80041F470014FF0000030BD7FEA645C1ABF41
:1003E800194610467FEA655C1CBF0B46024650EA78
:1003F800013406BF52EA033591EA030F41F40021A4
:1004080030BD00BF90F0000F04BF0021704730B529
:100418004FF4806404F132044FF000054FF00001FE
:1004280050E700BF90F0000F04BF0021704730B5BF
:100438004FF4806404F1320410F0004548BF404294
:100448004FF000013EE700BF42004FEAE2014FEAE9
:1004580031014FEA02701FBF12F07F4393F07F4FC4
:1004680081F06051704732F07F4208BF704793F0C7
:100478007F4F04BF41F40021704730B54FF46074DA
:1004880001F0004521F000411CE700BF50EA0102DD
:1004980008BF704730B54FF000050AE050EA010286
:1004A80008BF704730B511F0004502D5404261EBF6
:1004B80041014FF4806404F132045FEA915C3FF437
:1004C800D8AE4FF003025FEADC0C18BF03325FEAD4
:1004D800DC0C18BF033202EBDC02C2F1200300FA85
:1004E80003FC20FA02F001FA03FE40EA0E0021FAAA
:1004F80002F11444BDE600BF70B54FF0FF0C4CF498
:10050800E06C1CEA11541DBF1CEA135594EA0C0F49
:1005180095EA0C0F00F0DEF82C4481EA030621EA84
:100528004C5123EA4C5350EA013518BF52EA0335BF
:1005380041F4801143F4801338D0A0FB02CE4FF071
:100548000005E1FB02E506F00042E0FB03E54FF0A1
:100558000006E1FB03569CF0000F18BF4EF0010E99
:10056800A4F1FF04B6F5007F64F5407404D25FEA95
:100578004E0E6D4146EB060642EAC62141EA555148
:100588004FEAC52040EA5E504FEACE2EB4F1FD0C8A
:1005980088BFBCF5E06F1ED8BEF1004F08BF5FEA08
:1005A800500E50F1000041EB045170BD06F00046BA
:1005B80046EA010140EA020081EA0301B4EB5C0467
:1005C800C2BFD4EB0C0541EA045170BD41F480115F
:1005D8004FF0000E013C00F3AB8014F1360FDEBF84
:1005E800002001F0004170BDC4F10004203C35DA60
:1005F8000C341BDC04F11404C4F1200500FA05F3E3
:1006080020FA04F001FA05F240EA020001F0004283
:1006180021F0004110EBD37021FA04F642EB0601F9
:100628005EEA430E08BF20EAD37070BDC4F10C0423
:10063800C4F1200500FA04F320FA05F001FA04F2E7
:1006480040EA020001F0004110EBD37041F10001D3
:100658005EEA430E08BF20EAD37070BDC4F12005DE
:1006680000FA05F24EEA020E20FA04F301FA05F246
:1006780043EA020321FA04F001F0004121FA04F2EE
:1006880020EA020000EBD3705EEA430E08BF20EABE
:10069800D37070BD94F0000F0FD101F000464000F8
:1006A80041EB010111F4801F08BF013CF7D041EA7A
:1006B800060195F0000F18BF704703F0004652007E
:1006C80043EB030313F4801F08BF013DF7D043EA4F
:1006D8000603704794EA0C0F0CEA135518BF95EA05
:1006E8000C0F0CD050EA410618BF52EA4306D1D18C
:1006F80081EA030101F000414FF0000070BD50EAAB
:10070800410606BF1046194652EA430619D094EA34
:100718000C0F02D150EA013613D195EA0C0F05D11E
:1007280052EA03361CBF104619460AD181EA030172
:1007380001F0004141F0FE4141F470014FF000002A
:1007480070BD41F0FE4141F4780170BD70B54FF0C5
:10075800FF0C4CF4E06C1CEA11541DBF1CEA135545
:1007680094EA0C0F95EA0C0F00F0A7F8A4EB050427
:1007780081EA030E52EA03354FEA013100F088801E
:100788004FEA03334FF0805545EA131343EA1263E7
:100798004FEA022245EA111545EA10654FEA00269C
:1007A8000EF000419D4208BF964244F1FD0404F555
:1007B800407402D25B084FEA3202B61A65EB0305B1
:1007C8005B084FEA32024FF480104FF4002CB6EB6E
:1007D800020E75EB030E22BFB61A754640EA0C00EE
:1007E8005B084FEA3202B6EB020E75EB030E22BF2E
:1007F800B61A754640EA5C005B084FEA3202B6EB6F
:10080800020E75EB030E22BFB61A754640EA9C002D
:100818005B084FEA3202B6EB020E75EB030E22BFFD
:10082800B61A754640EADC0055EA060E18D04FEABB
:10083800051545EA16754FEA06164FEAC30343EA5B
:1008480052734FEAC2025FEA1C1CC0D111F4801F28
:100858000BD141EA00014FF000004FF0004CB6E721
:1008680011F4801F04BF01430020B4F1FD0C88BFC0
:10087800BCF5E06F3FF6AFAEB5EB030C04BFB6EBCB
:10088800020C5FEA500C50F1000041EB045170BDBE
:100898000EF0004E4EEA113114EB5C04C2BFD4EBEB
:1008A8000C0541EA045170BD41F480114FF0000E6F
:1008B800013C90E645EA060E8DE60CEA135594EAEB
:1008C8000C0F08BF95EA0C0F3FF43BAF94EA0C0FEE
:1008D8000AD150EA01347FF434AF95EA0C0F7FF463
:1008E80025AF104619462CE795EA0C0F06D152EAB7
:1008F80003353FF4FDAE1046194622E750EA41069B
:1009080018BF52EA43067FF4C5AE50EA41047FF4AB
:100918000DAF52EA43057FF4EBAE12E74FF0FF3C10
:1009280006E000BF4FF0010C02E000BF4FF0010CE1
:100938004DF804CD4FEA410C7FEA6C5C4FEA430C5A
:1009480018BF7FEA6C5C1BD001B050EA410C0CBFA9
:1009580052EA430C91EA030F02BF90EA020F00200B
:10096800704710F1000F91EA030F58BF994208BF72
:1009780090422CBFD8176FEAE37040F0010070472F
:100988004FEA410C7FEA6C5C02D150EA013C07D186
:100998004FEA430C7FEA6C5CD6D152EA033CD3D0D1
:1009A8005DF8040B704700BF8446104662468C46CB
:1009B8001946634600E000BF01B5FFF7B7FF0028FE
:1009C80048BF10F1000F01BD4DF808EDFFF7F4FF27
:1009D8000CBF012000205DF808FB00BF4DF808EDB2
:1009E800FFF7EAFF34BF012000205DF808FB00BFD5
:1009F8004DF808EDFFF7E0FF94BF012000205DF8F7
:100A080008FB00BF4DF808EDFFF7CEFF94BF0120AB
:100A180000205DF808FB00BF4DF808EDFFF7C4FFA4
:100A280034BF012000205DF808FB00BF4FEA4102F7
:100A380012F5001215D211D56FF47873B3EB625228
:100A480012D94FEAC12343F0004343EA505311F04F
:100A5800004F23FA02F018BF404270474FF00000E1
:100A6800704750EA013005D111F0004008BF6FF01F
:100A7800004070474FF00000704700BF80F0004012
:100A880002E000BF81F0004142001FBF5FEA41035E
:100A980092EA030F7FEA226C7FEA236C6AD04FEA5E
:100AA8001262D2EB1363C1BFD218414048404140A3
:100AB800B8BF5B42192B88BF704710F0004F40F455
:100AC800000020F07F4018BF404211F0004F41F471
:100AD800000121F07F4118BF494292EA030F3FD03D
:100AE800A2F1010241FA03FC10EB0C00C3F1200350
:100AF80001FA03F100F0004302D5494260EB4000DF
:100B0800B0F5000F13D3B0F1807F06D340084FEA49
:100B1800310102F10102FE2A51D2B1F1004F40EB3E
:100B2800C25008BF20F0010040EA030070474900A6
:100B380040EB0000013A28BFB0F5000FEDD2B0FA43
:100B480080FCACF1080CB2EB0C0200FA0CF0AABF66
:100B580000EBC25052421843BCBFD0401843704704
:100B680092F0000F81F4000106BF80F4000001320A
:100B7800013BB5E74FEA41037FEA226C18BF7FEAE1
:100B8800236C21D092EA030F04D092F0000F08BF23
:100B98000846704790EA010F1CBF0020704712F00A
:100BA8007F4F04D1400028BF40F00040704712F149
:100BB80000723CBF00F50000704700F0004343F0AE
:100BC800FE4040F4000070477FEA226216BF0846E4
:100BD8007FEA23630146420206BF5FEA412390EAA7
:100BE800010F40F4800070474FF0000304E000BF9D
:100BF80010F0004348BF40425FEA000C08BF70474E
:100C080043F0964301464FF000001CE050EA010211
:100C180008BF70474FF000030AE000BF50EA010226
:100C280008BF704711F0004302D5404261EB410113
:100C38005FEA010C02BF84460146002043F0B64338
:100C480008BFA3F18053A3F50003BCFA8CF2083A5D
:100C5800A3EBC25310DB01FA02FC634400FA02FC66
:100C6800C2F12002BCF1004F20FA02F243EB02006D
:100C780008BF20F00100704702F1200201FA02FCCF
:100C8800C2F1200250EA4C0021FA02F243EB0200C2
:100C980008BF20EADC7070474FF0FF0C1CEAD05206
:100CA8001EBF1CEAD15392EA0C0F93EA0C0F6FD0C7
:100CB8001A4480EA010C400218BF5FEA41211ED0A5
:100CC8004FF0006343EA501043EA5111A0FB013191
:100CD8000CF00040B1F5000F3EBF490041EAD37166
:100CE8005B0040EA010062F17F02FD2A1DD8B3F1E2
:100CF800004F40EBC25008BF20F00100704790F051
:100D0800000F0CF0004C08BF49024CEA502040EAA2
:100D180051207F3AC2BFD2F1FF0340EAC250704768
:100D280040F400004FF00003013A5DDC12F1190FA6
:100D3800DCBF00F000407047C2F10002410021FA18
:100D480002F1C2F1200200FA02FC5FEA310040F130
:100D5800000053EA4C0308BF20EADC70704792F0A9
:100D6800000F00F0004C02BF400010F4000F013AE1
:100D7800F9D040EA0C0093F0000F01F0004C02BFDC
:100D8800490011F4000F013BF9D041EA0C018FE74B
:100D98000CEAD15392EA0C0F18BF93EA0C0F0AD051
:100DA80030F0004C18BF31F0004CD8D180EA010077
:100DB80000F00040704790F0000F17BF90F0004F10
:100DC800084691F0000F91F0004F14D092EA0C0FF2
:100DD80001D142020FD193EA0C0F03D14B0218BF85
:100DE800084608D180EA010000F0004040F0FE40CB
:100DF80040F40000704740F0FE4040F44000704767
:100E08004FF0FF0C1CEAD0521EBF1CEAD15392EAE5
:100E18000C0F93EA0C0F69D0A2EB030280EA010CD5
:100E280049024FEA402037D04FF0805343EA11116E
:100E380043EA10130CF000408B4238BF5B0042F1CC
:100E48007D024FF4000C8B4224BF5B1A40EA0C0071
:100E5800B3EB510F24BFA3EB510340EA5C00B3EBA3
:100E6800910F24BFA3EB910340EA9C00B3EBD10F91
:100E780024BFA3EBD10340EADC001B0118BF5FEAE3
:100E88001C1CE0D1FD2A3FF650AF8B4240EBC2500C
:100E980008BF20F0010070470CF0004C4CEA5020CD
:100EA8007F32C2BFD2F1FF0340EAC250704740F41C
:100EB80000004FF00003013A37E792F0000F00F00E
:100EC800004C02BF400010F4000F013AF9D040EA8C
:100ED8000C0093F0000F01F0004C02BF490011F420
:100EE800000F013BF9D041EA0C0195E70CEAD15318
:100EF80092EA0C0F08D142027FF47DAF93EA0C0FFF
:100F08007FF470AF084676E793EA0C0F04D14B02E2
:100F18003FF44CAF08466EE730F0004C18BF31F094
:100F2800004CCAD130F000427FF45CAF31F000438E
:100F38007FF43CAF5FE700BF4FEA4002B2F1FE4FDB
:100F48000FD34FF09E03B3EB12620DD94FEA002383
:100F580043F0004310F0004F23FA02F018BF40425C
:100F680070474FF00000704712F1610F01D1420243
:100F780005D110F0004008BF6FF0004070474FF0F7
:100F88000000704742000ED2B2F1FE4F0BD34FF073
:100F98009E03B3EB126209D44FEA002343F00043E7
:100FA80023FA02F070474FF00000704712F1610F0A
:100FB80001D1420202D14FF0FF3070474FF00000DC
:100FC800704700BF53B94AB9002908BF00281CBFA1
:100FD8004FF0FF314FF0FF3000F06AB9ADF1080C67
:100FE8006DE904CE00F006F8DDF804E0DDE902233F
:100FF80004B070472DE9F047089D0C46002B4ED1F0
:1010080094468C458646B2FA82F262D94AB1C2F158
:101018002003914020FA03F30CFA02FC194300FA6A
:1010280002FE4FEA1C471FFA8CF6B1FBF7F44FEAB1
:101038001E4307FB141143EA014304FB06F19942DE
:101048000AD91CEB030304F1FF3080F012819942A6
:1010580040F20F81023C6344591A1FFA8EF3B1FB28
:10106800F7F007FB101143EA014300FB06F69E4226
:101078000AD91CEB030300F1FF3180F0FC809E428B
:1010880040F2F980634402389B1B40EA0440002187
:101098001DB1D3400022C5E90032BDE8F0878B427C
:1010A80005D90DB1C5E9000100210846F5E7B3FAF5
:1010B80083F1002946D1A34202D39042C0F0F080C8
:1010C800861A64EB03030120002DE6D0C5E900630E
:1010D800E3E7002A40F09080A1EB0C044FEA1C489B
:1010E8001FFA8CF70121B4FBF8F64FEA1E4308FB00
:1010F800164443EA044307FB06F0984208D91CEB60
:10110800030306F1FF3402D2984200F2CD8026464E
:101118001C1A1FFA8EF3B4FBF8F008FB104443EADC
:10112800044300FB07F79F4208D91CEB030300F1B7
:10113800FF3402D29F4200F2B0802046DB1B40EA17
:101148000640A5E7C1F120068B4022FA06F71F43A7
:1011580020FA06FC04FA01F343EA0C03F44000FA0F
:1011680001F8380C4FEA1349B4FBF0FE1FFA87FC6C
:1011780000FB1E4449EA04440EFB0CF9A14502FA9F
:1011880001F20AD93C190EF1FF3A80F08480A1459A
:1011980040F28180AEF1020E3C44A4EB09041FFA30
:1011A80083F9B4FBF0F300FB134449EA044403FB5E
:1011B8000CFCA44507D93C1903F1FF3067D2A445BC
:1011C80065D9023B3C4443EA0E40A0FB0293A4EBE2
:1011D8000C049C42CE469C4651D34ED055B1B8EB38
:1011E8000E0364EB0C0404FA06F6CB401E43CC4015
:1011F800C5E90064002150E7C2F1200320FA03F199
:101208000CFA02FC24FA03F394400C434FEA1C48FE
:1012180000FA02FE1FFA8CF7B3FBF8F008FB103156
:10122800230C43EA014300FB07F1994208D91CEB60
:10123800030300F1FF362CD299422AD902386344BD
:101248005B1AA4B2B3FBF8F108FB113344EA034478
:1012580001FB07F3A34208D91CEB040401F1FF3694
:1012680013D2A34211D902396444E41A41EA004175
:1012780039E70446F0E6084606E7C845AED2B9EBBA
:10128800020E63EB070C0138A8E73146EDE7034689
:1012980099E73046D4E7D6467FE7634402384DE7FE
:1012A8000646234608460FE7023E634430E700BF80
:1012B800704700BF1348144A08B54FF00043C0E90F
:1012C80000230422426101220023C2614FF48051AD
:1012D8000722C0E90233C0E90933C0E90C120361EF
:1012E8000383837680F8203080F82C30826380F87E
:1012F8003C30C36401F086FE18B1BDE8084000F038
:101308002DBB08BD2C010020002401400268084BB9
:101318009A4282B00AD14FF0B0431A6E42F400727A
:101328001A661B6E03F400730193019B02B07047A9
:10133800002401400268054B9A4201BF4FF0B042B9
:10134800136E23F400731366704700BF0024014036
:1013580030B585B000240546CDE901440394FFF774
:10136800A9FF144802F0E2F908B100F0F7FA1148B1
:10137800039401A9CDE9015401F0A2FF08B100F0DE
:10138800EDFA0C4802F0FCF808B100F0E7FA4FF06B
:10139800FF31084801F036FF064802F0A9F9054870
:1013A80001F08AFF0446034802F04CF9204605B0D4
:1013B80030BD00BF2C010020014B024A1A60704763
:1013C8002C0100200024014008B50948FFF7C0FFA0
:1013D80068B1084BB3F8AA304FF6FF72934216BFB4
:1013E80040F6E442044B5343B3FBF0F398B208BD14
:1013F800002000B40075FF1FD8084C0013B5002367
:10140800ADF80630FFF7E0FF04461948FFF7A0FFE4
:10141800184BB3F8C820B3F8A8108A4204FB00F0B0
:1014280018D040F6E443B0FBF3F364205B1A43435F
:10143800521A93FBF2F31E331BB2ADF80630BDF817
:1014480006305BB21B02ADF80630BDF8060000B2EC
:1014580002B010BD4FF47A7240F6FF73B0FBF3F39D
:101468005343A3F53923A3F50C6340F6C412E0E710
:10147800001000B00075FF1F4FF0B04307B59A6C1D
:1014880042F004029A649A6C02F004020192019AF2
:101498009A6C42F001029A649B6C03F0010300937A
:1014A800002202210F20009B02F0DEF90F2003B07A
:1014B8005DF804EB02F00ABA08B502F05BFC10B163
:1014C8006FF0040008BD064B9A6942F040429A61E9
:1014D8004CF2FA321A6102F05FFC0028F2D0EFE712
:1014E80000400058F0B585B000230D46009306462D
:1014F800A8B3FFF7E1FF044670BB02F03BFC88BBD2
:101508001A481B4A02230193D0F8E01506F17843E4
:1015180002EA8121B3FBF1F701FB1733DB0A0293DF
:10152800D0F8E00505F178410139314402EA80221A
:10153800B1FBF2F002FB1011C3EBD1230133694672
:1015480001A8039302F0A8FC20B1022814BF6FF091
:101558000104012402F020FC204605B0F0BD6FF024
:101568000504F9E76FF00404F6E700BF0070FF1FF9
:1015780000FCFF03014B1860002070479001002019
:101588002DE9F04FB0F1006F89B006460F4690463E
:10159800C0F0C080DFF89091644DD9F8E03505EAD5
:1015A800832303F10063013B984200F2B3800029D2
:1015B80000F0B38040EA02035B0740F0AE80FFF71B
:1015C8007BFF044690BB02F0D5FB002840F0A880C2
:1015D800D9F8E015009705EA812106F17842B2FBB7
:1015E800F1F301FB132208F17843013B3344B3FBC9
:1015F800F1F001FB1033DB0A01334FEAD22AA3EBE7
:10160800D222012A039388BFC6F30A050AF5803758
:10161800C6F108038CBFC5F500654546FF02B34611
:101628000693039B9A4505D302F0B6FB204609B002
:10163800BDE8F08FA6F10803069A1A4495421CD813
:10164800009B04950193CDF814B04FF00009059B59
:1016580009EB0301049B99453DD3009BAB442B4404
:10166800A8EB0505B5F5006F009328BF4FF400659A
:101678000AF1010A07F50067D3E753F8081F5A680B
:10168800B2F1FF3F08BFB1F1FF3FD5D0284B186832
:1016980010B96FF00504C7E727B14FF40062394667
:1016A8000EF098FDDFF888900099D9F80030CBF358
:1016B8000A001844AAB20EF08DFD4FF400613846B6
:1016C800FFF710FF00BBD9F8003001934FF4006317
:1016D80005970493B9E7019B07914B4402930120B6
:1016E800D3E9002302F092FB88B90799019BD1E95D
:1016F800000259F80310029B5B689A4208BF8842AF
:1017080005D109F10809A2E76FF001048CE76FF031
:10171800030489E74FF0FF3488E76FF0050485E795
:101728006FF0040482E700BF0070FF1F00FCFF0396
:1017380090010020B1F1006F70B510D30B4BD3F8B6
:10174800E0650B4B03EA862303F10063013B9942F2
:1017580005D838B192B20EF03DFD002070BD4FF0B3
:10176800FF30FBE76FF00500F8E700BF0070FF1FD0
:1017780000FCFF03B0F1006F10B40DD3084BD3F891
:10178800E045084B03EA842303F10063013B9842D8
:1017980002D810BCFFF7A6BE4FF0FF3010BC704750
:1017A8000070FF1F00FCFF034FF0B04382B0DA6CFB
:1017B8000243DA64DB6C03400193019B02B070477B
:1017C8002DE9F04387B01422002101A80FF02EF96B
:1017D8000220FFF7E9FF364F0420FFF7E5FF01205D
:1017E800FFF7E2FF4FF43A410022384602F0C8FC06
:1017F80001254FF40A430024CDE9013501A902234C
:1018080038460326CDE903434FF4041902F092FB4E
:1018180001A94FF09040CDE90169039502F08AFBD8
:101828004FF4405301A93846CDE901354FF040083F
:10183800CDE9034602F07EFB01A91E480395202747
:10184800CDE9018902F076FB01A94FF09040CDE97E
:101858000175CDE9035602F06DFB01A94FF09040E8
:10186800CDE90184CDE9035602F064FB22463946EE
:101878004FF0904002F084FC22462146062001F0F9
:10188800F3FF062002F022F822462146072001F045
:10189800EBFF072002F01AF822462146162001F035
:1018A800E3FF162002F012F807B0BDE8F08300BF8E
:1018B800000400480008004800B59BB048220021F9
:1018C80008A80FF0B3F81C22002101A80FF0AEF809
:1018D80002F070FC4FF0B0420120D2F8903023F0B3
:1018E8001803C2F89030D2F8003423F4C06343F4EC
:1018F8000073C2F80034D2F8003403F4C0630093D4
:10190800009B2423089381230B930023CDE9100324
:10191800B02208A8CDE9122302F0C4FD08B172B6BE
:10192800FEE74F23CDE90130CDE90300059007908C
:10193800022101A803F050F808B172B6FEE71BB007
:101948005DF804FB08B501F00BFBFFF7B5FFFFF7E7
:1019580037FF00F001FE00F006FEFCE772B6FEE776
:1019680000B58DB02C22002101A80FF05FF81748B0
:10197800174B03601F2383604FF080420023C0E9A8
:101988000433C0E9072383614FF48073436203F093
:10199800E3FA08B1FFF7E2FF0C4803F009FC08B1CD
:1019A800FFF7DCFF4FF00053002207930748089227
:1019B8004FF4807301A9029206920B9303F02CFB5B
:1019C80008B1FFF7CBFF0DB05DF804FB94010020D0
:1019D8000028004010B5044690B03822002102A823
:1019E8000FF024F82268194B9A422CD14FF4803317
:1019F800029302A84FF480730F9303F02BF908B1F8
:101A0800FFF7ACFF4FF0B0430220D3F8902042F428
:101A18000042C3F890209A6D42F480629A659B6DEB
:101A2800002203F4806311460193019B01F01CFF1F
:101A3800022001F04BFF00222A20114601F014FF7A
:101A48002A2001F043FF10B010BD00BF002800405D
:101A58007047000008B501F099FA044B0120C3F85B
:101A68008800BDE8084002F0FDBB00BF0004005834
:101A780001F093BA08B501F090FABDE8084000F00B
:101A88002BBD08B501F082FABDE80840012100200D
:101A980002F098BB70477047FEE7FEE7FEE7FEE7F7
:101AA800FEE770477047704770470000014803F031
:101AB800A5BB00BF94010020012002F06FBB0220EB
:101AC80002F06CBB014802F0D7B800BFF801002053
:101AD800402002F063BB0000014803F051BF00BF83
:101AE80058020020014803F0BDB900BF940100204E
:101AF800014803F0ACBD00BFE0010020F0B587B09D
:101B080000244FF0B0430594DA6C42F00102DA6425
:101B1800DB6C03F00103012500932026032701A9AC
:101B28004FF09040009B0395CDE90165049702F0C2
:101B380001FA402301A94FF09040CDE90134CDE9E5
:101B4800035702F0F7F9224631464FF0904002F071
:101B580017FB07B0F0BD00002DE9F843DFF86480FB
:101B680019491A4F0446D8F80000FEF78DFF1649A8
:101B78000546FEF789FF01462846FFF741F9D7F8E1
:101B8800009006462046FFF72FF84946FEF77AFFF1
:101B98003146FFF781F84946FEF776FFFFF7F2F97D
:101BA800314604464FF07E50FEF76CFF2946FFF79A
:101BB80073F8C8F800002046FFF716F8386020468A
:101BC800BDE8F883000000206F12833ACC010020A2
:101BD8000D4B0E4A1B68B3FBF2F3DBB258434FF0D0
:101BE800E023002258619A611A6942F001021A61E1
:101BF8001A6902F00112012AFAD01A6922F00102C8
:101C08001A6100229A6170477800002000127A0059
:101C1800012238B540214FF0904002F0B1FA01207E
:101C2800FFF7D6FF202100224FF0904002F0A8FADB
:101C380040214FF0904002F09DFA0128F8D0182476
:101C48000025012220214FF0904002F099FA01204E
:101C5800FFF7BEFF202100224FF0904002F090FADB
:101C680040214FF0904002F085FA6D00012804F100
:101C7800FF344FF0010008BF0135FFF7A9FF14F04A
:101C8800FF04DED1012220214FF0904002F078FAC3
:101C98000120FFF79DFF202122464FF0904002F0DF
:101CA8006FFA85F4000038BD13B5FFF7B1FF084C93
:101CB80020602068FFF750FF20602368009300220F
:101CC800044B114602200EF07FF902B010BD00BF90
:101CD800D8010020500C010808B5FFF70FFFFFF7E7
:101CE800E3FF0A2000F076F9BDE80840FFF7DCBF03
:101CF80007B5FFF78DFF0E4B18600E4B1A68904220
:101D080013D91B68C01AFEF773FF0B49FFF778F861
:101D1800FFF712F9FFF720FF084B00221860114661
:101D28000090074B02200EF04FF903B05DF804FB5A
:101D3800DC010020D80100200000C043D4010020AD
:101D4800770C0108F7B51D4F064614240025FFF748
:101D5800CFFF3868FEF74CFF01462846FEF794FE91
:101D6800013C14F0FF040546F1D1FEF76DFB144B5E
:101D78000022FEF7EBFCFEF759FE124B38602246B4
:101D88000090214602200EF01FF90F4A3B6833608D
:101D980013601268D21A642A0DD9642B0BDDFFF781
:101DA80083FF642000F016F9FFF77EFF03B0BDE85B
:101DB800F040FFF79DBF03B0F0BD00BFD401002085
:101DC80000003440950C0108D0010020054808B5F2
:101DD8000823036003F058FA18B1BDE80840FFF77C
:101DE800BDBD08BDE00100204FF0B04307B55A6EF5
:101DF80042F001025A665B6E002203F00103019370
:101E080011463220019B01F02FFD322003B05DF80E
:101E180004EB01F05BBD00000CB407B5054A05AB47
:101E2800102101930EF0E0FC03B05DF804EB02B062
:101E3800704700BFAB0C010830B585B0044602A856
:101E48000D460EF0FDFABDF90C30064A009310213C
:101E5800029B2046FFF7E0FF2046FEF789F928801D
:101E680005B030BDAB0C01084FF0B04210B5936817
:101E780023F4004393600EF06BFB114B01241C709C
:101E880000F0AEF80EF036F80E480EF04DF80E4B96
:101E98004FF400421A6102200EF04CF8FFF78CFA5A
:101EA80000F004F9FFF718FF0EF03EF9214620462E
:101EB8000EF05AF921462046BDE810400EF03EB912
:101EC800EC010020411E0008004000580EF062B9E5
:101ED80008B5FFF779FA40F6B83398420CD8B0F550
:101EE800E16F0BD3FE23A0F5E16058434FF49663EE
:101EF800B0FBF3F0C0B208BDFE20FCE70020FAE713
:101F08007FB5684600F0B6F80198FFF715F800B2FB
:101F180007B05DF804FB0000194A38B5D2F88035DF
:101F2800591C044619D101F03FF8054601F048F85C
:101F3800054401F03FF82B0EE3712B0CA3712B0A1B
:101F48006371030EE370C0F30742C0F307232571E2
:101F5800C0B2A2706370207038BD190AC371817154
:101F6800190C1B0E41710371D2F88435C370D2F875
:101F78008405C0F30722C0F30743000EE9E700BF5A
:101F88000070FF1F38B5094BD3F880350360013363
:101F9800054609D101F008F8044601F00BF8444061
:101FA80001F00EF844402C6038BD00BF0070FF1FE0
:101FB800012102200EF0C2B8002102200EF0BEB8A6
:101FC80000207047024B187808B100F0A7B8704796
:101FD800EC01002082B00190019802B000F03AB9FB
:101FE800F0B5224A224CD2F8903043F4804389B0AD
:101FF800C2F8903000F0EAFF00F0F0FF00F0F6FFC2
:10200800012304930323069300254FF0B04305955D
:102018000795DA6C42F00202DA64DA6C02F0020226
:102028000292029ADA6C42F00202DA64DB6C03F084
:10203800020301934FF4805703A92046019B03979D
:102048004FF4005601F076FF03A92046039601F0ED
:1020580071FF2A463946204602F092F82A46314650
:10206800204602F08DF809B0F0BD00BF0008005806
:102078000004004810B50446FFF7C0F9074BA360F9
:1020880040F30F20FEF7B4FD054B064A2360064BCC
:102098006060C4E90323002010BD00BF000048426F
:1020A80000007A440D093E00AB030500002070478C
:1020B800014B1868704700BFF001002003207047EB
:1020C80008B501464FF47A7200238002890DFEF7A5
:1020D80079FF08BD4FF47A73A0FB0303800A40EA36
:1020E80083507047034B98689A689042FBD1C0436D
:1020F800704700BF0028004008B5FFF7F3FF014B09
:10210800186008BDF001002008B5FFF7EBFF024B8F
:102118001B68C01A08BD00BFF0010020024B1878E8
:1021280008B1FFF7DFBF7047F401002010B5074B77
:10213800074C0122DA654FF48071204602F058FE00
:102148004FF0FF332363002010BD00BF002800407C
:102158009401002002460021014803F060B800BF46
:102168009401002002460121014803F058B800BF3D
:102178009401002010B58CB02C220021044601A83F
:102188000EF054FCFFF7D2FF0C4B0D481B681C44A3
:102198000023089306934FF00053E443079301226A
:1021A8004FF4807301A902940B9302F035FF08B134
:1021B800FFF7D4FB00200CB010BD00BFF0010020D9
:1021C8009401002038B50546FFF78CFF022104462C
:1021D800074803F02BF8C4F309024FF47A71A2FB05
:1021E8000121920AA30A2A8043EA805038BD00BF21
:1021F800940100200148002103F018B89401002040
:102208000148012103F012B894010020F8B50F4DE0
:102218002E78CEB90E4C4FF0FF372763FFF7A0FB9F
:10222800FFF784FF4FF48071204602F0E1FD20465D
:10223800276302F09FFF32462046022102F0EFFF9B
:10224800FFF75AFF01232B700020F8BDF40100208E
:1022580094010020014610B54FF47A7200238002E1
:10226800890DFEF7AFFE0146FFF73CFF0446FFF776
:1022780039FF031B8B4200D310BD00BFF7E70EF0F8
:102288006FBA000010B5064C0221204602F0CEFFBE
:102298000221421C2046BDE8104002F0C0BF00BF2A
:1022A800940100201648174A08B54FF4E133C0E9F5
:1022B800002300230C22C0E90233C0E90523C0E94A
:1022C8000733C0E90933036104F03FF908B1FFF7A8
:1022D80045FB0B48002104F0B0FA08B1FFF73EFBBC
:1022E8000748002104F0C9FA08B1FFF737FB044892
:1022F80004F083FA18B1BDE80840FFF72FBB08BD0A
:10230800580200200044004070B596B006461422DA
:10231800002103A80EF08AFB3822002108A80EF03D
:1023280085FB32682B4B9A4251D10223089308A8A7
:10233800294B0A9302F08EFC08B1FFF70FFB4FF010
:10234800B04300259A6D254C42F400329A659A6D87
:1023580002F400320292029ADA6C42F00102DA6464
:10236800DB6C03F001030193019B0C220223CDE9EE
:1023780003230323CDE9055303A907234FF0904016
:10238800079301F0D7FD164925621423C4E9001309
:102398001023C4E9023520468023C4E90435C4E982
:1023A800065501F0F3FA08B1FFF7D8FA0B481021E7
:1023B80001F0B8FC08B1FFF7D1FA2520F467002234
:1023C8000221A66201F050FA252001F07FFA16B02A
:1023D80070BD00BF0044004004000C00F80100205C
:1023E8005800024002680C4B9A4210B5044612D1BC
:1023F8004FF0B0420C21936D23F4003393654FF0F6
:10240800904001F043FEE06F01F032FBBDE8104060
:10241800252001F069BA10BD0044004008B50A46FD
:102428000146024803F010FA002008BD58020020B7
:1024380013B5114B114C18604FF40013009302AB05
:1024480013E90600204604F07CF92368DA69D10311
:10245800FCD4DA695202FCD59A68084842F4800232
:102468009A6004F0B4F906490448012204F022F9FC
:10247800002002B010BD00BFEC020020580200206E
:10248800F402002008B5074B1860FEF7F5FFFFF7C8
:1024980009FF054AD2F8803043F00063C2F8803063
:1024A800002008BDF00200200008005808B54FF0D1
:1024B800B04308489A6B42F400329A639A6B22F44C
:1024C80000329A63FFF78EFF0F2001F00DFA00200B
:1024D80008BD00BF5802002008B5074804F035F8C9
:1024E80008B1FFF73BFA054801F050FA18B1BDE80A
:1024F8000840FFF733BA08BD58020020F801002051
:102508000268044B9A4203D1034B00201B6818470A
:10251800704700BF00440040F002002002680B4BE7
:102528009A4210B504460FD1094B1B682BB1D0F85D
:10253800902012B907480121984720460549BDE86F
:102548001040012204F0B6B810BD00BF004400409E
:10255800EC020020F402002008B5FFF785FCBDE876
:10256800084000F057BB4FF0FF300DF077BE7047C2
:10257800014BD870704700BF10000020014B187441
:10258800704700BF1000002007B5064B00221B5CF7
:1025980000931146044B02200DF016FD03B05DF8C0
:1025A80004FB00BF1E0D0108040D010808B5022038
:1025B80000210DF01BFEBDE8084001480EF07EB872
:1025C8004C040020002101200DF010BE10B542F28D
:1025D8001073084C002818BF0346074823600EF004
:1025E8001FF8216804480EF0A3F8BDE8104002481F
:1025F8000EF064B80C0000204C04002037B50446E7
:1026080038B390F9065035BB14480EF009F8144851
:102618002A464FF4006101F0B3FD124B2A462946C1
:1026280002200DF0D1FCE379012B0CBF0E4B0F4BB0
:102638000022114602200DF0C7FC94F905300193E1
:1026480094F9043000930022094B114603200DF041
:10265800BBFC03B030BD074BEAE700BFF80200201F
:1026680000040048220D0108370D0108540D010827
:102678008A0D0108710D010808B50E4B1B78022B55
:1026880003D1002108200DF0B1FD0B4800224FF4C2
:10269800004101F075FD084800224FF4007101F077
:1026A8006FFDBDE80840044800224FF4006101F0C6
:1026B80067BD00BF740000200004004802480022E3
:1026C8004FF4004101F05CBD0004004802480022BC
:1026D8004FF4007101F054BD000400480A46014956
:1026E800FFF728B800F0030870B51F4801224FF41F
:1026F800004101F045FD1C4801224FF4007101F032
:102708003FFD01224FF40061174801F039FD1748D9
:102718000DF086FF04F012FD044650B10022144B60
:10272800114602200DF050FCBDE8704011480DF034
:10273800C5BF114D114B0246014602200DF044FC65
:1027480001260F4B2E702246214602200DF03CFC3C
:102758000C4804F087FB2878314604F0DBF803487E
:102768000DF0ACFFE0E700BF000400484C04002077
:10277800B30D01083404002074000020D10D0108B5
:10278800E50D0108100000202DE9F04391B0FFF796
:102798009FFB044604F0B8F9054600287CD103A83D
:1027A800FFF768FC09A8FFF7CDFA099B00930122FF
:1027B800594B294602200DF007FC584B0094012282
:1027C800294602200DF000FC0498554CFEF7B4FB96
:1027D80000B20122534B0090294602200DF0F4FB71
:1027E8000223059823705049FEF756FAFEF7CAFBF4
:1027F80086B20498FEF7A0FB4C4907B20398FEF78F
:102808004BFA4949FEF7FCFAFEF7BCFB484A6368F5
:1028180012781A706368C0F307225A706368987058
:102828006368DF706368320A1A7163685E71414ECB
:102838003378082B01D0012B40D8626800239371AC
:102848006268D3716268137253720A23099A6168C5
:10285800120ACA54626809991A44023351706370A3
:10286800354C637A63B104F03BF9012808D120465E
:102878000DF0D6FE314800224FF4006101F080FCD3
:10288800F1782748002204F055F9014688BB012257
:102898002B4B10460DF098FB00242A480DF0C0FE83
:1028A800294B28481968A14238BF21460DF040FF3E
:1028B80024480DF003FF11B0BDE8F083DDE9068779
:1028C800D4F80490FFF704FB89F8060063684FEA20
:1028D8002842DA7163684FEA28221A723A149A7207
:1028E8003A1283F80980DA721F735D739D730F23A0
:1028F800ACE70631D0D104F0EDF804460028CBD07F
:1029080001224FF47A730021B0FBF3F310460093D1
:102918000E4B0DF059FBC0E7040E0108180E010814
:1029280004000020230E0108000020410000C842D6
:102938004003002010000020F80200200004004896
:102948002E0E01084C0400200C0000203D0E01084A
:1029580002484FF4006101F018BC00BF00040048B1
:1029680000B503468DB000282CD0407802280AD044
:1029780003282AD0164B0022114602200DB05DF81C
:1029880004EB0DF021BB1A7F0B92DA7E0A929A7E35
:1029980009925A7E08921A7E0792DA7D06929A7DEB
:1029A80005925A680492DA68039293F91420029205
:1029B800B3F9122001921B7C00930022054B1146AB
:1029C8000DF002FB0DB05DF804FB034BD3E700BF2D
:1029D8005B0E0108720E0108E40E010801284FF091
:1029E80000020CBF024B034B114602200DF0ECBA5B
:1029F800030F0108150F010808B504F0A8FB80B9FA
:102A080004F06EF801280CD1BFF34F8F0549064B2F
:102A1800CA6802F4E0621343CB60BFF34F8F00BF74
:102A2800FDE708BD00ED00E00400FA051FB5044607
:102A3800002837D00378002B34D001224FF40071DE
:102A48001E4801F09DFB1E480DF038FE002211467D
:102A58001C4B02200DF0B8FA94F91830039394F93E
:102A68000A300293237C0193E36800930022114605
:102A7800154B03200DF0A8FA0022144B1146032031
:102A88000DF0A2FA237A012B0ED1617A104A114B6C
:102A9800002918BF13460022009311460E4B03204D
:102AA8000DF092FA04B010BD00220C4B1146032021
:102AB80004B0BDE810400DF087BA00BF000400481C
:102AC800280300202E0F01085F0F0108900F01084E
:102AD8002A0F0108290F01089D0F0108AE0F0108F0
:102AE800F0B5054687B00C46002937D02C4801229E
:102AF8004FF4004101F044FB2A480DF0DFFD267831
:102B08009EB1002D4AD06B682E7873B1022E27D063
:102B1800032E0AD16A78012A07D11878012802D031
:102B2800022800D008B904F0CFF8237C052B15D86B
:102B380094F90A20059294F9092004921A4A52F845
:102B48002330039394F90830CDE901630022E36848
:102B580000931146154B03200DF036FA07B0F0BD6F
:102B68006F78012FE1D11D78114B05F001051D701B
:102B780065B92A460F4B294603200DF025FA2A4647
:102B880007484FF4006101F0FBFACEE70022114636
:102B9800094B03200DF018FA3A46F1E72E46C4E730
:102BA8000004004810030020FC100108CF0F0108A2
:102BB80040030020BC0F0108C60F010838B50446C1
:102BC8000D4607484FF40061FEF7D4FD30B92A4698
:102BD80021460348BDE83840FEF7D2BC38BD00BFE7
:102BE80000F0030810B504F047FB10F1080F07D1F7
:102BF800064B0022BDE81040114602200DF0E4B952
:102C0800013001D1024BF4E710BD00BF16100108D6
:102C18002C100108F0B587B00024012603274F4B7C
:102C2800029422462146CDE9006702200225059438
:102C38000DF0CAF90523CDE900532246484B02940A
:102C4800214628460DF0C0F9464B009622462146FB
:102C5800CDE9017428460DF0B7F905A9204604F01E
:102C68005BFA059BC3F307220292C3F307421B0ECC
:102C78000192009322463C4B214628460DF0A4F9C8
:102C880005A9304604F048FA059BDAB20392C3F36B
:102C980007220292C3F307421B0E019200932246B9
:102CA800324B214628460DF08FF9314B31480094BC
:102CB80022464FF4FA710DF055FC2F4B2F48009423
:102CC80022464FF4FA710DF04DFC2D4B2D4800941F
:102CD80032464FF4FA710DF045FC2046FEF74AFCE7
:102CE80008B1FEF73BFE284B009400224FF4FA612E
:102CF80026480DF037FC264A002101200DF032FB52
:102D0800244A002102200DF02DFB234A0021042033
:102D18000DF028FB214A002108200DF023FB00F0CC
:102D280059F81F491F4804F0ADF91F4804F09AF8F4
:102D380014480DF0C3FC1D4B0021187803F0EAFD80
:102D48001B4900941B4B09681B4800220DF00AFC24
:102D580019480DF0B3FC07B0F0BD00BF44100108DE
:102D68006510010886100108A7100108C81001089D
:102D7800D526000828030020C526000810030020D7
:102D880059290008F8020020812600083404002090
:102D9800716C000891270008ED2B0008F126000847
:102DA800000003012800002010000020740000200B
:102DB8000C000020B52500084C040020022804D08F
:102DC800402806D10021042001E0002108200DF050
:102DD8000DBA7047044B0022C3E9022240F22111C8
:102DE8000122C3E9002170476404002000487047AD
:102DF8006404002000F034B800F072B800F0A4B801
:102E080000F0A4B800F0A4B800F0A4B80D488546B6
:102E180000F0A5F80C480D490D4A002302E0D458EB
:102E2800C4500433C4188C42F9D30A4A0A4C00230C
:102E380001E013600432A242FBD30DF0FFFDFEF760
:102E480081FDFEE700800020000000201001002026
:102E5800C81B01081001002060160020FEE70000D2
:102E68002DE9F04186B000244FF0B0430594DA6CA8
:102E78001A4D42F00402DA64DB6C039403F0040395
:102E88000093009B10270123CDE9017301A90323B7
:102E9800284604934FF0200801F04CF801A9284671
:102EA8000826CDF8048001F045F801A928460196C6
:102EB80001F040F822464146284601F061F92246D1
:102EC8003946284601F05CF928462246314601F089
:102ED80057F9204606B0BDE8F08100BF0008004859
:102EE80008B5032812D8DFE800F002131A260022DA
:102EF8001448082101F044F900221248102101F079
:102F08003FF900220F48202101F03AF9002008BDBE
:102F180001220C48082101F033F90122EDE70122D2
:102F28000848082101F02CF901220648102101F077
:102F380027F90122E6E701220248082101F020F9D9
:102F48000022F2E70008004800207047012070477F
:102F580001207047002814BF16200F2070477047C3
:102F680010B5032000F06EFC01F08CFA064B1860D7
:102F78000F20FFF725F8044618B9FEF78CFD204608
:102F880010BD0124FBE700BF780000204FF0E022CD
:102F9800136923F00203136170474FF0E0221369AD
:102FA80043F0020313617047014BD3F89005704753
:102FB8000070FF1F014BD3F8940570470070FF1F86
:102FC800014BD3F8980570470070FF1F024A5368F9
:102FD80043F0010353607047002004E0024A53683D
:102FE80043F0020353607047002004E0024A53682C
:102FF80043F0040353607047002004E08068C0F386
:1030080080007047F7B5002301930446002800F0BC
:10301800E980856D25B9FEF779F9E56584F854509E
:1030280023689A68D00040F1A1809A68D10000F125
:10303800B480A26D42F01002A265E26D42F0010276
:10304800E26501251846FFF7D9FFA26D02F01002CC
:10305800024340F0C980A26D206922F4817242F0D7
:103068000202A2659A68D2075DD4226BA67E94F804
:103078002CC0003A18BF01221703D4E902120A43F0
:10308800217E42EA8132617E42EAC13242EA463218
:10309800002842EA4C02B4BF20F000414FF400116E
:1030A8003A430A4394F82010012903D1002E76D11F
:1030B80042F48032616A21B1A66A01F4E0713143B9
:1030C8000A43D968E66C21F4FE3121F4FF711143FB
:1030D800D96094F83C206168012A01F0404C4CEA20
:1030E800060609D1D4E910273A433243A66C324385
:1030F80042EA0C0242F001061F693E4A3A40324356
:103108001A6121F00042B2F1804F0CD0B1F1004FAA
:1031180009D0394ED6F8082701F4701122F470123C
:103128000A43C6F808275A69666BA16B22F00702A2
:1031380032435A615A6922F0700242EA01125A6116
:10314800002835D19A6A62F00F029A625B6903F02F
:1031580007039E423CD10023E365A36D23F00303DC
:1031680043F00103A365284603B0F0BD9A682349DC
:1031780022F0104222F0170242F080529A60204A50
:103188001268B2FBF1F2013252000192019A002A50
:103198003FF44BAF019A013AF7E7002552E7A16DDA
:1031A80041F02001A165E16D41F00101E16581E790
:1031B800B0F5001FCAD19A6AE269013A92006FF02D
:1031C8000F0102F01C0201FA02F2216E0A43BCE769
:1031D800A36D23F0120343F01003A365E36D43F0DE
:1031E8000103E3650125BEE7A36D43F01003A36562
:1031F800F8E700BF02FCFF1F00200140400D03005C
:1032080078000020F8B54569082D04460E460AD016
:103218000368DB68D80705D5A36D43F02003A365D1
:103228000120F8BD0425FEF7CDFE074623681A687D
:103238002A4220D0A26D42F40072A265DA6812F424
:10324800406F14D1A27E92B91A6812070FD518469A
:10325800FFF7D4FE20BB5A6822F00C025A60A26D18
:1032680022F4807222F0010242F00102A265227E5D
:10327800FAB10020D5E7711CD9D0FEF7A3FEC01B18
:10328800B04201D8002ED1D123681B682B40CDD184
:10329800A26D84F8543042F00402A2650320C0E70E
:1032A800A26D42F02002A265E26D42F00102E265E1
:1032B800DDE70C221A60DCE70368186C7047000031
:1032C800F7B50023019390F85430012B044600F021
:1032D800C08005680269012380F854302846FFF74A
:1032E8008DFE002840F0AF80D1E90030022822F09E
:1032F80004027ED0B2F1004FC3F3110E35D1AA6A91
:1033080042EA0E02AA628A68686902EA032222F087
:103318007C4222F0FF0220EA03210A43002B6A6163
:103328001DDA4D4A4D4DD2F80817AB4201F0E07056
:1033380043D10D0213D4D2F8083723F0E0730343C6
:1033480043F40003C2F80837454B1A68454BB2FBF3
:10335800F3F20C2302FB03330193019B53BB0020C0
:10336800002384F8543003B0F0BD226E00F01F072C
:103378004FF00F0C0CFA07FC6FEA0C0622EA0C0C53
:10338800BEF1000F11D1C3F38462BA4042EA0C02C5
:1033980022668008E26901309042B4D8A86AC3F373
:1033A8008362BA4006403243ACE793FAA3F2B2FA1A
:1033B80082F2EAE7019B013BCEE72B4DAB420BD1F2
:1033C800C901CCD4D2F8083723F0E073034343F0A3
:1033D8008073C2F80837C2E7244DAB42BFD14B0215
:1033E800BDD4D2F8083723F0E073034343F48003D5
:1033F800EFE7B2F1004F01BFAA6AC3F311018A4394
:10340800AA62002BABDA154813498342D1F8082782
:1034180009D1D1F8083702F0A07223F0E0731A43FB
:10342800C1F808279BE71048834204D1D1F8083730
:1034380002F44002F1E70D48834290D1D1F80837F1
:1034480002F0C072E9E7A26D42F02002A2651846B8
:1034580086E7022087E700BF00200140001000B087
:1034680078000020400D0300004000B8002000B4A0
:10347800026838B504461046FFF7C0FD08B90020B9
:1034880038BD9368990707D4936823F0004323F065
:10349800170343F010039360FEF794FD0546236875
:1034A8009B685B07EBD5FEF78DFD401B0228F6D91C
:1034B80023689B685A07F2D5A36D43F01003A365F0
:1034C800E36D43F00103E3650120D9E773B50023F9
:1034D800026801939368DD07044602D5002002B014
:1034E80070BD9168214B194209D0A36D43F01003B8
:1034F800A365E36D43F00103E3650120EFE79368FB
:1035080023F0004323F0170343F001039360184BA3
:10351800D3F8083718021CD4637E012BDED0FEF7DF
:1035280051FD144E054622681368DB07D6D493680C
:10353800D9075FBF9368334043F001039360FEF7F8
:1035480041FD401B0228EED923681B68DA07EAD43C
:10355800CBE7094B094A1B68B3FBF2F3013301932C
:10356800019B002BD8D0019B013BF8E71700008096
:1035780000200140E8FFFF7F78000020400D030095
:1035880038B504460068FFF739FD054620BB94F8B6
:103598005430012B20D0012384F854302046FFF703
:1035A80095FFB0B9A36D226823F4706323F001037B
:1035B80043F48073A3651C23E065136084F854000A
:1035C800936823F0004323F0170343F00403936048
:1035D80038BD84F85450FBE70220F9E7026838B593
:1035E800936891680446C80701D4002038BD99073C
:1035F800FBD4936803F00503012B19D1936823F0DA
:10360800004323F0170343F002039360032313607E
:10361800FEF7D8FC054623689B68DB07E5D5FEF76F
:10362800D1FC401B0228F6D923689B68DA07F2D53B
:10363800A36D43F01003A365E36D43F00103E36555
:103648000120D3E770B5044600284BD0836D43F0C2
:1036580002038365FFF70CFF054668B92046FFF7AC
:10366800BDFF054608B90123A3652268936823F0C6
:10367800104323F01703936023685A6822F4677293
:1036880022F003025A6040F29F321A60D968164A43
:103698000A40DA601A6922F040421A615A6922F037
:1036A80007025A611A6A02F0F0221A625A6A02F094
:1036B800F0225A62DA6A02F0F022DA629A6A0B4A57
:1036C80000269E62D2F8083723F0FE73C2F8083746
:1036D8002046FDF72FFEE6652666A66584F8546049
:1036E800284670BD0125FBE700023E83002001400B
:1036F80010B590F85430012B044615D0012380F8FA
:103708005430FFF7B5FE58B92046FFF767FF38B9C0
:10371800A36D23F4807323F0010343F00103A36531
:10372800002384F8543010BD0220FCE7F7B50023CD
:10373800019390F85430012B04467FD0012380F880
:103748005430FFF74BFF23689A6812F001020546D0
:1037580007D0A36D43F01003A365002384F8543009
:103768002DE0A16D364F21F4817141F00201A16570
:10377800DE68D96826F4FF4626F07C0621F400416D
:10378800360421F00301360CD960082099683940C5
:1037980041F0004199609968002913DA01990131D3
:1037A80001910199B1F52E3FF5D3A36D23F01203D2
:1037B80043F01003A365002384F8543001252846FC
:1037C80003B0F0BDD3F8B410013801F07F010A440A
:1037D800DCD199681A48014041F001019960D3F899
:1037E800B41021F07F0141EAD202C3F8B4209A68EC
:1037F800024042F002029A60FEF7E4FB07462368A3
:103808009A68D20708D4DA683243DA60A36D23F0E5
:10381800030343F001039FE7FEF7D4FBC01B022814
:10382800EDD923689B68D907E9D5A36D43F0100348
:10383800A365E36D43F00103E365BFE70225BEE737
:10384800E8FFFF7F0749CA6822F4E0620302120416
:1038580003F4E063120C134343F0BF6343F40033F3
:10386800CB60704700ED00E0164B30B5DC68C4F360
:103878000224C4F10703251D042B28BF0423062DA9
:103888004FF0FF358CBF033C002405FA03F321EA0F
:103898000303A54022EA0502A340002843EA0203E5
:1038A800ACBF00F16040084A4FEA0313B8BF00F00C
:1038B8000F00DBB2AABF00F56140135480F8003353
:1038C80030BD00BF00ED00E014ED00E0002807DB8C
:1038D800044A4109012300F01F00834042F82130C7
:1038E800704700BF00E100E000280CDB43090649EF
:1038F80000F01F0020330122824041F82320BFF34B
:103908004F8FBFF36F8F704700E100E070B5D0E9CB
:1039180013456560446D14B1D0E916456560D0E97A
:10392800105404F01C060124B4406C600468636001
:103938008368102B0BBFA260A160E160E26070BDDC
:103948000268416CD3B210B5083B1424B3FBF4F3FE
:103958000B4CA24288BF0B4A21F0030199BF01F129
:10396800804202F50232521807338264064AC26462
:1039780003F01F03012202FA03F3036510BD00BF21
:10398800070402401C0802408008024038B500289D
:103998005CD002682E4B9A424FF014014AD82D4B46
:1039A8001344B3FBF1F32C499B00C0E91013022325
:1039B80080F825301368056923F4FF4323F070036A
:1039C8001360D0E9024323432B43456911682B4315
:1039D80085692B43C5692B43056A2B430B43136049
:1039E800FFF7AEFFB4F5804F04BF00234360436880
:1039F800816C03F07F020A60D0E91314013B032BAA
:103A08004C601ED8154B1649816513449B00012153
:103A1800013A01FA02F200214365C2651960114BAF
:103A28005A6400230122C36380F8243080F82520DB
:103A3800184638BD0C4B1344B3FBF1F30B499B00FC
:103A4800B3E70023C0E91533C365EAE70120F0E7CF
:103A580007040240F8FFFDBF000002403F8200104B
:103A68004009024000090240F8FBFDBF0004024083
:103A780038B5002841D00268136823F001031360A9
:103A88001F4B9A424FF0140130D81E4B1344B3FB1E
:103A9800F1F31D499B00C0E91013012403F01C0336
:103AA80004FA03F3002515604B60FFF749FF836CA8
:103AB80041681D60D0E913325A604A1E032A06D8AD
:103AC800124B0B449B0094401D60114B5C64002317
:103AD800C363C0E91533C0E90B33C0E90D33C365CF
:103AE80080F8253080F82430184638BD094B134437
:103AF800B3FBF1F308499B00CDE70120F5E700BFD0
:103B080007040240F8FFFDBF000002403F8200109A
:103B180000090240F8FBFDBF0004024070B590F8B0
:103B28002450012D04463BD090F825600125AE4273
:103B380080F824504FF000062CD1022580F825503B
:103B48000568C6632E6826F001062E60FFF7DEFEC4
:103B5800036BBBB12B6843F00E032B60A36C1A6890
:103B6800D20342BF1A6842F480721A60636D1BB1B7
:103B78001A6842F480721A602B6843F001032B60C4
:103B8800002070BD2B6823F004032B602B6843F0E2
:103B98000A03E2E78023C36380F824602846F0E73D
:103BA8000220EEE7034640B190F82520022A06D00D
:103BB8000422C263002280F8242001207047026892
:103BC800806C116821F00E011160016821F4807188
:103BD8000160116821F001011160D3E9100202F0BF
:103BE8001C0101228A404260D3E9132151605A6DB9
:103BF80032B1116821F480711160D3E91621516046
:103C08000122002083F8252083F82400704708B596
:103C180090F82530022B03D00423C363012008BD8C
:103C280003681A6822F00E021A601A6822F001026C
:103C38001A60826C136823F480731360D0E9101340
:103C480003F01C02012393404B60D0E913325A6001
:103C5800436D33B11A6822F480721A60D0E91632C3
:103C68005A60012380F82530002380F82430836BC4
:103C780003B198470020D2E770B4426C046C036823
:103C880026681D6802F01C020421914031420FD0C1
:103C980015F0040F0CD01A6892065EBF1A6822F05D
:103CA80004021A60036B6160002B33D070BC1847A4
:103CB80002219140314217D015F0020F14D01A6832
:103CC800940606D41A6822F00A021A60012280F8C3
:103CD8002520114A93428CBF104B114B5960002389
:103CE80080F82430C36ADFE708219140314211D0BF
:103CF80029070FD5196821F00E011960012303FA6D
:103D080002F26260C36380F82530002380F8243013
:103D1800436BC9E770BC7047800002400004024052
:103D28000000024060B10268C806136805D5C902E0
:103D38004CBF43F4801323F48013136000207047B2
:103D4800012070470A4A536943F4802330B5536110
:103D5800EFF3108472B60023CD58C5500433B3F581
:103D6800807FF9D11369DB03FCD484F3108830BD5C
:103D780000400058064B5A69002ABFBF054A9A609E
:103D880002F188329A60BABF5869C00F00207047A4
:103D98000040005823016745044B5A6942F000422D
:103DA8005A615869C043C00F704700BF00400058AF
:103DB80070B50546FEF706F9124E04463369D90375
:103DC80013D43369DA0744BF012232614CF2FA3264
:103DD800134011D10B4E306910F480200BD0FEF740
:103DE800F1F8001BA842F6D304E0FEF7EBF8001B3D
:103DF800A842E3D3032070BD024A1361024A01209E
:103E08005360F8E700400058740400202DE9F041A1
:103E1800184D98462B78012B06460C46174626D097
:103E280001232B704FF47A7000236B60FFF7C0FFFB
:103E3800A0B9012E16D1104A536943F0010353610A
:103E48002760BFF36F8FC4F804804FF47A70FFF7D0
:103E5800AFFF094A536923EA0603536100232B7015
:103E6800BDE8F08139462046FFF76CFFEDE70220F8
:103E7800F6E700BF7404002000400058054A536963
:103E880023F47E7343EAC00040F4803040F002001F
:103E980050617047004000582DE9F041234F3B78AE
:103EA800012B054688463FD001233B704FF47A70BA
:103EB80000237B60FFF77CFF044688B92B68042B3E
:103EC80013D11B4A536943F4803343F0040353610D
:103ED8004FF47A70FFF76CFF0446154B1A681B689D
:103EE80000233B702046BDE8F0814FF0FF33C8F84F
:103EF80000306E68D5E901321344B3420AD930461E
:103F0800FFF7BCFF4FF47A70FFF752FF50B1C8F8C3
:103F180000600446064A536923F47E7323F00203C3
:103F28005361DAE70136E5E70224DBE77404002091
:103F3800004000582DE9F04F524C00234FF00F0974
:103F48000A6832FA03F501D1BDE8F08F012505FAB8
:103F580003F818EA020200F08E804E68032706F084
:103F680003054FEA430E07FA0EFC6F1E012F6FEA96
:103F78000C0C32D8876807EA0C0ACF6807FA0EF7E4
:103F880047EA0A078760476827EA0808C6F3001760
:103F98009F4047EA08074760C76807EA0C088F6828
:103FA80007FA0EF747EA0807022DC76017D14FEA4C
:103FB800D30800EB880803F0070AD8F820704FEA06
:103FC8008A0A09FA0AFB27EA0B0B0F6907FA0AF7AC
:103FD80047EA0B07C8F8207001E0032DDCD1076819
:103FE80005FA0EF507EA0C073D4316F4403F056055
:103FF80041D023F0030707F1804707F5803703F026
:10400800030CBD684FEA8C0C4FF0070E0EFA0CFE3D
:10401800B0F1904F25EA0E0E2FD01B4DA8422ED09E
:1040280005F58065A84214BF0725022505FA0CF599
:1040380045EA0E05BD602568D74316F4801F0CBFFE
:104048003D4015432560656816F4001F0CBF3D40D0
:1040580015436560D4F8805016F4803F0CBF3D408E
:104068001543C4F88050D4F88450B60354BF3D407B
:104078001543C4F88450013362E70025D6E70125CB
:10408800D4E700BF0008005800040048374A2DE96B
:10409800F04F00234FF0010A4FF0070B4FF00F09C4
:1040A80031FA03F401D1BDE8F08F0AFA03FC1CEAE7
:1040B800010654D023F0030404F1804404F580344D
:1040C80003F00307A568BF000BFA07F8B0F1904F9B
:1040D80008EA050E45D0264DA84244D005F580656E
:1040E800A8420CBF02250725BD40754517D1D2F857
:1040F800805025EA0605C2F88050D2F8845025EA97
:104108000605C2F88450156825EA06051560556845
:1041180025EA06055560A56825EA0805A56005682D
:1041280003265C0006FA04F423FA06F6254300EB9E
:104138008606056003F00705376AAD0009FA05F53C
:1041480027EA05073762856825EA0405856045681A
:1041580025EA0C054560C56825EA0404C4600133F6
:104168009EE70025C0E70125BEE700BF000800580C
:10417800000400480369194214BF01200020704759
:104188000AB18161704781627047436901EA03029D
:1041980021EA030141EA024181617047044AD1687A
:1041A800014208B502D0D060FEF708FE08BD00BF86
:1041B80000080058024A136843F48073136070477C
:1041C800000400580D4B10B55B690C4628B99A05D8
:1041D80007D500F027F820B110BD9B0501D400F0E9
:1041E80019F8074A1369012C23F00403136101D15C
:1041F80030BFF1E740BF20BF20BFEDE70004005803
:1042080000ED00E0024B186800F4C060704700BF82
:1042180000040058024A136843F48043136070474F
:10422800000400580C4A136823F4804313600B4BB6
:104238001B6832214B430A49B3FBF1F351698905E5
:1042480000D533B9536913F4007F14BF032000204D
:104258007047013BF2E700BF0004005878000020D7
:1042680040420F000B4A136823F0070343F0020390
:104278001360094B1A69012842F004021A6105D13A
:1042880030BF1A6922F004021A61704740BF20BF8C
:1042980020BFF6E70004005800ED00E04FF0B043FF
:1042A8001868C0F3404070474FF0B0431868C0F337
:1042B800400070474FF0B042536823F47F4343EA0D
:1042C8000023536070474FF0B0431868C0F3406054
:1042D800704700007FB54FF0B0432C4AD3F808313F
:1042E800C0F3031003F00F0352F82040284A52F895
:1042F8002330B4FBF3F4FFF785FF264B054693E81C
:104308000700B5F5007F04AB03E9070010D0224B86
:104318009C4218D303F5B70303F67F539C4229D96F
:1043280003F5741303F510639C4225D802230BE0B0
:104338001A4B9C4207D91A4B9C421BD903F53703E9
:1043480003F5D853F0E7002304AA02EB830353F8DC
:104358000C4C144D2B6823F0070323432B60FDF707
:1043680031FE06462B6803F007039C4206D1002065
:1043780004B070BD0123E7E70024EAE7FDF722FE59
:10438800801B0228EED90320F2E700BF14110108B0
:1043980074110108A80B0108C0CF6A00BFEA210107
:1043A8003F933402004000584FF0B04310B59A686C
:1043B800D96812F00C0205D00C2A4AD101F0030387
:1043C800012B51D14FF0B0412B480B6813F0080373
:1043D80006D00B6813F0080337D1D1F8941007E022
:1043E8000C68240756BFD1F894300968C3F3032337
:1043F80050F82330002A0CBF184600204FF0B04177
:104408008A6802F00C020C2A1ED1CA6802F0030264
:10441800022A2ED0032A06D10B68184A13F4801FEB
:10442800174B18BF13464FF0B042D068D168D26816
:10443800C0F306205843C1F302130133B0FBF3F075
:10444800530F0133B0FBF3F010BD0B68C3F3031334
:10445800CEE7042A05D0082A06D11B6813F4801376
:1044680005D006480023C9E700231846C6E70448D4
:10447800C4E7024BD7E700BF141101080024F40079
:104488000048E80108B5FFF78FFF4FF0B043044A32
:104498009B68C3F3031352F82330B0FBF3F008BD55
:1044A800741101082DE9F0410446002853D04FF05B
:1044B800B0439D68DE6803689B0605F00C0506F0AE
:1044C800030668D5026A1DB10C2D46D1012E44D1D0
:1044D800002A40D04FF0B043A16A1A68170756BFA8
:1044E800D3F894301B681B0903F0F00399421FD9D5
:1044F8000846FFF7EFFE00282DD14FF0B0421368B1
:1045080043F0080313601368A16A23F0F0030B4318
:104518001360606AFFF7CEFEFFF7B4FFAB4B18607D
:10452800AB4B1868FDF74CFD002834D0BDE8F0818E
:104538004FF0B042136843F008031360136823F088
:10454800F0030B431360606AFFF7B4FE0846FFF7F9
:10455800C1FE0028E0D00120E8E74FF0B043002A70
:1045680054D01A6842F001021A60FDF72BFD074685
:10457800FFF79AFE002842D04FF0B042136843F08C
:10458800080313601368A16A23F0F0030B43136058
:10459800606AFFF78FFE2368D80748D42368990715
:1045A80000F18C8023681E0740F1FA80A3694FF060
:1045B800B046002B00F0E180D6F89430E16903F0B2
:1045C8001002914200F0C48003F00302022AC2D014
:1045D800D80740F1B380D6F8943023F00103C6F829
:1045E8009430FDF7EFFC0746D6F89430990740F170
:1045F800A580FDF7E7FCC31B112BF5D904E0FDF7F7
:10460800E1FCC01B0228B3D903208FE71A6822F007
:1046180001021A60FDF7D6FC0746FFF745FE0028A1
:10462800B9D0FDF7CFFCC01B0228F6D9ECE7082D5E
:1046380003D00C2D05D1032E03D16368002BADD117
:1046480089E74FF0B043A1681A6822F480120A4340
:104658001A606268B2F5803F10D11A6842F480325D
:104668001A60FDF7AFFC0746FFF718FE002895D142
:10467800FDF7A8FCC01B6428F6D9C5E7B2F5041FEE
:1046880004D11A6842F400121A60E6E7196821F4A6
:1046980080311960196821F400111960002AE0D1ED
:1046A800FDF790FC0746FFF7F9FD00283FF476AFC9
:1046B800FDF788FCC01B6428F5D9A5E7042D2369FC
:1046C80003D00C2D0ED1022E0CD1002B3FF443AF9A
:1046D8004FF0B0426169536823F0FE4343EA016337
:1046E80053605FE74FF0B046BBB1336843F4807363
:1046F8003360FDF767FC074633685A0505D4FDF7B4
:1047080061FCC31B022BF7D97EE77368626923F04B
:10471800FE4343EA0263736044E7336823F480731B
:104728003360FDF74FFC074633685B057FF53AAF0A
:10473800FDF748FCC31B022BF6D965E74FF0B042E2
:10474800E169D2F8943023F010030B43C2F8943097
:104758004FF0B047D7F8943043F00103C7F89430CE
:10476800FDF730FC0646D7F894309A0718D4FDF7C1
:1047780029FC831B112BF6D946E7D6F8943023F091
:104788000103C6F89430FDF71DFC0746D6F89430AF
:104798009B0705D5FDF716FCC31B112BF6D933E78C
:1047A8002368580754D50B4F3B68D90514D4FFF735
:1047B80001FDFDF707FC06463B68DA050CD4FDF75A
:1047C80001FC831B022BF7D91EE700BF78000020ED
:1047D8007C00002000040058E3684FF0B046002B2E
:1047E80058D023F08003052B02BFD6F8903043F051
:1047F8000403C6F890304FF0B046FDF7E3FBD6F857
:10480800903043F001030746C6F8903041F28838EB
:10481800D6F890309B0705D4FDF7D4FBC31B43455E
:10482800F6D9F1E6E36823F00403812B1BD1FDF7E9
:10483800C9FBD6F8903043F08003C6F8903007469D
:104848004FF0B04641F28838D6F89030180504D5B4
:10485800E36A002B4AD1002068E6FDF7B3FBC01BD2
:104868004045F1D9D0E6FDF7ADFBD6F8903023F0FE
:104878008003C6F8903007464FF0B04641F28838BA
:10488800D6F890301905E3D5FDF79CFBC01B4045D1
:10489800F6D9B9E6FDF796FBD6F8903023F08003F9
:1048A8000746C6F8903041F28838D6F890301A0595
:1048B80016D4FDF787FBD6F8903023F00103C6F82D
:1048C800903007464FF0B04841F28836D8F890301B
:1048D8009B07BDD5FDF776FBC31BB342F6D993E61C
:1048E800FDF770FBC01B4045DFD98DE60C2D4ED07F
:1048F800022B4FF0B0431A6822F080721A6033D14D
:10490800FDF760FB0546FFF7DEFC38BBD4E90C3148
:104918004FF0B0420B43D0682D4901400B43E16B87
:104928000B43216C0B43616C0B43A16B43EA0123DE
:10493800D360136843F080731360D36843F08053E7
:10494800D360FDF73FFB0446FFF7BDFC002882D18A
:10495800FDF738FB001B0A28F6D955E6FDF732FBB0
:10496800401B0A28CFD94FE6FDF72CFB0446FFF77A
:10497800AAFC30B94FF0B042164BD1680B40D36057
:1049880069E7FDF71FFB001B0A28F0D93CE6012B5D
:104998003FF4E1AD4FF0B043D868236B00F0030259
:1049A8009A427FF4D8AD626B00F0700393427FF4B3
:1049B800D2ADA26B00F4FE43B3EB022F7FF4CBAD74
:1049C800636C00F06040C01A18BF0120AEE500BF5C
:1049D8008C80C111FCFFFEEE2DE9F0410D46044626
:1049E80010B90120BDE8F081754E336803F0070364
:1049F8008B4216D32368980727D54FF0B047A26893
:104A0800BB6823F0F0031343BB60FDF7DBFA0646EF
:104A1800BB68D90319D4FDF7D5FA831B022BF7D944
:104A280011E0336823F007030B433360FDF7CAFA3C
:104A38000746336803F00703AB42DBD0FDF7C2FA41
:104A4800C01B0228F5D90320CCE723689A0616D59F
:104A58004FF0B0476269D7F8083123F0F0031343E9
:104A6800C7F80831FDF7AEFA0646D7F808319B03B8
:104A780005D4FDF7A7FA831B022BF6D9E3E72368D1
:104A8800580617D54FF0B047A269D7F8083123F078
:104A98000F0343EA1213C7F80831FDF793FA0646E5
:104AA800D7F80831D90305D4FDF78CFA831B022BFC
:104AB800F6D9C8E723685A0713D54FF0B047E2681C
:104AC800BB6823F4E0631343BB60FDF77BFA06463B
:104AD800BB689B0305D4FDF775FA831B022BF7D936
:104AE800B1E72368180714D54FF0B0472269BB68AF
:104AF80023F4605343EAC203BB60FDF763FA06463A
:104B0800BB68590305D4FDF75DFA831B022BF7D95F
:104B180099E72368DA070FD4294C236803F00703C1
:104B2800AB4239D8FFF7AEFC264B1860264BBDE8E0
:104B3800F0411868FDF744BA6268022A1DD1FFF7F0
:104B4800ADFB00283FF44DAF4FF0B04641F2883836
:104B5800B36823F003031343B360FDF733FA074642
:104B6800B368626803F00C03B3EB820FD4D0FDF78F
:104B780029FAC01B4045F3D965E7032A02D1FFF79C
:104B8800A2FBDEE712B9FFF78FFBDAE74FF0B0437D
:104B98001B685B05D8D424E7236823F007032B435D
:104BA8002360FDF70FFA0646236803F00703AB42BC
:104BB800B8D0FDF707FA801B0228F5D943E700BFF4
:104BC80000400058780000207C00002008B5FFF75E
:104BD80059FC4FF0B043044A9B68C3F3022352F8D0
:104BE8002330D84008BD00BF5411010808B5FFF7AD
:104BF80049FC4FF0B043044A9B68C3F3C22352F800
:104C08002330D84008BD00BF541101084FF0B0430D
:104C1800D3F89000C0F3400070474FF0B04102094C
:104C2800D1F8883002F47F22000123EA020300F45D
:104C38007F200343C1F8883070474FF0B041020C21
:104C4800D1F88830120423EA020343EA0040C1F88D
:104C5800880070470368DA0370B5044639D5FFF752
:104C6800A9FAFDF7AFF9614E05463368DB0532D581
:104C78004FF0B043616BD3F8902002F44072914238
:104C88001DD0D3F89010D3F8902042F48032C3F8A6
:104C98009020D3F8902021F4407022F480328D07C0
:104CA800C3F89020C3F8900009D5FDF78BF941F2BD
:104CB80088360546FFF7AAFF012840F090804FF09C
:104CC800B042616BD2F8903023F440730B43C2F8C2
:104CD8009030002605E0FDF775F9401B0228C4D97D
:104CE80003262568E8070AD54FF0B0416268D1F875
:104CF800883023EA124392B21343C1F88830A907D7
:104D08000AD54FF0B041A268D1F8883023EA12439F
:104D180092B21343C1F88830AA0609D54FF0B042C1
:104D28002169D2F8883023F440630B43C2F88830F5
:104D3800AB0502D5206AFFF780FF680502D5606AD7
:104D4800FFF77BFF290502D5A06AFFF776FF6A0601
:104D580002D56069FFF761FF2B0602D5A069FFF74E
:104D68005CFFE80502D5E069FFF757FFE90610D5B3
:104D78004FF0B042E168D2F8883023F440730B4317
:104D8800C2F88830B1F5807F02BFD36843F08073E2
:104D9800D3602A040ED54FF0B042216BD2F8883088
:104DA80023F040430B43C2F8883019B9D36843F065
:104DB8008073D3606B0410D54FF0B042E16AD2F82B
:104DC800883023F040530B43B1F1005FC2F88830BC
:104DD80003D1D36843F48033D360304670BDFDF708
:104DE800F1F8401BB0427FF665AF79E70004005840
:104DF80030B590F82C30012B02464FF0020022D03B
:104E0800174B82F82D00CA24012582F82C505C62C9
:104E180053245C62B1F5807F146B996914D121F435
:104E280088519961596C24F0010421F000415964BA
:104E38001463DD650A4BFF2159620020012382F8C3
:104E48002D3082F82C0030BD21F408519961D96CBD
:104E580024F0020421F00041D9641463D865E9E71D
:104E68000028004070B50B4E036B756D1D40EA07B6
:104E7800044603D50123F365FDF701FAAB0704D512
:104E88000223F365204600F0C9F9012384F82D3088
:104E980070BD00BF0028004038B50A4CE36823F015
:104EA8002003E360FDF78EF80546E3689B0601D50D
:104EB800002038BDFDF786F8401BB0F57A7FF4D99D
:104EC8000320F6E700280040F8B5114DEC6814F00F
:104ED800400406461AD1EB6843F08003EB60FDF707
:104EE80071F823460746EC6814F0400401D1032BFF
:104EF80001D11846F8BDFDF765F8C01BB0F57A7FFB
:104F0800234684BF032386F82D30ECE70023F0E71F
:104F18000028004038B50F4CE36823F08003E360B5
:104F2800A3699B06054606D4FFF7B6FF10B1032018
:104F380085F82D0038BDA36923F02003A361FFF78E
:104F4800ABFF10B1032085F82D00A36943F02003BF
:104F5800A361EFE70028004038B5044600284BD08D
:104F680090F82D3003F0FF021BB980F82C20FCF7D5
:104F780031FD0223214D84F82D30EB68DB0636D451
:104F8800CA236B6253236B622046FFF79DFF10B163
:104F9800FF236B6238BDAB6923F08E6323F04003B7
:104FA800AB6121696368AA690B431343A269134380
:104FB800AB61D4E9022343EA02432B61D4E9093106
:104FC800EA680B4322F4F8521343EB602046FFF7DC
:104FD800A1FF0028DCD1D4E90713AA690B4322F00A
:104FE8006042134362691343AB61FF236B62012381
:104FF80084F82D300020CDE70120CBE700280040C1
:105008000023092803D840EA0310C0B270470A38C1
:105018000133C0B2F5E700002DE9F04790F82C30D5
:10502800012B05464FF0020069D0012385F82C308A
:105038004E4B85F82D00DE6806F44076B6F5807F85
:1050480078D04C69087891F8019091F802A091F80D
:105058002470002A55D19B6913F0400308BFCB7018
:10506800FFF7CEFF80464846FFF7CAFF0246504684
:10507800FFF7C6FF81463846FFF7C2FF0B6ACF78B5
:10508800234343EA875343EA090343EA084343EACD
:10509800022343EA0063354ACA2050625320506213
:1050A8008C6A8869B4F5807F946945D124F4885462
:1050B80094610124D465B6F5807F09BFCB69136478
:1050C8000343536418BF5064284B4A681A672A6B15
:1050D80042F001022A639A6942F488529A61244A8A
:1050E800D2F8803043F40033C2F880301F4BFF22DF
:1050F8005A620020012385F82D3085F82C00BDE880
:10510800F087B4F1803F07D0B4F5000F04D09B6955
:1051180013F0400308BFCB700B6ACA781C4344EAFB
:105128000A0444EA004343EA092343EA825343EA70
:105138000763B0E70023AEE724F40854946102241F
:10514800D465B6F5807F09BFCB6993640343D36404
:1051580018BFD064054B4A685A672A6B42F00202AE
:105168002A639A6942F40852B8E700BF0028004051
:105178000008005890F82C20012A03464FF002003E
:1051880012D00A4A83F82D00CA2151625321516274
:10519800916941F020019161FF21516200200122B3
:1051A80083F82D2083F82C00704700BF00280040AA
:1051B80090F82C20012A03464FF0020019D00D4A1E
:1051C80083F82D00CA2151625321516291690A481E
:1051D80041F080019161D0F8801041F48021C0F83D
:1051E8008010FF2151620020012283F82D2083F8CE
:1051F8002C0070470028004000080058064B5A6DE4
:10520800520610B5044603D54022DA65FDF73AF890
:10521800012384F82D3010BD002800407047890014
:1052280001F1804101F531410A607047890001F1BF
:10523800804101F53141086870470000034AD2F8FF
:10524800903043F40043C2F890307047000400588F
:10525800034AD2F8903023F40043C2F890307047E4
:1052680000040058074B1A6822F040021A6040F404
:1052780041704FF4B85218605A601A6842F0400200
:105288001A6070470000015837B5054600284ED00F
:10529800837903F0FF046BB1032C0BD0254B4FF43B
:1052A80000629A612868FFF7DDFF002401232B7153
:1052B800AC602FE000236B712846FCF795FD1E4A71
:1052C800D2F8903043F48053C2F89030002CE5D1E6
:1052D80002234FF0B042AB71D2F8943023F400436C
:1052E800C2F89430154B1B681C214B43DB0C64211E
:1052F8004B430193019B93B90124AC60FFF79EFFD8
:105308000C4B9A6842F400629A604FF400629A610A
:10531800002CC7D00123AB71204603B030BD019BE0
:10532800013B0193D2F894305B04E3D4E6E701240F
:10533800F2E700BF00040058000800587800002079
:1053480037B5174D2B6802461C204343DB0C6420FD
:10535800434314480193019B93B901209060114C79
:1053680021732B681C214B43DB0C64214B430193B5
:10537800019B6BB9012090600A4BDB6803B030BD1C
:10538800019B013B019383689C07E4D50020E6E775
:10539800019B013B0193A368DB07E9D5ECE700BF5C
:1053A800780000200000015837B5184D2B680246D8
:1053B8001C204343DB0C6420434315480193019BA5
:1053C800A3B901209060124CFF2323732B681C257E
:1053D8006B43DB0C64256B430193019B73B901207C
:1053E80090600B4BDB680B7003B030BD019B013B39
:1053F800019383689C07E2D50020E4E7019B013B09
:105408000193A368DB07E8D5EBE700BF780000202D
:10541800000001580E4B0F491B681822534382B0F5
:105428001B0D6422534301934B69019AC3F3800314
:1054380022B902238360012002B07047019A013A21
:1054480001924A69920701D5002BEDD10020F3E7BC
:10545800780000200004005807B50379012B0FD10C
:105468000A4B1B68182253431B0C0193FFF7F0FEED
:10547800019B013B0193019B002BF9D1FFF7DEFE55
:1054880003B05DF804EBFFF7C5BF00BF780000204C
:10549800F8B51E468379012B154604460F46DAB245
:1054A8002DD14379012B2AD0022342718371FFF752
:1054B800D3FF0D212046FFF7CBFEFFF741FF390A46
:1054C8002046FFF73DFFF9B22046FFF739FF2E448B
:1054D800B5420ED12046FFF7B1FEFFF79BFFA0684B
:1054E80001230038A3714FF0000318BF0120637136
:1054F800F8BD15F8011B2046FFF722FFE8E7022058
:10550800F6E7F8B51E468379012B154604460F4683
:10551800DAB22FD14379012B2CD04271FFF79CFFCF
:105528001D212046FFF794FEFFF70AFF390A20469F
:10553800FFF706FFF9B22046FFF702FF00212046D9
:10554800FFF7FEFE2E44B5420ED12046FFF776FE49
:10555800FFF760FFA06801230038A3714FF0000334
:1055680018BF01206371F8BD29462046FFF71CFFCC
:105578000135E8E70220F6E7F8B51F468379012BE5
:10558800154604460E46DAB22CD14379012B29D0B0
:105598004271FFF761FF06F0EF03A3F18402534263
:1055A8005341237131462046FFF752FEFFF7C8FEEC
:1055B8002F44AF4210D1FFF741FE842E02D020467F
:1055C800FFF728FFA06801230038A3714FF00003FC
:1055D80018BF01206371F8BD15F8011B2046FFF7BD
:1055E800AFFEE6E70220F6E7F8B51E468379012B01
:1055F800154604460F46DAB227D14379012B24D049
:105608004271FFF729FF39462046FFF721FEFFF7D1
:1056180097FE00212046FFF793FE2E44B5420ED197
:105628002046FFF70BFEFFF7F5FEA06801230038C0
:10563800A3714FF0000318BF01206371F8BD29461C
:105648002046FFF7B1FE0135E8E70220F6E737B557
:105658000023ADF8043001AA022312210546FFF702
:10566800C3FFBDF80440022364BA01AAA4B21946D4
:105678002846FFF781FFE20702D528460AF03EFBDD
:10568800A30702D528460AF03FFB600702D5284643
:105698000AF064FB210702D528460AF065FBE206FA
:1056A80002D528460AF066FBA30602D528460AF06A
:1056B8004FFB600602D528460AF02CFB210606D5CA
:1056C80014F4807118BF012128460AF029FBA205AD
:1056D80002D528460AF034FB630402D528460AF0AE
:1056E8004FFB03B030BDF8B51E468379012B154634
:1056F80004460F46DAB227D14379012B24D04271F0
:10570800FFF7AAFE0E212046FFF7A2FDFFF718FEBD
:1057180039462046FFF714FE2E44B5420ED12046E6
:10572800FFF78CFDFFF776FEA06801230038A37110
:105738004FF0000318BF01206371F8BD15F8011B75
:105748002046FFF7FDFDE8E70220F6E7F8B51E461C
:105758008379012B154604460F46DAB22BD14379DB
:10576800012B28D04271FFF777FE1E212046FFF754
:105778006FFDFFF7E5FD39462046FFF7E1FD002103
:105788002046FFF7DDFD2E44B5420ED12046FFF737
:1057980055FDFFF73FFEA06801230038A3714FF0C5
:1057A800000318BF01206371F8BD29462046FFF7A2
:1057B800FBFD0135E8E70220F6E7026852E8003F02
:1057C80023F0C00342E8003102680029F5D102F154
:1057D800080353E8003F23F4000302F1080C4CE8E7
:1057E80000310029F3D12023C0F888307047000029
:1057F80010B5026852E8003F23F4907342E8003184
:1058080002680029F5D10F4C02F1080353E8003F64
:10581800234002F1080C4CE800310029F4D1C36E92
:10582800012B07D152E8003F23F0100342E8003172
:105838000029F7D12023C0F88C300023C3664367C2
:1058480010BD00BFFEFFFFEFF8B504461346D4F8BD
:105858008850202D32D1F1B1EAB1E06FA4F856207A
:10586800A4F8542000262122C4F890602165C4F8C9
:105878008820226888B1124FC762124F0763124FFF
:105888002832C0E90D76FEF749F930B11023C4F883
:105898009030C4F888500120F8BD236840221A626D
:1058A800226802F1080353E8003F43F0800302F145
:1058B800080141E800300028F3D1EDE70220EBE7CA
:1058C800D55800081D5900082959000808B503468D
:1058D800806A1B681B6813F0200317D1A0F85630A4
:1058E800026802F1080353E8003F23F080030832FE
:1058F80042E8003102680029F2D152E8003F43F043
:10590800400342E800310029F7D108BDFCF7F8FD53
:10591800FBE7704708B5806AFFF7FBFF08BD7047D3
:10592800806A38B50468D0F88830D0F88C50A268FE
:10593800120606D5212B04D10023A0F85630FFF714
:105948003CFFA3685B0606D5222D04D10023A0F8EE
:105958005E30FFF74DFFD0F8903043F01003C0F8E9
:105968009030FFF7DCFF38BD08B5806A0023A0F847
:105978005E30A0F85630FFF7D2FF08BD7047000030
:105988000368D9691A682DE9F04140F60F063142DB
:105998009D68044610D18E0640F1978002F02006DB
:1059A80005F080573E4300F09080436F002B00F0D5
:1059B8008580BDE8F0411847AB4EAC482E401040FA
:1059C800304300F08280CF0709D5D00507D50120E4
:1059D8001862D4F8900040F00100C4F890008F07D6
:1059E80009D5E80707D502201862D4F8900040F0DE
:1059F8000400C4F890004F0709D5E80707D504202C
:105A08001862D4F8900040F00200C4F890000F0724
:105A18000BD502F02000304307D008201862D4F8D4
:105A2800900040F00800C4F890000E050AD5500117
:105A380008D54FF400601862D4F8903043F0200382
:105A4800C4F89030D4F89030002B37D08B0609D5A5
:105A580002F0200205F080552A4303D0636F0BB192
:105A6800204698472668D4F89020B36802F02802A8
:105A780003F0400353EA0205204621D0FFF7B8FEA1
:105A8800B3685F0617D5226802F1080353E8003FA0
:105A980023F04003083242E800310029F3D1D4F85A
:105AA800800040B1724B8363FEF7B1F830B1D4F88F
:105AB8008000836B7DE72046FFF731FFBDE8F0816A
:105AC800FFF72DFFC4F89050F8E7E06E012840F08A
:105AD8008980CE0640F18680D00640F1838010226E
:105AE8001A629A6851064BD5D4F8802011684A6822
:105AF80092B2002AE2D0B4F85C009042DED9A4F851
:105B08005E200A6892062FD453E8002F22F4807290
:105B180043E800210029F7D103F1080252E8002FD9
:105B280022F0010203F1080040E800210029F3D126
:105B380003F1080252E8002F22F0400203F10800A6
:105B480040E800210029F3D12022C4F88C20E16626
:105B580053E8002F22F0100243E800210029F7D172
:105B6800D4F88000FEF71EF802232367B4F85E30ED
:105B7800B4F85C10C91A89B22046FFF7FFFE9DE70A
:105B8800B4F85E20B4F85E00B4F85C1080B292B24B
:105B9800002893D0891A89B200298FD053E8002FA2
:105BA80022F4907243E800200028F7D1314D03F128
:105BB800080252E8002F2A4003F1080646E80020B0
:105BC8000028F4D12022C4F88C206067E06653E8EE
:105BD800002F22F0100243E800200028F7D102230A
:105BE8002367C9E7CF0209D56E0207D54FF48012A3
:105BF80020461A62BDE8F04100F0A0BD08060BD5AA
:105C080002F0800005F40005284305D0A36F002B9F
:105C18003FF454AF2046CCE64F0611D556060FD5B3
:105C280053E8002F22F0400243E800210029F7D171
:105C38002023C4F88830A1672046FCF761FC3DE7C3
:105C48000D0206D5500004D52046BDE8F04100F00D
:105C580077BDCB017FF532AF002ABFF62FAF2046C4
:105C6800BDE8F04100F06BBD010000102001000408
:105C780071590008FEFFFFEFD0F88C20B0F86010D3
:105C8800222A08B5036855D15B6A826D0B401370F0
:105C9800836D01338365B0F85E30013B9BB2A0F899
:105CA8005E30B0F85E309BB2002B42D1026852E8F9
:105CB800003F23F4907342E8003103680029F5D1CE
:105CC80003F1080252E8002F22F0010203F1080C48
:105CD8004CE800210029F3D12022C0F88C20184A72
:105CE80041679342016705D1C26E012A0ED0FCF7C5
:105CF80015FC1EE05A681102F6D553E8002F22F071
:105D0800806243E800210029F7D1EDE70022C2664E
:105D180053E8002F22F0100243E800210029F7D1B0
:105D2800DA69B0F85C10D20644BF10221A62FFF795
:105D380025FE08BD9A6942F008029A61F9E700BF9A
:105D480000800040D0F88C20B0F86010222A08B5F6
:105D5800036852D15A6A1140826D22F8021B82658B
:105D6800B0F85E20013A92B2A0F85E20B0F85E204A
:105D780092B2002A40D153E8002F22F4907243E8EF
:105D880000210029F7D103F1080252E8002F22F080
:105D9800010203F1080C4CE800210029F3D120226C
:105DA800C0F88C20174A41679342016705D1C26E3B
:105DB800012A0ED0FCF7B2FB1EE05A681102F6D594
:105DC80053E8002F22F0806243E800210029F7D130
:105DD800EDE70022C26653E8002F22F0100243E8E4
:105DE80000210029F7D1DA69B0F85C10D20644BF67
:105DF80010221A62FFF7C2FD08BD9A6942F0080234
:105E08009A61F9E7008000402DE9F84F0368B0F87F
:105E18006060D3F81CB01F689D68D0F88C20222AD7
:105E2800044640F0B980B0F8683043B1DFF87491A7
:105E3800DFF874A14FF000081BF0200F20D1B4F850
:105E48005E309BB2D3B1B4F868209A4216D9226862
:105E580002F1080353E8003F23F08053083242E878
:105E6800003122680029F2D1504B636752E8003FA5
:105E780043F0200342E800310029F7D1BDE8F88F4C
:105E88002368A26D5B6A33401370A36D0133A36569
:105E9800B4F85E30013B9BB2A4F85E302368D3F8B7
:105EA8001CB01BF0070F2ED01BF0010F09D0F9050D
:105EB80007D501221A62D4F8902042F00102C4F8F2
:105EC80090201BF0020F09D0EA0707D502221A62B8
:105ED800D4F8902042F00402C4F890201BF0040F7C
:105EE80009D0E80707D504221A62D4F8903043F0A5
:105EF8000203C4F89030D4F8903023B12046FFF75D
:105F08000EFDC4F89080B4F85E309BB2002B93D19C
:105F1800226852E8003F23F4807342E80031236886
:105F28000029F5D103F1080252E8002F02EA09021C
:105F380003F1080040E800210029F3D1202253454D
:105F4800C4F88C20616721670AD05A68110207D506
:105F580053E8002F22F0806243E800210029F7D19E
:105F6800E26E012A14D10022E26653E8002F22F0E3
:105F7800100243E800210029F7D1DA69B4F85C106F
:105F8800D20644BF10221A622046FFF7F7FC53E7F7
:105F98002046FCF7C3FA4FE79A6942F008029A6173
:105FA8006CE700BFFEFFFFEF00800040815C000847
:105FB8002DE9F84F0368B0F86060D3F81CB01F688B
:105FC8009D68D0F88C20222A044640F0B780B0F8AB
:105FD800683043B1DFF87091DFF870A14FF0000826
:105FE8001BF0200F20D1B4F85E309BB2D3B1B4F8C7
:105FF80068209A4216D9226802F1080353E8003F44
:1060080023F08053083242E8003122680029F2D197
:106018004F4B636752E8003F43F0200342E80031EA
:106028000029F7D1BDE8F88F2368A26D596A31407D
:1060380022F8021BA265B4F85E20013A92B2A4F8D5
:106048005E20D3F81CB01BF0070F2ED01BF0010FF9
:1060580009D0F90507D501221A62D4F8902042F038
:106068000102C4F890201BF0020F09D0EA0707D5F7
:1060780002221A62D4F8902042F00402C4F8902058
:106088001BF0040F09D0E80707D504221A62D4F8D8
:10609800903043F00203C4F89030D4F8903023B124
:1060A8002046FFF73CFCC4F89080B4F85E309BB201
:1060B800002B95D1226852E8003F23F4807342E810
:1060C800003123680029F5D103F1080252E8002FB6
:1060D80002EA090203F1080040E800210029F3D18F
:1060E80020225345C4F88C20616721670AD05A687A
:1060F800110207D553E8002F22F0806243E80021FF
:106108000029F7D1E26E012A14D10022E26653E891
:10611800002F22F0100243E800210029F7D1DA69A4
:10612800B4F85C10D20644BF10221A622046FFF76A
:1061380025FC55E72046FCF7F1F951E79A6942F04A
:1061480008029A616EE700BFFEFFFFEF0080004083
:106158004D5D000838B5044603682169A2681D68CA
:10616800C0690A4361690A437749024329400A43DF
:106178001A605A68E16822F440520A435A60734A26
:10618800A16993421CBF226A11439A6822F06E42A9
:1061980022F430620A439A60DA6A616A22F00F02D6
:1061A8000A43DA626A4A934219D14FF0B043694A06
:1061B800D3F8883003F0030343F44033934200F0EC
:1061C800B480B3F1031F24D0013A934240F0B58064
:1061D800B0F5004F40F08F80FEF7E6F86EE05E4ABB
:1061E80093421CD14FF0B0435C49D3F8883003F098
:1061F8000C0343F440228A4200F0978006D8002B13
:106208007CD0574B9A42E3D0012026E0B2F10C1F14
:10621800FAD1B0F5004F53D04FF4004075E04B4A27
:106228009342F1D14FF0B043D3F8883003F4406380
:10623800B3F5006F18D006D85BB1B3F5806FE3D122
:10624800FEF7B2F807E0B3F5406FDDD14FF4004038
:106258000BE0FEF7BBFC40B900204FF00113A3662A
:106268000023C4E91D3338BD3E4865683E4B626A69
:1062780005EB450133F81220B0FBF2F39942C3D87D
:10628800B3EB053FC0D800231946FAF79BFE090275
:1062980041EA10616B080002C0182A464FF000035B
:1062A80041F10001FAF78EFE304BA0F540729A4298
:1062B800AAD82368D860CFE7FEF788FC0028CBD09F
:1062C8006168294B626A33F81220B0FBF2F24B087E
:1062D80003EB42034FF6EF72B3FBF1F3A3F11001A6
:1062E800914291D823F00F02216892B2C3F342037E
:1062F8001343CB60B0E7FEF757F804E0B0F5004F62
:10630800DAD0FEF763FC0028A6D06368616A164AF3
:1063180032F81120B0FBF2F000EB5300B0FBF3F0C1
:106328004FF6EF73A0F11002C1E7B0F5004F0D482A
:10633800EBD1C5E7FEF75AFCC0E7B0F5004FF9D03E
:10634800FEF754FCDFE700BFF369FFCF0080004091
:1063580000380140020003000044004008000C001F
:1063680004000C000024F400B4110108FFFC0F0025
:10637800836ADA0710B506D50168C46A4A6822F448
:10638800003222434A609C0706D50168046B4A68BC
:1063980022F4803222434A60590706D50168446BCB
:1063A8004A6822F4802222434A601A0706D5016807
:1063B800846B4A6822F4004222434A60DC0606D510
:1063C8000168C46B8A6822F4805222438A60990665
:1063D80006D50168046C8A6822F4005222438A6058
:1063E8005A060FD50168446C4A6822F48012224389
:1063F800B4F5801F4A6005D14A68846C22F4C00253
:1064080022434A601B0606D50268C16C536823F410
:1064180000230B43536010BD2DE9F843DDF82090AD
:1064280005460F46164698462A68D36937EA030395
:106438000CBF01230023B34201D0002029E0B9F1A9
:10644800FF3FF2D0FBF7BEFDA0EB080048452C68E3
:1064580002D8B9F1000F1ED154E8003F23F4D073DD
:1064680044E80032002AF7D104F1080353E8003F5A
:1064780023F0010304F1080141E80032002AF3D1B6
:106488002023C5F88830C5F88C30002385F884307F
:106498000320BDE8F88323685A07C5D5E3691B05BF
:1064A800C2D54FF40063236254E8003F23F4D0734D
:1064B80044E80032002AF7D104F1080353E8003F0A
:1064C80023F0010304F1080141E80032002AF3D166
:1064D8002023C5F88830C5F88C30C5F89030D4E74B
:1064E80073B504460026C0F89060FBF76BFD23687F
:1064F8001B681A07054619D423681B685B070AD569
:106508006FF07E43009300222B464FF48001204613
:10651800FFF782FFB0B900202023C4F8883084F840
:106528008400C4F88C30E06620670CE06FF07E438E
:106538000093324603464FF400112046FFF76CFFE4
:106548000028D9D0032002B070BD10B5044650B35E
:10655800D0F888301BB980F88430FBF7D5FE226864
:106568002423C4F88830136823F0010313602046FD
:10657800FFF7F0FD012816D0A36A13B12046FFF7F4
:10658800F7FE23685A6822F490425A609A6822F00B
:106598002A029A601A6842F0010220461A60BDE891
:1065A8001040FFF79DBF012010BD000030B5816588
:1065B8008168A0F85C200023B1F5805FA0F85E2018
:1065C800436735D10369002B40F2FF1318BFFF233F
:1065D800A0F860300023C0F890302223C0F88C3037
:1065E800016801F1080353E8003F43F00103083153
:1065F80041E800340368002CF2D1456E84680169D3
:10660800B5F1005F32D1B0F8685095422ED8B4F594
:10661800805F244A03D1244C002908BF22464267E0
:10662800B1B153E8002F42F4807243E80021F7E744
:1066380029B90369002B14BF7F23FF23C8E7B1F1F1
:10664800805FC5D10369002B14BF3F237F23BFE7B9
:1066580003F1080252E8002F42F0805203F10800CB
:1066680040E800210029F3D1002030BDB4F5805F57
:106678000E4A03D10E4C002908BF2246426741B199
:1066880053E8002F42F4907243E800210029F7D123
:10669800EAE753E8002F42F0200243E800210029EE
:1066A800F7D1E1E7115E0008B95F0008815C0008D6
:1066B8004D5D0008D0F88C30202B30B415D1B9B11D
:1066C800B2B100230468C3660A4B9C420AD06368CF
:1066D8001B0207D554E8003F43F0806344E80035C7
:1066E800002DF7D130BCFFF761BF022030BC7047E6
:1066F8000120FBE700800040436E30B52BB9012331
:10670800A0F86A30A0F8683030BD0368094D9A686F
:106718009968094C490FC2F342626B5C615CDB000B
:10672800B3FBF1F3A0F86A30AB5CA25CDB00B3FB0F
:10673800F2F3E7E7D4110108CC110108704770475C
:1067480070471FB504AB03E9060090F88430012BAD
:1067580004463AD0012380F884302423C0F88830D6
:1067680003681A6822F001021A609A6822F440123B
:106778000A439A6071B95A68BDF80C009DF80E106A
:1067880022F0100202435A605A6822F07F4242EA1D
:1067980001625A601A6842F001021A60FBF712FCA3
:1067A8006FF07E42034600924FF48001002220469B
:1067B800FFF732FE38B92023C4F88830002384F864
:1067C800843004B010BD0320F8E70220F9E790F800
:1067D8008430012B0FD0012380F88430016851E800
:1067E800002F42F0020241E80023002BF6D180F886
:1067F8008430184670470220704710B590F88430EE
:10680800012B044617D02423C0F8883003681A687F
:10681800196821F00101196042F000524FF000514F
:1068280041661A60FFF768FF2023C0F8883000200F
:1068380084F8840010BD0220FCE770B590F884301D
:10684800012B044617D005682423C0F888302E6829
:106858002B6823F001032B60AB6823F060431943D6
:10686800A960FFF749FF20232E60C0F88830002078
:1068780084F8840070BD0220FCE770B590F884307D
:10688800012B044617D005682423C0F888302E68E9
:106898002B6823F001032B60AB6823F06063194376
:1068A800A960FFF729FF20232E60C0F88830002058
:1068B80084F8840070BD0220FCE7000038B5084D5C
:1068C800052455F8043B2BB9013C14F0FF04F8D11A
:1068D800204638BDDB6898470028F5D0F9E700BFA7
:1068E800C8050020034BD870034B1B681B6C03B111
:1068F80018477047B0050020AC050020034B1874FA
:10690800034B1B685B6C03B118477047B005002048
:10691800AC050020F0B5314D314B95F90420314ECE
:1069280091B00C46012795F905108DF804700228DE
:106938008DF809208DF80A1010D18DF80800D8714B
:106948001C7202F063FD337803B114B101A803F09F
:10695800C1F9254B059A1A6011B0F0BD59714FF471
:1069680080711A71D9801C7233788DF8087053BB06
:106978001F2306A88DF81C208DF8183002F024FF7C
:1069880020238DF8183006A82B798DF81C3002F0DA
:106998001BFF22238DF8183006A86B798DF81C3060
:1069A80002F012FF21238DF8183006A86B798DF8B4
:1069B8001C3002F009FF29238DF8183006A80B4B6C
:1069C800079302F001FF02F021FD012306A88DF8CC
:1069D80018308DF81C3002F0F7FEB4E7B00500203F
:1069E800B00000208C040020800500200004000175
:1069F8007FB5092301A88DF8043003F06BF900383E
:106A0800044B059A1A6018BF0120404207B05DF890
:106A180004FB00BF8005002070B504460B461449EE
:106A280062784A700020A2780A7208701A884A723E
:106A38009A788A72DB780B746368CB600D4B1B689D
:106A4800DA6A2AB1237803F0FB030A2B00D09047B7
:106A5800094E002556F8043B1BB15B6A0BB1204672
:106A680098470135EBB2052B6DB2F3D170BD00BF6D
:106A780080000020AC050020C805002070B5044641
:106A880011480123037063784370A3788372E36825
:106A9800C360E378037623694376237943720B4B0B
:106AA8001B689B6A03B19847094E002556F8043BBA
:106AB8001BB19B690BB1204698470135EBB2052BFA
:106AC8006DB2F3D170BD00BF94000020AC0500206A
:106AD800C8050020014B1868704700BF80050020DA
:106AE80000B58BB0012368468DF8003002F046FDF2
:106AF80038B99DF80400003818BF01200BB05DF8C4
:106B080004FB0020FAE7000008B501F037FE40B9A1
:106B1800FFF7E6FF012806D0054B197AD879FFF769
:106B2800F9FE012008BDBDE80840FFF7C7BE00BF59
:106B3800B00000202DE9F04186B005460E46174604
:106B480001F01CFE002873D101F030FE044640B964
:106B5800FFF7C6FF01280AD03D4B197AD879FFF70D
:106B6800D9FE6FF00204204606B0BDE8F081DFF8D8
:106B7800E48088F80860003E18BF01268DF804609C
:106B8800354E687833798DF81230694602F094FCF6
:106B980000283FD08DF804400394ADF810406FF002
:106BA800060495E803002D4B83E80300337988F841
:106BB8000A30394601A803F091F9294B059A1A6061
:106BC80011283FD801A353F820F000BF3F6C0008FC
:106BD800396C00084D6C00084D6C00084D6C0008BD
:106BE8004D6C00084D6C00086B6B00084D6C00087C
:106BF8004D6C00084D6C0008336C00084D6C0008A3
:106C08004D6C0008396C0008396C0008396C0008B4
:106C1800536C00082B788DF808306B78ADF810307D
:106C28006B6803934FF0FF34BBE76FF005049AE7F6
:106C38006FF0010497E70B4B00221A70E31D18BF91
:106C4800144690E74FF0FF348DE76FF004048AE7AD
:106C5800B000002094000020B0050020A40000200F
:106C6800800500207F05002037B501F0A9FD134DF0
:106C7800052455F8043B4BB11A693AB19B682BB10E
:106C8800984718B155F8043C1B699847013C14F023
:106C9800FF04EED1FFF712FE68B9094D2B7853B106
:106CA800084BADF80040D978019422466846FFF7B2
:106CB80041FF00B92C7003B030BD00BFC8050020EB
:106CC8007F050020B005002030B58BB0044601F0E8
:106CD80055FD0546002835D1FFF702FF012834D1BC
:106CE80068468DF8005002F049FC40BB9DF804301E
:106CF800A34204D0012C22D0022C12D014B10020BF
:106D08000BB030BD002BFAD068468DF8044002F075
:106D18005BFDA0B90E4B1B681B6B002BEFD098478F
:106D2800EDE763B968468DF8044002F04DFD30B9CF
:106D3800074B1B681B6B002BE1D02046EFE74FF099
:106D4800FF30DDE76FF00100DAE76FF00200D7E708
:106D5800AC05002010B504468AB018B94FF0FF30D2
:106D68000AB010BD002368468DF8003002F006FC1A
:106D78000028F3D19DF804302370F1E77FB5002295
:106D88000B4620498DF8072001220A7042784A7084
:106D98000446002A33D102790A721A884A729A780C
:106DA8008A72DB780B740369CB60C378164D8DF853
:106DB8000830037B8DF80930836803932B68DB6AFE
:106DC8000BB102A898472B689B6B13B1227E02B1C6
:106DD80098470E4E052556F8043B1BB1DB690BB1ED
:106DE80020469847013D15F0FF05F4D10DF1070045
:106DF800FFF7B0FF637913B1054B01221A7004B095
:106E080070BD00BF80000020AC050020C805002030
:106E18007F05002010B504468AB018B94FF0FF303E
:106E28000AB010BD202368468DF8003002F0A6FB9A
:106E38000028F3D1024A9DF9043023701371EFE75B
:106E4800B005002000B58BB02323019068468DF86B
:106E5800003002F0B9FC003818BF012040420BB0E6
:106E68005DF804FB70B5654C01468EB018222046CB
:106E780007F0ECFB624B00221A70FBF7B7FF237890
:106E88004068012202FA03F1014004D15D4B084633
:106E980009F09AF8FEE75C495C481A4602F0F8F8EF
:106EA80018B14FF0FF300EB070BD272304A88DF83D
:106EB800103002F089FC564E564D002870D101233F
:106EC80033702B68DB690BB100209847272304A88F
:106ED8008DF8103002F052FB059B93F84820227081
:106EE80093F8182193F81A316270A370464BD3E9CE
:106EF800020107F09BFA05460028D2D1464E062328
:106F080004A88DF8103002F039FB059B736104A8C2
:106F180002F05AFC022304A88DF81030059602F0FE
:106F28002DFB0836032304A88DF81030059602F0CF
:106F380025FB0F2607F040FB012304A88DF8143029
:106F48008DF8106002F040FC10230DEB03008DF863
:106F580010308DF8145002F037FC04238DF81030EF
:106F680004A8A3788DF8143002F02EFC3A238DF88B
:106F7800103004A86369059302F026FC02A9207862
:106F88008DF8086004F0A2F8003818BF0120E071FD
:106F98001420FFF757FFE07903F062F9284682E7EB
:106FA80028238DF810302B681B6943B104A802F020
:106FB800E5FA2B6805981B6940F2D45198472723B6
:106FC80004A88DF8103002F0FFFB50B9012304A883
:106FD8008DF8103002F0D2FA9DF81430002B7FF4AF
:106FE8006EAF3378002B7FF46CAF052204A88DF8C0
:106FF8001020059302F0E8FB78E700BFB0050020F9
:107008007F050020DC110108840500209C05002074
:107018008C040020AC050020EC05002037B50023C7
:107028000D4601930446D0B900F0A8FB0190019BDE
:10703800D3B10F4A42F824300E4A9A620E4A1268B7
:10704800916B1963916C596392690C49D9625A61C1
:1070580028465B680A49F2229847002006E001A901
:1070680000F092FB0028E2D04FF0FF3003B030BDB3
:10707800C80500201D690008AC050020F969000852
:107088008D040020194B07B51860194B194A1A606E
:10709800194A5A60194A9A60194ADA60194B026803
:1070A8001A6042685A6082689A60C268DA60164A52
:1070B8001A6182695A61154BC26B5A60144A019170
:1070C80019609A601946134ADA600020FFF7A6FF94
:1070D80048B901A800F056FB003818BF012040420B
:1070E80003B05DF804FB4FF0FF30F9E7AC05002072
:1070F8009C050020856A0008856D000899710008C4
:10710800216A00088405002079B00008DC05002009
:10711800ED6800080569000849B118B1012804D0D4
:1071280000207047034B0B60FAE7034BFBE74FF077
:10713800FF307047000400010100010208B503F0A8
:10714800ABF8002814BF6FF00100002008BD08B597
:1071580002F084F9002814BF6FF00100002008BD78
:1071680010B504468AB018B94FF0FF300AB010BD08
:10717800212368468DF8003002F000FA0028F3D188
:10718800024A9DF9043023705371EFE7B0050020DF
:107198002DE9F0412F4D304F00232B7043786B7051
:1071A8003B689B6A8AB004460BB128469847DFF8CB
:1071B800AC80002658F8043B1BB11B6A0BB1204673
:1071C80098470136F3B2052B76B2F3D12378052B15
:1071D8002FD00B2B35D0012B25D1214C0623684607
:1071E8008DF8003002F0CAF90199E07907F064F9E6
:1071F80010B91C4B019A5A611B48FFF70BFE1B483C
:10720800FFF7AEFF6B788BB9A371194B5878FFF76E
:107218005BFD3B685B6A0BB1114898476B7813B903
:10722800E07907F0DBF90AB0BDE8F081FF23A3712C
:10723800EFE7104B01225A74227A9A74627ADA7450
:10724800F1E76378002BEED00AB0BDE8F041FFF714
:10725800CFBB00BF94000020AC050020C80500206B
:10726800B0000020EC050020B4000020B50000208C
:10727800B00500208000002030B58BB0FFF767FF15
:107288000446F0B903F0FCFE831C1DD0F8B9134D79
:107298002B685B69DBB1272368468DF8003002F064
:1072A8006DF92B6801985B694FF4BB61984703F04F
:1072B800F9FE78B92CB9094B1B68DB690BB10120C1
:1072C800984720460BB030BD6FF00704EFE74FF04A
:1072D800FF34ECE74FF0FF34F3E700BFAC050020C4
:1072E800014B1878704700BF20060020014B5878E2
:1072F800704700BF2006002070470000044B9A7AB0
:107308000AB101225A70034B5B6903B118477047F1
:1073180020060020BC00002073B5224C6378002BA7
:1073280033D009F039F966680546FFF7D3FB064400
:10733800AE4214D2A37A93B1E0228DF800208DF8E2
:107348000130217AE368019301226846FFF7F2FBD6
:1073580008B1073010D100236370A372656094F8F8
:107368003430EBB1002384F834300F4B5B6BBBB186
:1073780002B0BDE87040184740F2DC510B4809F0F4
:10738800D7F90A4809F09AF9E8E794F83520002A6D
:10739800E5D094F8360084F83530FFF795FCDEE741
:1073A80002B070BD20060020BC00002004060020AA
:1073B80037B5104D104CC8B1C1B16272012300221B
:1073C8002860E16023700D480D4B00924FF0FF31AB
:1073D80009F0C8F800250B4825822022294607F025
:1073E80049F96570A574A58603B030BD00232B60EC
:1073F8002370EFE71C06002020060020040600206A
:1074080005730008340600202DE9F0478E4C2378D8
:107418008CB0002B56D0C2780AB9837B13B1238A6B
:1074280001332382437B002B4CD0E02A4AD100232E
:10743800A372876897F80080B8F1220F27D8B8F1AF
:10744800220F30D8DFE818F04100FB0052005A0044
:1074580061006E0075008E009D00B400C7002F000B
:107468002F002F002F002F002F002F002F002F009C
:107478002F002F002F002F002F002F002F002F008C
:107488002F002F002F002F00C900D000D400B8F122
:107498007E0F00F0CC80B8F17F0F00F0DF80B8F1EC
:1074A8007D0F00F0AB80A57A002D00F05B81674C62
:1074B800637A3BB94FF47A71204609F039F92046CE
:1074C80009F0FCF80CB0BDE8F087E3680122002160
:1074D800A2721970A37AE1689818A0720620C8549D
:1074E800A37AE1689818A072CA54DCE7584B9B6AE3
:1074F800002BD8D0012102209847D4E77B7884F864
:107508003630012384F83530CDE704238DF8043074
:107518007B78003B18BF012301A88DF8083002F0E2
:1075280053F9C0E77878003818BF012002F098FEB8
:10753800B9E7484E0FCE01AD0FC50FCE0FC596E87F
:10754800070085E807007B780A2BACD8424A126806
:107558005268002AA7D00CA901EB830353F82C0C1E
:107568009047A0E77878431E012B9CD83A4B013806
:107578001B6818BF012020729B68002B93D0984786
:1075880091E7E26801230821A3721170627A057BF2
:10759800A17AAA4228BF2A46934284D285685A1CF7
:1075A800EB5CE56801334E1CA6726B54D3B2EDE771
:1075B800E3680122A27209221A70A37AE268218A7A
:1075C800581CA072D154A27A238AE1681B0A501C65
:1075D800A0728B5467E7238265E705238DF8043092
:1075E80001A802F077FB5EE7194BDB6A98475AE778
:1075F800194B78781B686075DB68BEE7037B072B3F
:107608007FF451AF06238DF80430B7F80130ADF898
:1076180008307B793A791B0443EA0223FA7813434A
:10762800642253430393BB798DF81030D8E73B228B
:1076380001A88DF804208DF8083002F0C5F8012360
:1076480084F834302FE700BF20060020040600200D
:10765800BC000020B40B01081C0600202A2301A846
:107668008DF8043001F08AFF94F80A90E6689DF8D6
:1076780008009DF809509DF80A709DF80BC09DF808
:107688000D309DF80E209DF80F109DF80CE009F1C3
:10769800010A84F80AA006F80980354E94F80A9081
:1076A8003668D4F80C8009F1010A84F80AA096F823
:1076B80003A008F809A094F80A90D4F80C8009F1FE
:1076C800010A84F80AA096F802A008F809A094F81C
:1076D8000A90D4F80C8009F1010A84F80AA096F8F7
:1076E80001A008F809A094F80A9009F1010A84F8A1
:1076F8000AA096F80080E66806F8098094F80A80DF
:10770800E66808F1010984F80A9006F808C094F8B8
:107718000AC0E6680CF1010884F80A8006F80C70C3
:10772800A77AE66807F1010C84F80AC0F555A57A2E
:10773800E6686F1CA7727055A07AE568461CA672A9
:107748002954A17AE0684D1CA5724254A27AE168D6
:10775800501CA0728B54A37AE268591CA17202F8DB
:1077680003E0A0E6034808F05BFF6570AAE600BFE7
:107778001C060020040600207047000000487047DF
:10778800BC000020002070474FF0FF307047000019
:10779800044B054A93F81831022B18BF062382F8C8
:1077A800903470470080002000070020034BD3F876
:1077B800483313B15B6903B11847704700070020CD
:1077C800034A137843F004031370FFF7EFBF00BFB9
:1077D8006C0600201FB50A4B8DF8090093F87C2031
:1077E8008DF80A2093F88C2093F848000D3202A9EE
:1077F8008DF8082003F06AFCC0B205B05DF804FB00
:107808000080002008B5074808F00AFF064B93F8E7
:107818001A2412B1012283F81924BDE80840FFF7A1
:10782800C5BF00BF000B00200007002010B50C4C9E
:10783800D4F8403343F08003C4F8403394F81A3442
:1078480013B10020FFF7DEFF94F8913423F0120300
:1078580043F0120384F89134BDE81040FFF798BF55
:10786800000700202DE9F041DFF8AC8098F81831C6
:10787800022B06460D4602D0284BDB6A984702F0D9
:10788800A6FD044628B1022002F097FD002002F070
:1078980099FD98F81831012B17D102F09AFD074687
:1078A80030B1002002F08AFD002002F08CFD3C4639
:1078B80002F091FD48B1002002F081FD002002F0A5
:1078C80083FDBDE8F041FFF763BF002CF9D1144CEC
:1078D80094F8902494F81A34BAB90BB184F8416436
:1078E800304602F017FFD8F82C0008F05FFED4F8F5
:1078F800B4339842E5D30B4808F092FE94F89134DB
:1079080043F0100384F89134DBE70BB184F8415459
:10791800284602F0FFFEF1E700800020101A010857
:1079280000070020980A0020074A10B5137843F092
:1079380002031370FFF73AFFBDE81040034B012222
:107948000021022008F040BB6C0600202512010827
:10795800074A10B5137843F008031370FFF726FFA2
:10796800BDE81040034B01220021022008F02CBB87
:107978006C060020351201082DE9F0410F46164625
:107988001D46804608F008FE0B4A0C4C13782781E8
:1079980023F0110343F01103C4E900081370668152
:1079A8002573FFF703FFBDE8F041054B01220021D5
:1079B800022008F009BB00BF6C0600205806002012
:1079C8004512010813B508F0E7FD0D4B6C46186029
:1079D800204608F035FD94E803000A4A0A4B83E87C
:1079E8000300137843F020031370FFF7DFFE074B03
:1079F80001220021022002B0BDE8104008F0E4BADC
:107A0800680600206C060020380A0020521201087F
:107A18002DE9F04192B0064602F0D9FC002840F06A
:107A28005881AD4D95F81831012B09D02B6BAB4C13
:107A380093B194F80431BBB1042B6FD0032003E059
:107A480002F0C7FC18B10F2012B0BDE8F08102F0B7
:107A5800C2FC0028EAD0F6E7B5F82031D4F81C2497
:107A6800013B53432B63E4E79D4803F060FA002889
:107A780040F0128194F80C3123802B6B0C930DF19C
:107A8800180895F839308DF83830404695F81C318B
:107A98008DF83A3008F0FAFCD5F82831009302AF97
:107AA80098E80600D5F82431384608F086FC97E8AF
:107AB80003000FAB83E80300EB6A0D9300238DF8F6
:107AC80044302388ADF8463095F8303101228DF8DE
:107AD80039201BB98DF844208DF83930814B00933B
:107AE800814B95F84800A3F179020CA903F0EEFB4D
:107AF800C0B10B28A8D1D4F8941499B1002EA3D002
:107B0800D4F84033794843F02003C4F8403308F0F0
:107B18000FFE764808F0D2FD002095E7704803F084
:107B28003AFAA4E795F8487095F9693095F939203B
:107B380095F87D106E4E384603F0DFFB009641B293
:107B4800EB6C95F850203846183603F01CFB00966D
:107B5800EB6C95F8502095F9701095F8480003F0F3
:107B680012FBD4F8C413AB6DD4F8DC230B44C4F86F
:107B7800B033EB6D1344C4F8B43394F80431042BD8
:107B880007D02B6E0B44C4F8B0336B6E1344C4F8A3
:107B9800B4330023089395F83031002B40D10023EB
:107BA8008DF8133095F839308DF8213095F8383044
:107BB8008DF82230D5F880300993D5F884300A93AF
:107BC8002388ADF82C3095F8303194F81B648DF883
:107BD8002E3095F84800474B8DF820600DF11302C0
:107BE80008A903F0F6FA012384F8413495F83930EE
:107BF80084F842349DF8133084F84334D4F81C34A4
:107C0800C4F85064C4F84834C4F8583402F0E5FBAA
:107C1800C8B1D4F81C0402F0F2FBA0B1102013E79D
:107C280008A802F0A7FC60B995F9390094F8376202
:107C38009DF82070FFF7CEFD3E44B042AFD2082039
:107C480002E7132000E795F81831012B01D102F063
:107C5800D8FB02F0C5FB0023059394F8043195F98D
:107C6800395094F81B649BB1042B7FF4E7AE05A848
:107C780002F0B4FE58BB94F8183413B1059B013BCD
:107C88000593174B05983246E9B202F00DFF02E062
:107C9800134802F0DDFE08B11120D5E6D4F84033D0
:107CA80094F80C11218043F00203C4F8403394F88F
:107CB800183411480133DBB284F8183484F8453499
:107CC8000E4B00259B6AC4F89854984724E7122065
:107CD800BAE60E20B8E600BF0080002000070020AA
:107CE8000808002030800020940B0020680A00203B
:107CF800B80A00201C0B002002070020101A0108F7
:107D080073B5134D134E0096EB6C95F8502095F90A
:107D1800781095F8480003F036FA95F83031337545
:107D280095F8480040F2012306F13C02314673827F
:107D380003F03FFA50B196F83C3086F88230064B93
:107D480000205B6B9847F37C86F8A83002B070BDC2
:107D580000800020E80A0020101A0108F8B5324C0B
:107D680094F81831012B05460ED0022B4ED0002B6B
:107D780057D138B9D4E91B0104F1740383E803002F
:107D88000020F8BD012806D102F02CFB0028F8D10C
:107D980084F81851F5E7022843D1244E84F81801D5
:107DA80006F5747CBCE80F0006F57A770FC79CE8E7
:107DB800030094F8E92094F8003187E8030086F876
:107DC800FB53D2B1022B18D1D4F804316367C6F83B
:107DD800EC3394F87D3094F8082186F8F83394F859
:107DE8008C3084F8782086F8F93396F81B2486F8C6
:107DF800E82340F20133A6F8FA33002386F81A3450
:107E08000B4BDB6A9847FFF77BFFB9E748B9074B8D
:107E180084F81801062283F89024054BDB6A9847FA
:107E2800AEE70320ADE700BF008000200007002078
:107E3800101A0108F0B5504C504EB4F8DC202287D7
:107E4800D4E92D0194F8B12084F8692004F16C027A
:107E580082E80300D4E92F0104F1740282E80300E8
:107E6800B4F8C420A4F87C2091B0D4F8CC20D4F87D
:107E7800C810C4F884200025D4F8D020C4F888207D
:107E88000123A4F82031C4F8801084F83051A56289
:107E980084F81B5184F83A5084F81D5184F81E5117
:107EA800C4F83451C6F89854A6F8185486F81A54E9
:107EB800A4F838518DF8183004F50973039304F5C4
:107EC8000E7394F84800049303A92D4B84F8455188
:107ED800C4E94F55A4F84651059303F019F9E36E28
:107EE800C6F8D43394F87D3086F8E03394F88C30B3
:107EF80086F8E1334FF48073A6F8E23386F8D0535E
:107F080094F8303186F8E43306F574770FCF06F528
:107F18007A740FC497E8030040F2012384E8030051
:107F2800A6F8FA33D6F8483386F81B54CDE901553C
:107F38001BB15A685B6901920293124B0793A3F134
:107F480048020892A3F1140209920F4A0B922933AE
:107F58000A93A2F19C030C93A2F198030D93131DAD
:107F68000E9301A902F14C0307A802F59B620F9337
:107F780002F022FA11B0F0BD0080002000070020B6
:107F880070060020680B0020E4800020F8B50D4F33
:107F98000D4E0C4608F044FB3B6B98470B4A96F88D
:107FA8004800214603F005F950B1094D706D95F868
:107FB800243485F86A347B6B9847E37C85F89034E1
:107FC800F8BD00BF101A010800800020240B002013
:107FD800000700200F4890F81B3480F8B8330E4B88
:107FE80093F8692080F8BB2393F87D2080F8C82394
:107FF80093F88C2080F8C92393F8303180F8CC337B
:108008000022A0F8CA2300F56E7100F56070FFF732
:10801800BDBF00BF0007002000800020114890F875
:108028009034EBB190F81B3480F8D0330E4BDA6EF5
:10803800C0F8D42393F87D2080F8E02393F88C20AF
:1080480080F8E12393F8303180F8E4334FF48072FC
:10805800A0F8E22300F5747100F56670FFF796BF8B
:10806800704700BF000700200080002070B5344C26
:108078002421204606F000FB636A984218BF60621C
:108088004FF01C012F4814BF0125002506F0F4FA13
:10809800636C984218BF60644FF480712A4818BF17
:1080A80045F0020506F0E8FAD4F84831984218BFBE
:1080B800C4F848014FF0D401244818BF45F004051E
:1080C80006F0DAFAD4F82032984218BFC4F8200231
:1080D8004FF010011E4818BF45F0080506F0CCFA0D
:1080E800D4F83432984218BFC4F834024FF460719F
:1080F800184818BF45F0100506F0BEFAD4F8B83590
:10810800984218BFC4F8B8054FF01401124818BFB8
:1081180045F0200506F0B0FAD4F8D03598420F4B58
:1081280018BFC4F8D005D3F8483318BF45F0400548
:108138002BB11B691BB12846BDE87040184770BDBC
:108148000080002028800020488000204C810020EA
:108158002482002038820020BC85002000070020EF
:108168002DE9F04F8FB04FF00009012B06460F465E
:1081780090468DF80D90ADF8109002D84C46BC4250
:1081880002D30FB0BDE8F08F305D02F033FA20441F
:10819800B842F6DC335D651C023BEDB2112BF0D81A
:1081A80001A252F823F000BFF981000823820008D9
:1081B8002183000849830008C7830008ED8300086D
:1081C800538400087B840008018500088B8100081F
:1081D8008B810008558500088B8100088B81000879
:1081E800FD850008258600085D8600089186000840
:1081F800052002F0A7FA70B10521002002F068FA04
:10820800725DBA4BE51C0234E4B283F85C24325D3B
:1082180083F85D24EDB22C46B1E700238DF80E30CB
:108228008DF80F308DF814308DF81830B9F1000F33
:108238006DD1AF4C4FF0050994F87C208DF83120B2
:108248006B1E94F839208DF83320334494F8382085
:108258000B938DF8342094F81A3194F868208DF82F
:108268003520D4F82C218DF832300A9273B37B1C58
:108278005B1BDBB28DF8303006AB019305AB009386
:1082880094F848000DF10F030DF10E020AA902F04F
:10829800B6FF8DF80D0000F00700072813D194F9F8
:1082A80039209DF90E3084F839309A429DF80F3004
:1082B80084F83830B8BF01229DF81430B8BF84F86C
:1082C8001D2184F868304FF0000A09E00523D1E742
:1082D80001220DF10D01032002F0A4F80AF1010AB0
:1082E8005FFA8AF29DF81830B3FBF9F19142EFD8A2
:1082F8002B44DDB26B1EDBB29F420BD9F25C032A22
:108308009AD0AF4288BF1D464FF0010983E7053474
:10831800E5B2F9E71D46F7E7735D754903F00F030A
:10832800012281F81B31023402FA03F3A1F820314B
:10833800E4B2002204A9042002F074F825466AE792
:1083480007238DF80D30735DC3F3021203F00F039A
:108358008DF82830E31CDBB28DF82920F25C231D50
:10836800DBB2651DF35C0234E4B21B0443EA02236A
:10837800325D5F4C13436422534394F848000B93D7
:108388000AA902F057FF00F00703072BEDB28DF89A
:108398000D000CD19DF8283084F8703084F87830BE
:1083A8000B9BE36663679DF8293084F869308DF884
:1083B8001000012204A9052002F034F82BE74B4BEA
:1083C800D3F8483363B11B6853B1984708F03F03AB
:1083D8008DF810008DF81130022204A90620EBE771
:1083E800FF20F3E703238DF80D30735D8DF81C3003
:1083F8000AAB0693E31CDBB2A51DF25C231DDBB2BE
:1084080006A9F35C1B0443EA0223A21CD2B205347A
:10841800B25C134364225343E4B20A9300230B93E0
:10842800335D8DF83030324B93F8480002F011FF7D
:10843800C3B20028EDB28DF80D30FFF6ECAE8DF822
:108448001030012204A90720B6E7735D03F00F037B
:10845800012B4FF47A7238BF01235343244A023464
:10846800936503F57A73D365E4B2002204A9082062
:1084780062E7735D1E4DC3F340128DF8152095F821
:108488004800C3F3001205A903F00F038DF8142068
:108498008DF8163002F0ECFE02340130E4B23FF4FD
:1084A8004DAFBDF81430134AA5F87C309DF816304E
:1084B8009DF814A0D05CF8F797FB0223C5F880005C
:1084C8000AA995F848008DF828308DF82AA002F0FE
:1084D800FDFD95F93930069040B29842B8BF18466C
:1084E80085F83900002204A9092025E700070020A3
:1084F800008000205F12010803238DF80D30735DA2
:108508008DF82830E31CDBB2651DF25C231DDBB25D
:108518000234F35CE4B21B0443EA0223325D1343E2
:10852800642253430B93644B0AA993F8480002F062
:10853800AEFEC3B20028EDB28DF80D30FFF66BAE7B
:108548008DF81030012204A90A2035E7092002F02D
:10855800F9F8DFF868B1002849D00921002002F0B5
:10856800B7F80023ADF81E30A31CDBB2F25CE31CA5
:10857800DBB216F803A0735D4FEA0A4A4AEA022AF8
:108588004AEA030A231DDBB2A51D0534F35CE4B2F5
:108598004AEA036A335D4FF47A7253430AAC1B12FA
:1085A8002046ADF81C3007F04BFF454B534406936B
:1085B800DBF83C3300930DF1180A9AE80600DBF863
:1085C800383308A807F0F9FE099B009394E80600E1
:1085D800089B504607F0D6FE9AE8030007F008FF0C
:1085E80001F00AFF0123EDB28BF8383413E68BF85B
:1085F800380410E60C2002F0A5F800283FF40BAE72
:108608000C21002002F064F82C4B93F89034043BC2
:10861800012B7FF600AE01F0EBFEFCE5A31CDBB2FC
:10862800725DF15CE31CDBB2651DF35C0434E4B2FB
:108638001B04305D43EA012313436421594300F0CE
:108648000F0001F0D6FEEDB28DF81000012204A94A
:108658001120B1E60D2002F075F800283FF4DBADDB
:108668000D21002002F034F8A31CDBB2154AF05C9F
:10867800735D1268251D0334E4B243EA0020315DBE
:10868800EDB201F0B8FEC6E5725DA31C251D0334EA
:10869800DBB2E4B2F15C335D1B0443EA012313430C
:1086A8006420584301F0A9FEEDB28DF810000122B4
:1086B80004A9132080E600BF0080002000070020E6
:1086C800803DD512580600200E4B93F8912492074E
:1086D80003D593F88F24012A08D90B4991F81A2158
:1086E80022B18A6A501C18BF01328A620022A3F89C
:1086F800182483F81A24D3F8402322F00202C3F87E
:1087080040237047000700200080002070B5184CF7
:108718001848194D07F084FFD4F84033D4F898046A
:10872800D5F8906023F02003C4F8403338B107F03F
:108738003DFF864203D2002385F83A3070BD012000
:10874800FFF766F90028F9D00B28F7D095F83930EB
:1087580084F84234092094F8183484F8453484F8AD
:10876800410401F0D7FFBDE87040FFF7ADBF00BF7F
:1087780000070020680A002000800020094BD3F879
:108788004023012A0AD008490978C90708D43AB908
:1087980093F89204013818BF0120704700207047F1
:1087A80001207047000700206C060020034BD3F817
:1087B8004003431E58425841704700BF000700203D
:1087C8002DE9F04FA9B0EFF3108272B6DFF8F0B2DE
:1087D8000021DBF80030CBF8001082F31088B94C88
:1087E800002B00F0E180DAB29B06039264D5B64D07
:1087F80095F81831022B02D0B44BDB6A9847EFF397
:10880800108872B6B24F07F0C7FE3E68D4F8B013AE
:10881800361A3144AF4807F08BFFAE4807F04EFFD9
:10882800D4F8B413AC48314407F082FFAA4807F0E3
:1088380045FF88F3108894F81A34002B00F06B81F8
:10884800152312A995F848008DF8483002F03EFC2F
:10885800D4F8B4130F900144A04807F069FF9F486B
:1088680007F02CFF3B6894F81B24EB620DAF3846E9
:108878008DF870201D9307F009FED5F82831009374
:1088880006AE97E80600D5F82431304607F095FD86
:1088980096E803001FAB83E80300D4F81C341E934A
:1088A80095F8303195F84800003B18BF01231CA902
:1088B8008DF8713002F01EFC039BDF0648D5824D0F
:1088C800DFF81CA2D5F8E42004929BF80020BAF93E
:1088D8000A809AF90C90A4F88C84002363F30002B0
:1088E8000A9384F84434A4F8223484F82534C4F86C
:1088F8002834A4F82C3484F82E34C4F8303484F89E
:108908002034C4F8343484F83834C4F83C346F4B19
:108918008BF8002094F89024DB6A84F88E9484F80D
:108928008F24DAF80470BAF80860984794F88F34FE
:1089380013B9694807F074FE3146384601F045FD21
:108948008346002800F0EA80A4F87E8484F88094A6
:10895800039B19071AD55C4B93F81831022B02D0E8
:108968005A4BDB6A98470220FEF712FF84F841044D
:1089780001F0D0FE94F81A3413B1012384F81934A5
:1089880094F8913443F0100384F89134039B5A0708
:1089980003D506210520FEF765FF039B9B0703D53A
:1089A80004210320FEF75EFF01F02DFD94F89124C9
:1089B800D7065FD5002384F89234D4F840331E06D6
:1089C80044BF23F08203C4F8403312F0050F00F0CF
:1089D800FB820B2001F0B6FE002800F0F58294F827
:1089E8009134DD0700F1F082580740F10783D4F88D
:1089F800403323F00203C4F84033D4F8402382BB49
:108A080094F8915415F001011EBF2B4662F3000340
:108A180084F8913494F891345E0744BF6FF382036D
:108A280084F89134012384F8923421B1D4F8443382
:108A38002C481B6898476D070BD52B4801F08EFE14
:108A480001F0BCFE28B194F8913443F0040384F893
:108A5800913401F0C6FC94F891346FF3041384F850
:108A68009134012384F8923494F8913443F020032C
:108A780084F8913494F8913418070AD56FF3C30336
:108A88001A4984F89134D4F84433A1F12400DB68FE
:108A9800984794F8913499070AD56FF3410313491D
:108AA80084F89134D4F84433A1F16C005B6898479A
:108AB80094F89034022B1BD1FFF722F918E000BF7D
:108AC8006C0600200007002000800020101A010812
:108AD80068060020800A0020980A0020000B002069
:108AE80058060020400B0020540B00208C0B00205F
:108AF80094F891349A0640F1C4826FF3451384F8D0
:108B08009134D4F84033002B40F0BB8229B0BDE843
:108B1800F04FFFF7ABBA84F84134A3E695F8183163
:108B2800012B0CD101F055FC804668B1584601F084
:108B380045FC584601F047FC042384F88F347EB97D
:108B4800012384F821344FE101F045FC0028F6D0D8
:108B5800404601F034FC404601F036FC0523ECE7C2
:108B68003B7805935B09013B062B00F21782DFE88F
:108B780013F007001502950015029200150206026F
:108B8800102EDDD995F830311297F6B28DF84C6079
:108B9800002BD5D11CA805F081FC12AA1CA9FF2026
:108BA80002F09EF89DF85830C3F3030307468DF88A
:108BB8002C3095F8480095F87D308DF82D30072237
:108BC8000BA902F0B3FA002F5DD100285BD09DF805
:108BD80053309DF852201599C5F8E4101B0443EA58
:108BE80002239DF8512002201343C5F8E03005F018
:108BF80063FC9DF8583095F8480085F82E71C3F34A
:108C08000212C3F3030385F8703085F878309DF8B5
:108C1800593085F86920012B38BF01234FF47A7247
:108C28005343AB651344EB650DF15A034FF001084C
:108C38001093113E94F81B348DF83C300FA985F839
:108C480068808DF8446002F081FA0223404685F876
:108C5800303101F077FD18B14146384601F038FD52
:108C680094F88F34012B00F2A78194F81A34002B62
:108C780040F09A8194F8913443F0100384F89134C9
:108C8800FEF786FD64E6012001F05CFD0028E7D0D0
:108C980001210720E2E7012384F8203495F87D308C
:108CA8008DF82E3094F824348DF82D3095F88C30CA
:108CB80095F848000D330BA98DF82C3002F006FA10
:108CC800A6F10D031BB2099023EAE37300B28342B5
:108CD8003FF736AF0B2E7FF633AFBA4B25931CA860
:108CE800FF231C978DF874608DF8983002F0C4F853
:108CF800074600287FF424AF95F81831012B13D1CB
:108D080001F067FB002872D0384601F057FB38465F
:108D180001F059FB04239DF87C101E9884F88F34C9
:108D2800C1F3001101F06EFB9DF87C301E99C4F868
:108D3800341413F00F0203D09DF89000002862D17C
:108D48009DF89800002861D0002A7FF4F9AE9DF8BC
:108D58009020002A14BF4FF003084FF002080022A9
:108D68000A92D5F8EC2095F8E900914251D10028F3
:108D78004FD0D5F80C1195F8EAB009680A9195F822
:108D88001811022902D1032184F88F14B8F1030FB6
:108D98007FF4D6AE13F0600F7FF4D2AE04920127B1
:108DA80095F82E31BBF1000F36D0BBF1010F13D16E
:108DB800012B33D16FF0090646FA08F606F00106D2
:108DC800C6F10206F6B2BDF87E100AAA304601F0D6
:108DD80011FE38B3072823D0012384F821340A9BD5
:108DE800C4F83034C4F86C34FEF720FDB0E501F067
:108DF800F2FA002898D0384601F0E1FA384601F036
:108E0800E3FA052387E74FF00008A8E74FF00108C9
:108E1800A5E74FF0010BC3E70426D4E70326D2E702
:108E28000823DAE71CAB009304990A9B324658469C
:108E380001F0A2FE20B1022814BF0B230A2380E60A
:108E48000A9BC4F83034C4F86C349DF87C3084F83C
:108E58002104C3F3401384F82E3484F8443494F87E
:108E68008F3484F82274012B9EBF0122A86285F8F2
:108E78001E21012FC4F8280484F82C0484F8410426
:108E880038D1022284F8202495F83A20002A4AD1C1
:108E98009DF87C20D60646D4012B94F840149DF802
:108EA8007C2005D8012901D1900601D501F04CFBA1
:108EB800B8F1020F94F88F3443D0B8F1030F0AD0F9
:108EC8009DF87C10B8F1010F4A4601F00F0120A867
:108ED8003BD0FFF745F99DF8903084F82334259B63
:108EE800C4F828349DF8983084F82C34012384F889
:108EF8002D3430E0059A02F0E002A02A1BD195F843
:108F08002E11012285F83A2009B927996963012BA6
:108F180084F8202407D9D5F89020C4F83C24DAF83E
:108F28000020C4F8982495F81821002AB4D1012209
:108F380084F82524B0E7002285F83A2084F8202414
:108F4800A6E79DF8981025984A46FFF709F99DF875
:108F5800903084F823349DF89020E02A08D195F8C1
:108F68001F312BB984F82324C4F82834A4F82C34EE
:108F780094F8913443F0020384F8913470E6114D6B
:108F8800013EB2B2791C284605F060FB0323A4F821
:108F98002034C4F8285484F82C64E9E7012384F8C1
:108FA8002134FEF743FC5BE694F84434002B3FF48D
:108FB80061AE0020FEF726FC94F88F34022B3FF4B4
:108FC8005FAE57E63809002094F89134590715D553
:108FD800012001F0B7FB60B1012001F08BFB08B95B
:108FE80084F81804D4F8403323F00203C4F840335B
:108FF80004E0062001F0A6FB0028F3D194F8913490
:10900800DA077FF5FAAC94F840240AB1032A18D19C
:109018001D4A94F8181492F86820914205D29B07CB
:1090280023D594F88F34012B1FD8184807F0F8FA85
:10903800D4F8403323F02003C4F84033FFF744FB4F
:10904800DBE4012A11D194F81924002A3FF4D5ACA5
:109058000D4A94F8181492F868209142E5D29F07B7
:1090680003D594F84434002BDFD194F891340020D0
:109078006FF3041384F8913484F81904FFF746FB5E
:10908800BBE429B0BDE8F08F00800020680A00200A
:109098002DE9F04F89468DB090460746002800F02C
:1090A8008F81002900F08C810368002B00F08881F3
:1090B8004368002B00F084818368002B00F08081D6
:1090C800C368002B00F07C81104601F0F5FF0028F2
:1090D80000F07881BD4CBE4D384601F0AFFA40F241
:1090E800D4520021204605F0C5FA40F21C52002156
:1090F800284605F0BFFAB74BC4F82C3104F50973BC
:10910800089304F50E7300264046099308A9B24B4C
:1091180084F848800A9384F8186184F88C608DF884
:109128002C6001F0F5FF0F2306A994F848008DF88C
:10913800183001F0CBFF801B18BF01204FF00A0B3D
:1091480084F81C0106A994F848008DF818B001F0BD
:10915800BDFF4FF0060A84F8DC0006A994F8480021
:109168008DF818A001F0B2FF102384F8DD0006A9DD
:1091780094F848008DF8183001F0A8FF1123C4F8BE
:109188009C0006A994F848008DF8183001F09EFF5D
:109198001223C4F8A00006A994F848008DF81830E6
:1091A80001F094FF1323C4F8A40006A994F848001A
:1091B8008DF8183001F08AFF1423C4F8A80006A916
:1091C80094F848008DF8183001F080FF1623C4F891
:1091D800AC0006A994F848008DF8183001F076FF25
:1091E800172384F8B10006A994F848008DF81830C0
:1091F80001F06CFF18230DEB0301C4F8B400C4F8A8
:10920800BC0094F848008DF8183001F05FFFC0B238
:109218001D2384F8B80084F8C00006A994F8480013
:109228008DF8183001F052FF1E2384F8C40006A9F7
:1092380094F848008DF8183001F048FF1F2384F88F
:10924800C50006A994F848008DF8183001F03EFFD3
:109258002023C4F8C80006A994F848008DF81830EF
:1092680001F034FF0B23C4F8CC0006A994F8480099
:109278008DF8183001F02AFF0C2306A9A4F8D000B5
:1092880094F848008DF8183001F020FFD4F89C308D
:109298006365D4F8A030A365D4F8A430E365D4F8A6
:1092A800A83023664FF00108D4F8AC300590A4F834
:1092B800D200636684F8B080C4F894B084F898A0AB
:1092C800C4F84CB084F850A084F8688084F81F81F2
:1092D800C5F84893FEF7AEFDC5F84473C4E90B66BC
:1092E8003E4B84F8198185F89164C5F8408332466D
:1092F8004FF0FF31009605F55A7007F033F9384BF7
:10930800009632464FF0FF3105F5607007F02AF9F4
:10931800344B009632464FF0FF3105F5667007F082
:1093280021F902AF304B009632464FF0FF3105F578
:10933800806007F017F9384607F0A8F897E80300A7
:1093480004F5927383E80300284B294F1E60294BCC
:10935800C5F84C33284BC5F85433284BC5F85C3353
:10936800274BC5F85033274BC5F8583305F55370CC
:109378003B68984704F5A67004F0ACFE20B11126AE
:1093880030460DB0BDE8F08F204601F003FB002801
:10939800F5D101F039F8B8B91B4801F04DFB064684
:1093A8000028ECD17B69984705F02EF9BB6D94F83D
:1093B80019019847FB6A9847012385F89234DFE73B
:1093C8000326DDE70926DBE71326D9E7008000201E
:1093D800000700200004000170060020158700081F
:1093E800DD7F0008258000080D7800086C06002045
:1093F800101A0108CD79000881790008C97700089A
:109408005979000831790008E880002008B5034B35
:109418000020C3F84003FEF7BBF908BD0007002091
:1094280010B5FFF7ABF90A4C60B90A4B93F818313D
:10943800022B02D1084BDB6A98470123C4F840335A
:10944800002010BDD4F84003013818BF0120F8E708
:109458000007002000800020101A010838B5124CBF
:10946800204607F0DDF804F1180007F0D9F804F1F8
:10947800300007F0D5F804F1980007F0D1F800F0B3
:10948800AFFF0A4B0025DB6A984744F8285CFEF7D3
:10949800EDFD0749074840F2D45205F0D7F80123FB
:1094A80044F8283C284638BD680A0020101A0108EC
:1094B80000800020D485002070B52E4B8AB0054668
:1094C80093F8DD008DF8090093F8DC008DF80A00A8
:1094D80029489A6A90F81804039200268DF80B0020
:1094E80004960C46002940D00692D3F888200792AB
:1094F8001A8F93F81A118DF8151052BAADF820206A
:1095080093F87C2093F848308DF8243003AB8DF81D
:1095180022008DF8232000930DF10A020DF10B03B0
:109528000DF1090105A88DF8146000F0D7FE9DF92A
:109538000900FEF74FF9607004A801F01BF8B0B9F4
:10954800049A0F2A0DD863789A420AD81544AB4278
:10955800A3EB02012CBF002001202170C0000AB03B
:1095680070BD002323700820F9E70320F7E71320D4
:10957800F5E700BF00800020000700201FB5044663
:10958800002800F010810378412B00F20781DFE802
:1095980013F0420049004D005100550059005E008B
:1095A8000501050105010501050105010501050183
:1095B800650069006D0078007F00820085008A00E0
:1095C80088008C0090009300960099009C009F00F2
:1095D800AE00B200BA00B600BE00C100C500CE00A1
:1095E800CA00CC000501D2000501050105010501ED
:1095F8000501050105010501050105010501050133
:10960800050105010501DA00DE00E200E700EB00D4
:10961800EF00F300FC00664B93F81831237100202B
:1096280004B010BD624B93F83031F7E7406804F09E
:10963800EFFEF4E7406804F031FFF0E75C4B93F885
:109648001A31EBE75A4BD3F8E0306360E7E7584B41
:10965800011D93F8300104F039FFE0E7544B93F80B
:109668001931DBE7524B93F88C30D7E71C238DF880
:1096780008304F4B02A993F8480001F027FD6060BD
:10968800CDE74C4B043493E8030084E80300C6E7B5
:10969800494B0434F7E7494B0434F4E7484B0434A6
:1096A800F1E71A23E3E71923E1E7414B93F8683020
:1096B800B4E73F4B5B6DC8E73D4B9B6DC5E73C4B43
:1096C800DB6DC2E73A4B1B6EBFE7394B5B6EBCE7FD
:1096D80002238DF80830364B02A993F87C2093F8C2
:1096E80048008DF80A2001F0F1FC207197E7304B13
:1096F80093F8DD3092E72E4B93F839308EE72C4BF8
:1097080093F8DC308AE72A4B93F8383086E7284B01
:10971800DB6C9AE7264B93F850307FE7244BD3F85D
:10972800843063607BE7224B8FE7264B8DE7204B25
:10973800D3F8CC30F5E71E4BD3F82C31436001F059
:10974800F3FDA0606BE71A4BD3F890307DE7184B18
:1097580093F81F3162E7164BB3F88830A3805EE7B1
:10976800134BB3F88A30F9E7114BB3F8D030F5E76B
:109778000F4BB3F8D230F1E70D4B93F848200AB1FC
:10978800062A12D1B3F8B035E8E7094B93F8482018
:109798000AB1062A09D1D3F8B43556E704B0BDE8B2
:1097A800104000F021BE03203AE7182038E700BF38
:1097B800008000206C800020B4800020748000208D
:1097C800BC800020D48500207FB5044610B9032052
:1097D80004B070BDA34DD5F840339A0700F16F82ED
:1097E8000278412A00F26882DFE812F0420047005E
:1097F80055005B005F006400690076008100870007
:109808008D00930099009F00A500AB00B50066028B
:10981800BA00DC00EF0016013801290142014B01B2
:109828004F01530157015B0166025F017101990104
:109838008701AB01B101B801BD01C201660228026E
:1098480066026602660266026602660266026602D0
:1098580066026602660266026602660266026602C0
:10986800340239023E02430248024D0252025C02AF
:109878000079FEF773FA30B1AAE70379022BA6D074
:10988800794A82F8303195F8913443F0200385F80D
:10989800913400209CE7406804F0ACFD0028F2D029
:1098A80095E7406804F0EAFDF8E76F4B027983F822
:1098B8001A21E8E76C4B4268C3F8E020E3E76A4EF8
:1098C800416896F8300104F0F7FD00287FF47FAF77
:1098D8006368C6F8E430D6E7416800293FF477AFFB
:1098E800002001F0DDF90028CDD0112070E7416893
:1098F80000293FF46CAF0120F3E7416800293FF4E9
:1099080066AF0820EDE7416800293FF460AF092001
:10991800E7E7416800293FF45AAF0C20E1E74168C6
:1099280000293FF454AF0D20DBE7416800293FF4DC
:109938004EAF0E20D5E7416800293FF448AF0F200D
:10994800CFE74A4C484B007983F81901A36D984733
:10995800E36A984797E7444B027983F88C2092E7AB
:10996800414E037A8DF8043096F8480096F87D3019
:109978008DF80530072201A901F0D8FB00283FF433
:1099880026AF636896F848000193002201A901F008
:10999800CDFB00283FF41BAF6C36D4E9010186E803
:1099A800030070E7304E037A8DF8043096F84800CB
:1099B80096F87D308DF80530072201A901F0B6FB35
:1099C80000283FF404AFB436E7E7274E037A8DF852
:1099D800043096F8480096F87D308DF80530072257
:1099E80001A901F0A3FB00283FF4F1AED4E901017D
:1099F80006F1740383E8030096F81831022B7FF40C
:109A080042AF96F83031002B3FF43DAF174BDB6A7D
:109A18009847FEF775F936E7134E037A8DF8043048
:109A280096F8480096F87D308DF80530072201A990
:109A380001F07CFB00283FF4CAAEBC36ADE74368B2
:109A4800029301238DF80C30074B02A993F84800C4
:109A580001F08AFB00287FF416AFB8E6436802934A
:109A68000023EFE70007002000800020101A0108FB
:109A780003795A1E0E2A3FF6AAAE934A82F8683036
:109A880001E7914B42685A65FDE68F4B42689A653B
:109A9800F9E68D4B4268DA65F5E68B4B42681A6643
:109AA800F1E6894B42685A66EDE6874C037994F8EB
:109AB80048008DF80430062201A901F037FB002880
:109AC8003FF485AE9DF8043084F8DD30DBE67E4C4B
:109AD80003798DF8043094F8480094F87C308DF8B8
:109AE8000630052201A901F021FB00283FF46FAEE2
:109AF8009DF8043084F83930C5E6734C037994F83E
:109B080048008DF804300A2201A901F00FFB002853
:109B18003FF45DAE9DF8043084F8DC30B3E66A4C5F
:109B2800037994F848008DF80430092201A901F05E
:109B3800FDFA00283FF44BAE9DF8043084F8383025
:109B4800A1E6614B4268C3F89420DA649BE65E4B59
:109B5800027983F8982083F8502094E65A4B42689B
:109B6800C3F884208FE6584B4268C3F8CC208AE6B5
:109B7800012B40F0A480554C2421204604F07CFDA4
:109B8800636A984201D0172022E61C2104F12800BC
:109B980004F072FD636C9842F5D14FF4807104F1C2
:109BA800480004F069FDD4F848319842EBD1D4213B
:109BB80004F5A67004F060FDD4F820329842E2D192
:109BC800102104F5097004F057FDD4F83432984296
:109BD800D9D14FF4607104F50E7004F04DFDD4F83E
:109BE800B8359842CFD1142104F2BC5004F044FD9A
:109BF800D4F8D0359842C6D1334E2146304640F28B
:109C0800D45204F023FD204640F2D452002104F03F
:109C180031FD95F81B3485F8E833736FC5F8EC33DC
:109C280096F87D3085F8F83340F20123A5F8FA3329
:109C3800274B96F819019B6D984724E68379012BE9
:109C48003FF6C5AD204B42684068C3F82C2100F0B0
:109C5800BDFE48E61C4B4268C3F8902013E61A4B39
:109C6800027983F81F210EE6174B8288A3F8882013
:109C780009E6154B8288A3F88A2004E6124B8288ED
:109C8800A3F8D020FFE5104B8288A3F8D220FAE58C
:109C98000D4B93F848200AB1062A12D1A288A3F8DE
:109CA800B025F0E5084B93F848200AB1062A08D1F8
:109CB8006268C3F8B425E6E500F098FBDBE501200F
:109CC80086E5182084E500BF00800020D4850020A8
:109CD800101A01082DE9F04387B00023ADF80030D1
:109CE8000646002800F0EE800361FEF747FD20B12C
:109CF8000124204607B0BDE8F08300F065FD002888
:109D0800F6D100F05BFD014618B96F48142204F043
:109D1800B1FC6E4D95F89134012243F0040385F8A7
:109D2800552485F8913433788DF804300021013BAF
:109D38008DF80520ADF806100C2B00F2BB80DFE88B
:109D480003F007B9B9B97982B9B990B9AD9AA90040
:109D5800D5F8407317F02007CAD196F80480B8F1F7
:109D6800020F46D1DFF868815A4CFEF763F896F97E
:109D7800051098F848003A4601F098FA88F8390032
:109D8800B37988F83830384607238DF80530FDF761
:109D9800E5FFFF2304F58670A5F80C31C5F80841E6
:109DA80085F8047104F07AFB04F58A7004F030FB3E
:109DB8003846FDF72DFE0446002839D096F90510DF
:109DC80098F84800012201F071FA88F83900D5F8AE
:109DD80094343361002C71D000F0F0FC002888D155
:109DE80095F8913485F81A0460F3820385F8913464
:109DF8007FE7B8F1010F4FF00204E8D1DFF8D09007
:109E08008DF8144099F8480089F81D7102A901F0ED
:109E18007FF9337989F830318DF805708DF806802F
:109E2800FDF7C4FC95F8913443F0100385F891349C
:109E38000024CCE700226946022000F0F3FA00284B
:109E4800F6D01324C3E7244BB288DB6B96F90C10C9
:109E5800B0689847D5F8403343F00203C5F840335B
:109E6800E6E702A90D2000F053FB0028E0D000220D
:109E780069460D20E1E7164B93F81831D3B93479C8
:109E880004F0070000F0ABFA8DF8004001226946A3
:109E98001020D2E7002269461220CEE78DF807206D
:109EA80000F08EFA044638B900F087FA204600F030
:109EB80089FABDE702248AE7012488E701A800F0AF
:109EC800D1FB16E7032414E7540B002000070020F9
:109ED8000080002002070020101A01082DE9F04F29
:109EE80099B08046059118B9032019B0BDE8F08FE4
:109EF80000230361FEF742FC0446002840F0A580D9
:109F080046460FCE0EAD0FC51422524898F800A051
:109F1800B8F80C7098F90EB04F4E214604F0AAFB21
:109F28004E4B012283F8412496F83021022A254617
:109F38000BD196F81821022A07D196F81E2122B9CA
:109F4800BAF1010F38BF4FF0010ABAF1010F2BD057
:109F5800BAF1030F2AD0BAF1000F33D102229DF8CB
:109F68003C30DDF84090029362F34715012496F8DF
:109F78007C108DF8321002220CA996F848008DF852
:109F8800302001F0A3F896F81A3196F830C196F807
:109F98001D1140B2002B63D0BCF1010F57D100292D
:109FA80055D1002C61D153E00422D8E70023DDF815
:109FB8003C90BDF840709DF942B0029365F01F05D2
:109FC8000124D4E74FF0000BD946CDF808B0CEE70E
:109FD8004FF0010084F81A04D2E005F29A420BA966
:109FE80000F0D4FA002800F015811320049B338771
:109FF8001A4B002283F81A2423E105F29A452A46CF
:10A008000BA900F0C3FA0028EFD10B9B84F82801B4
:10A01800C4F82C5184F83031FCE0B9F1000F00F09D
:10A02800F980002A00F0F6804946E01C04F00EFB97
:10A0380094F8373201332380ECE01220D6E702206F
:10A04800D4E70720D4E71320D2E701204DE7FCB975
:10A058000220F6E0400B00200080002000070020CE
:10A06800002CF5D05845B8BF584696F87C308DF886
:10A078002000052296F848008DF8223008A901F042
:10A0880055F800283FF430AF9DF8203086F8393075
:10A098006F4A704BD2F89804D3F8904038B106F064
:10A0A80085FA6C4B84423CBF002283F83A20198F12
:10A0B8001A8F93F830010491996A099152BA0028CD
:10A0C800BFD093F81B0100B9186393F81801ADF8D5
:10A0D8005820013893F87C2093F81A411491D0F154
:10A0E800000BD3F888108DF85B204BEB000B93F82E
:10A0F800482093F83A0093F868308DF85A3009AB45
:10A108000093554B03904FF001008DF84C001591CA
:10A118008DF85C20A3F12F01A3F1300213A88DF86C
:10A128004D4000F0DBF8039B4FEA0B1B4BEA431B47
:10A1380000264BEA801B4BEAC413B145444C0393F9
:10A1480008BF37463A46494604F59C70CDE90A6689
:10A158009B46268084F81A6404F078FAE9B2A57060
:10A16800C5F34215FAB2042D3A4E039B84F8372200
:10A178003FF42EAF072D3FF450AF022D7FF45FAFB1
:10A18800364D84F80D110420029984F80401FF204B
:10A1980084F80C0184F8281184F81431D6F8E410F6
:10A1A800C4F8085105F59B730AA8C4F8101184F87F
:10A1B8003021C4F82C3100F011FC00287FF43DAFA9
:10A1C8000A9BA4F844040BA8A4F81631C4F84C342C
:10A1D80000F0D0F900287FF408AF0B9BD3B196F9B3
:10A1E8003900FDF7F7FA94F83732002B3FF405AF42
:10A1F8000B9B0F2B3FF6F1AE05F58B720BA90F20C9
:10A2080000F0C4F900287FF4F0AE0B9B63F3030B56
:10A2180084F814B10598FDF7FBFB00287FF4E6AE3F
:10A22800099B86F83A00B36200F080F900287FF4B1
:10A238000AAF94F8913484F840A443F0010384F8F9
:10A248009134034BD3F89434C8F810304DE600BF6E
:10A2580000070020008000206880002002070020FE
:10A2680037B50B4D8DF8040004460F2295F84800C9
:10A2780001A900F05BFF40B1064A85F81C4192F83D
:10A28800913443F0200382F8913403B030BD00BF0D
:10A29800008000200007002010B5FFF7C1F8044631
:10A2A80088B90A4806F0BCF9094806F0B9F909481E
:10A2B80006F0B6F900F094F8FDF7BCFD064BDB6A32
:10A2C8009847204610BD0124FBE700BF680A00201C
:10A2D800800A0020980A0020101A01082DE9F04F82
:10A2E8008BB047780093149B90F90C8090F90D601F
:10A2F80090F80EB08A464168196004469146002FCE
:10A3080058D002238DF8103004A9C37B007C8DF847
:10A31800123000F0DBFEB4F808C0618943B260680F
:10A32800984545466144B8BF1D46604534BF00277F
:10A338000127884209D30A218DF81010207C019347
:10A3480004A900F0C3FE019B46B2B4F808C06089B6
:10A3580061680CEB400E714519D3A1EB0C01B1FB00
:10A36800F0FC00FB1C1191B9984503DC2378CBB9AC
:10A378004FF0010B21238DF81030207CE37B8DF802
:10A38800115004A98DF8123000F0A0FE45B2009BD0
:10A398008AF80050384689F8006083F800B00BB09E
:10A3A800BDE8F08F0223207C8DF8243006A900F048
:10A3B800AFFEDDE74546EAE77047704770477047EC
:10A3C8000020704770477047704700207047002092
:10A3D8007047002070470020704700207047704782
:10A3E800704770470220704702207047022070476C
:10A3F8007047002070477047704700207047002062
:10A40800704770477047704710B5054C4FF403729A
:10A418002046002104F02EF90020C4E9000010BDF8
:10A428001C0C00202DE9F8438146904600293CD0B9
:10A438001F4C2023224604F1100012F8017F6FBB45
:10A448008242FAD11B4E3368013403B93460736811
:10A4580003B11C6000252560C4F8088074601FFAE9
:10A4680088F284F80490601D04F0F0F8B9F1110F37
:10A478004FF0000398BF104D6373D6F8083298BFA9
:10A4880025FA09F503F1010398BF05F001054344D6
:10A498002573C6F808323846BDE8F883013B13F047
:10A4A800FF030446C6D10227F5E70127F3E700BFFB
:10A4B800230C00201C0C00202007020010B518B344
:10A4C800124A1368984204D103681360002305E018
:10A4D8000B46002BFAD019688842F9D15168884296
:10A4E80008BF53600BB101681960D2F8083281685F
:10A4F800013B00245B1A04602146C2F8083210228E
:10A5080004F0B8F8204610BD0120FCE71C0C002020
:10A51800054B1B6813B11A798242FAD1002B0B60E4
:10A528000CBF0320002070471C0C002010B5054B01
:10A53800186800B910BD037B04680BB9FFF7BEFFAC
:10A548002046F6E71C0C002038B5084B084C186864
:10A5580000B938BD03790568112B05D824FA03F32F
:10A56800DB0701D5FFF7AAFF2846F1E71C0C0020FE
:10A578002007020028B1044BD3F8083203600020FA
:10A5880070470120704700BF1C0C00202DE9F041E6
:10A5980007460E46154642B339B3154B1C680023CF
:10A5A8002CB93046FFF7E6FF0020BDE8F081A2682D
:10A5B800F91A0132914215D32279EA54581C22899A
:10A5C8005FFA80F8611D55FA80F004F03FF8A3683F
:10A5D800246898445FFA88F3E2E720462568FFF785
:10A5E8006DFF2C46002CF8D1DBE70120DDE700BF2A
:10A5F8001C0C00200238C0B211289ABF014B185C0D
:10A60800002070476F12010830B50B4B93F82020DB
:10A618000446084672B100211C330578A54208D0CB
:10A6280001319842CDB214BF04301038AA42F4D890
:10A63800002030BD1046FCE7280E002010B5084C5D
:10A6480000232060142204F10C00FF2184F820303C
:10A65800C4E9010004F00EF8012384F8213010BD8C
:10A66800280E002010B50E4A92F82010042915D89B
:10A67800936804781C7044785C70C478807898700B
:10A688000131DC7082F8201002F11C018B4214BFEA
:10A69800043302F10C039360012010BD0020FCE795
:10A6A800280E0020094B93F8200068B15A6803F17E
:10A6B8001C018A4200F1FF3014BF043203F10C027E
:10A6C80083F820005A600120704700BF280E002040
:10A6D80010B5074B93F820200446084632B1596854
:10A6E800FFF792FF10B101234470837010BD00BFC3
:10A6F800280E002008B5064B93F820202AB1596887
:10A70800FFF782FF08B1407808BD0120FCE700BFD1
:10A71800280E002030B50A4A92F82010536882F8B3
:10A72800210061B1916801241C32DD78587005B9A7
:10A738009C70934214BF0433103B9942F5D130BD4D
:10A74800280E002008B5044B5968FFF75DFF003854
:10A7580018BF012008BD00BF280E0020F7B504224D
:10A76800154E044600210DEB020096F8207003F008
:10A7780081FF0025EBB29F4201D803B0F0BD73689A
:10A78800197821705A786270987838B13368204601
:10A798009B689847FFF786FF0135EBE7DB788DF874
:10A7A80004108DF805208DF80730FFF77BFF01A80E
:10A7B800FFF758FFF0E700BF280E0020014B93F881
:10A7C80020007047280E0020034B93F8200004282F
:10A7D80094BF002001207047280E00201FB50024D8
:10A7E800CDE90244C41F8DF800408DF801100C0A11
:10A7F800ADF80420090C120C8DF803108DF8062012
:10A808008DF8073002461B0A012168468DF8024080
:10A818008DF8083003F089FD002818BF0E2004B019
:10A8280010BD2DE9F04188B090460D460F9A0746B5
:10A83800002847D000240121CDE904448DF81010E8
:10A848009DF838108DF81510ADF81630190CCDE9B3
:10A8580000441B0ECDE902448DF81930ADF81A20DA
:10A86800130C120E07948DF818108DF81C308DF803
:10A878001D20E3B21E01002DF6B203DC002008B053
:10A88800BDE8F081013310218DF81F3042466B4638
:10A898000DEB010003F0DFFC0346A8B9102D284694
:10A8A8003E44A8BF10206946327811F801CB013325
:10A8B80082EA0C02984206F8012BF5DC103D2DB215
:10A8C8000134D6E70920DAE70E20D8E70138032853
:10A8D80015D8DFE800F002080C100A4B1B681B694A
:10A8E8000B6000207047074B1B685B69F8E7054B56
:10A8F8001B689B69F4E7034B1B68DB69F0E70520DD
:10A90800704700BF4C0E00202DE9F041C4B00C4642
:10A918004A9E17461D468046B8B3B1F5807F36D8A3
:10A928004FF488720021684603F0A4FE492300937F
:10A938004FF48073ADF804302B0C8DF80830330CCD
:10A94800ADF80650ADF80A608DF80C3022460023A9
:10A95800414604A82D0E360E8DF80E308DF809509C
:10A968008DF80D608DF80F4003F070FE04F11001B2
:10A978004B9A3B4689B2684603F057FC10B1012850
:10A9880018BF0E2044B0BDE8F0810920FAE70D2079
:10A99800F8E7000010B590B10A4C28220021206089
:10A9A80003F068FE2368084A1A6000204FF0FF325F
:10A9B800C3E90302C3E90522C3E9072210BD082041
:10A9C800FCE700BF4C0E002000010101024B1B6890
:10A9D80018600020704700BF4C0E002030B1044BB7
:10A9E8001B68DB680133036000207047092070474B
:10A9F8004C0E002013B500230C460193CAB101A9DF
:10AA0800FFF764FF18B9019B591C02D1146002B00A
:10AA180010BD99B2611A002901DD5C18F6E702D170
:10AA280013600720F3E71B0C1B0403F580331C4459
:10AA3800ECE70920EBE7000028B1044B1B681C3346
:10AA48004362002070470920704700BF4C0E002069
:10AA58001FB5044600B3002303A8039303F0BCFC0E
:10AA6800104ABDF80C30126820469380E38200F04B
:10AA78005EFA98B904F118030093216801231322A0
:10AA880003F0C8FB60B9204600F051FA003818BF3F
:10AA98000120000104B010BD0920FBE71020F9E7F0
:10AAA8000E20F7E74C0E0020F0B5054687B01C468F
:10AAB80013B9092007B0F0BD2E4E3368DB68834216
:10AAC80055D894F82020002A0CBF08220922834276
:10AAD80005D3204600F05FFA68B11020EAE70023AA
:10AAE80001900093A36894F82810606AFFF799FE14
:10AAF8000028EED0DEE723792168B4F808C0A768FB
:10AB0800043B9AB20029D4D0B2F5807F2DD8ADF895
:10AB18000EC08DF817304FEA174C04F12C033F0E86
:10AB28008DF8117000932F0C08234FF0490EADF8E3
:10AB38000C008DF814708DF816002F0E0DEB030025
:10AB4800CDF808E08DF810C0ADF812508DF81570EA
:10AB580003F060FB08B10E20ACE7204600F01BFABA
:10AB68000028BAD13368DD60A4E70D20A2E70620EB
:10AB7800A0E700BF4C0E00202DE9FF410A9D80464A
:10AB88000F4616461C46002D5AD0002303A910462E
:10AB98000393FFF79BFE18B1062004B0BDE8F081CF
:10ABA800039B9C4201D80133F6D1284600F064F992
:10ABB800002847D1264B1A78424503D01A794245D6
:10ABC80042D10120AA68BA4240D103EB8002EB6A65
:10ABD80092F801802979CDE90043043992782868F0
:10ABE8003B4689B2FFF790FE0028D6D195F8203071
:10ABF8000194002B4FF00103009314BF4246082232
:10AC080095F82810686A3B46FFF70BFE0028C4D168
:10AC1800013E032EC1D8DFE806F002070B0F0D4BEB
:10AC28001B681C611C62B8E70A4B1B685C61F9E78A
:10AC3800084B1B689C61F5E7064B1B68DC61ACE7B9
:10AC48000920AAE70F20A8E70B20A6E70220A4E71F
:10AC5800F40000204C0E00201FB50B294FF0000314
:10AC6800CDE90033CDE902330A4607D00C2914D0C8
:10AC78000A2910D00A2005B05DF804FB012802D18A
:10AC880020238DF800300021684603F04EFB002891
:10AC980018BF0E20EFE73023F3E70B21F4E700009D
:10ACA80038B5054603F03CFB044610B10E24204697
:10ACB80038BD002DFBD1094B1B680B219878FFF795
:10ACC800CBFF0028F2D10C21FFF7C6FF0028EDD1F9
:10ACD8000A21FFF7C1FF0028E9D0E7E74C0E002062
:10ACE8002DE9F04380468FB00C461746002A6BD0FA
:10ACF800002969D0002529461D2206A8059505F0DA
:10AD080095FE8DF81350344D2B680DF114099E886B
:10AD1800CDF804900DF1130302933B7900933B683F
:10AD280032462146404603F01CFB00284ED13868C5
:10AD38003A79494603F08AFC384600F04FF8002873
:10AD480046D13C7AFA79BB79240444EA02241C43AC
:10AD58002B689A6894423DD99C609DF813000B219A
:10AD6800FFF77AFF034658BB0C21FFF775FF034630
:10AD780030BB0A21FFF770FF034608BB7B7ABA7A1B
:10AD8800FF7A3F0447EA02271F433A4633462146E3
:10AD98000920FFF723FD034690B933463A4621467A
:10ADA8000820FFF71BFD034650B92A689DF81310C9
:10ADB80091700021D1604FF0FF31C2E90411916117
:10ADC80018460FB0BDE8F0830923F9E70E23F7E72B
:10ADD8000F23F5E70323F3E74C0E002010B50446D4
:10ADE800002845D00168002942D011F8013B437181
:10ADF8000322063003F02AFC2046032250F8091BE0
:10AE0800043103F023FC2168CB79E3600A7A43EA32
:10AE18000223E3604A7A43EA0243E3608A7A43EA18
:10AE28000263E360CB7A23740B7B63742379212B51
:10AE38001AD110220D3104F1120003F007FC1D2273
:10AE48002168501C8B5C6362085C43EA0023901CF9
:10AE58006362085C033243EA004363628A5C43EA44
:10AE680002636362002010BD112B03DC0D22E7E7AB
:10AE78000220F8E70120F6E710B50446002854D070
:10AE88000168002951D00B7843714B7883608A7828
:10AE980043EA02238360CA7843EA024383600A795B
:10AEA80043EA026383604B7903738B79C381CA7960
:10AEB80043EA0223027BC38102F00F0208311030FB
:10AEC80003F0C4FB237B002203F00F0384F8202047
:10AED80084F82820227903F10800111A04290DDDCD
:10AEE80021680933043AD21A085C84F82000D2B2E7
:10AEF800606A84F82820194403F0A8FB23792268A3
:10AF08001A44002012F8043CE36212F8031C43EAD6
:10AF18000123E36212F8021C43EA0143E36212F8D8
:10AF2800012C43EA0263E36210BD0220FCE710B57E
:10AF3800044660B3036853B30279162A29D94279C3
:10AF48001A700146082251F8060B013003F088FBFD
:10AF58002146082251F80E0B093003F081FB2368C3
:10AF6800E28A5A74E38A22681B0A93742368A269E6
:10AF7800DA74A36922681B0A13752368628B5A75F1
:10AF88002368E27E9A7517232371002010BD0120E3
:10AF9800FCE70220FAE738B50446002863D00168C8
:10AFA800002960D0037B90F8282003F00F03002AC3
:10AFB80057D10833207904321344984255D3637922
:10AFC8000B702368A2685A70A36822681B0A9370E2
:10AFD80023686289DA702368E27A1A712368227B0F
:10AFE8005A712368E2899A71E38922681B0A21460B
:10AFF800D371227B51F8100B02F00F02083003F0D6
:10B0080025FB237B94F8282003F00F0303F10805A0
:10B018002AB1226894F82010515503F109052068D7
:10B0280094F82820616A284403F010FB94F828302B
:10B038002268E16A2B44D1545A1CE16A206892B212
:10B04800090A81549A1C2168E08D92B28854DA1C4E
:10B05800216894F82F0092B2043388542371002099
:10B0680038BD0933A6E70120FAE70220F8E7000017
:10B07800024B1A8810431880704700BF500E0020FA
:10B0880008B5074B1B883BB1FEF7CAF9002814BF67
:10B098006FF00200002008BD6FF00100FBE700BF61
:10B0A800500E002010B5034B00241C80FEF7AEF9AB
:10B0B800204610BD500E002008289DBF40F22113E5
:10B0C80023FA00F000F00100002070470346052B2A
:10B0D80082B0084605D0082B06D043B902B000F06C
:10B0E80065B902B001F05CBA02B001F07DBF002082
:10B0F80002B070470346052B084604D0082B04D03D
:10B108002BB900F009BA01F0E3BA02F00FB87047A2
:10B118000346052B084604D0082B04D02BB900F0B1
:10B1280017BA01F0F1BA02F01DB870470346052BB3
:10B138000846114604D0082B04D02BB900F05CBA9D
:10B1480001F04ABB02F098B8002070470346052B6F
:10B15800084604D0082B04D02BB900F0AFBD01F08D
:10B168009FBE02F0ADB870470346052B084604D0D1
:10B17800082B04D02BB900F06BBA01F053BB02F0D6
:10B18800CBB80020704710B40446052C0846114679
:10B198001A46019B05D0082C06D044B910BC00F013
:10B1A80071BA10BC01F058BB10BC02F0F1B810BC69
:10B1B80070470346052B0846114604D0082B04D0D7
:10B1C8002BB900F091BA01F079BB02F00DB900205B
:10B1D800704710B40446052C084611461A4605D097
:10B1E800082C06D044B910BC00F0F6BA10BC01F027
:10B1F800DDBB10BC02F052B9002010BC704730B45F
:10B208000446052C084611461A46DDE9023506D0E3
:10B21800082C08D05CB9029530BC00F06BBB0295D5
:10B2280030BC01F051BC029530BC02F0C3B900201B
:10B2380030BC70470346052B084604D0082B04D0C1
:10B248002BB900F00FBC01F0EDBC02F0AFBA002042
:10B2580070470346052B084604D0082B04D02BB9A9
:10B2680000F06ABD01F05ABE02F0C9BA002070476A
:10B278000346052B084604D0082B04D02BB900F050
:10B288000CBC01F0EDBC02F0BDBA002070470346CB
:10B29800052B084604D0082B04D02BB900F000BCBD
:10B2A80001F0E2BC02F0B1BA002070470346052B5A
:10B2B8000846114604D0082B04D02BB900F012BC64
:10B2C80001F0FABC02F0A4BA0020704710B404469A
:10B2D800052C084611461A46019B05D0082C06D0B5
:10B2E80044B910BC00F000BC10BC01F0E7BC10BCB5
:10B2F80002F0A4BA092010BC704710B40446052C0B
:10B30800084611461A4605D0082C06D044B910BC88
:10B3180000F034BD10BC01F022BE10BC02F02EBB00
:10B32800C8B210BC70470000004870470100010215
:10B33800064B10B51B6A0446984730B10448054BC4
:10B34800204498428CBF0020012010BD101A01082B
:10B35800403576C9405DC600F0B5114B85B00C4646
:10B3680010491F56054601F061F80F4BE4B25E6ABA
:10B37800072D4FF00103CDE9024301460AD105220A
:10B388000023CDE900234FF47A727A431846B04778
:10B3980005B0F0BD08220020CDE900203A46F5E7C7
:10B3A8003C1301081C130108101A01081FB50023DB
:10B3B80000930378013B372B21D8DFE803F01C24E6
:10B3C8002020201E202020204143454E2055585B38
:10B3D8005E6164206C1E6E73787A7D207F832620E0
:10B3E80020202020202020202020202085878C201D
:10B3F80020858C208E92C3780BB10223009300988D
:10B4080005B05DF804FB8378F6E743788DF80430DF
:10B4180007238DF805308378003B18BF01235B00B4
:10B428008DF8063010238DF80730314B1B6801A8C2
:10B4380003F55872CDE9022300F0D8FF0090DEE74B
:10B448004023DBE72023D9E7827890F9013012B94D
:10B45800284AD35CD2E7284AFBE7827890F9013082
:10B46800002AF8D1254AF4E740F6B833C6E74FF486
:10B478007A73C3E74FF4FA63C0E741F28833BDE754
:10B4880041F27073BAE71E484FF47A7103F0C2F8BC
:10B4980000F5FA60D2E71B4BB0E7154B1B6803F5C4
:10B4A8005873ABE7124B1B6803F55B73A6E71023D1
:10B4B800A4E70F4B1B68A1E701239FE74FF08343E5
:10B4C80000939CE7104BFBE7104B97E740F21113F2
:10B4D800ADF8003093E7032390E790F901300C4A68
:10B4E800B7E70C4990F9010000F0A0FFA6E700BFFC
:10B4F800580E00201113010801130108091301084F
:10B5080018FCFFFF00EA06379A99094040F7093707
:10B518003C1301081C13010837B50B4B02781B6854
:10B528000C2101FB02335B7A03EB4304074B1D68D4
:10B5380003690093C3684278816805EBC40000F092
:10B54800F0FC03B030BD00BF580E0020540E0020A0
:10B5580030B587B0027B6423ADF80030012A4FF084
:10B568000003CDE90133CDE903338DF802308DF8BE
:10B57800143028D0022A2FD01ABB03680BB34368B3
:10B58800FBB11A4C80682360194B18226946186071
:10B5980003F05CF8174B246893E807000C3384E841
:10B5A800070093E8070004F10C05032385E807006A
:10B5B800A4F86C33012204F55B7104F5587000F0AF
:10B5C800A1FC07B030BD094908684360036100F574
:10B5D8005B7100F55870F2E7044B1B68B3F8602301
:10B5E800B3F86C130A43A3F86023EAE7580E002067
:10B5F800540E0020E00B010808B503460A2924D898
:10B60800DFE801F006232323230B161B2321210047
:10B61800BDE808400068FFF78BBE90F900009978F4
:10B62800072271B900F02EFC003818BF012008BDB0
:10B63800052293F900000021F4E790F900005978F9
:10B64800EEE70221EEE70722F3E70020EFE700002C
:10B6580008B502791AB1012A0BD0002008BD084BA1
:10B6680001681B68012203F5587000F04BFC0120AB
:10B67800F4E7034B01681B6803F55B70F5E700BF4F
:10B68800580E0020F7B50728144D1C46A8BF072000
:10B6980058700E462946174600F0C8FE94F9013046
:10B6A800A070072B13D1322000F0C0FD0C4BDB6DCE
:10B6B8000546984704F10C020834034601920094A9
:10B6C8003A463146284600F0B6FD03B0F0BD054ABB
:10B6D80055F82310D05C00F0A1FDE7E71C13010822
:10B6E800101A01083C1301082DE9F04F344F90F966
:10B6F80001607B68D0F804908BB004468846984770
:10B708000546002859D1E37C73B92E4A237812687C
:10B7180003EB4303990002EB8303D3F80490B9F1D8
:10B72800000F01D152F80190274B484613F906B093
:10B73800FB689847A37C2289D7F818A00993072E9D
:10B7480028D100230121CDE90223204A0693CDE91F
:10B758000431CDE907330521CDE900214FF47A7290
:10B7680002FB0BF24CF250311846D047637C13B3FE
:10B77800174B995D7B6D0D31C9B228469847E07C1F
:10B788003246494600F064FE88F8006001200BB09C
:10B79800BDE8F08F002101250823CDE90013CDE98C
:10B7A8000715CDE90511CDE903110292A1782B46C1
:10B7B8005A462846D9E7074BDBE70020E7E700BFF2
:10B7C800101A0108580E00203C1301088545010095
:10B7D80009130108111301082DE9F04F8DB090F9F4
:10B7E8000130DFF8FCA0DFF8FC90CDE90A123E4AF0
:10B7F80012F903B00278DAF800300C2505FB0233A1
:10B808003A4A5B7A126803EB430302EBC30304462C
:10B8180093F9021090F9020000F003FE344906463D
:10B8280094F9010000F002FEA26861688046304683
:10B8380000F029FD2178DAF80020D9F80C306943A6
:10B84800074650589847D9F81C309C4694F901305F
:10B858000025072B4FF47A63CDE90753CDE9055549
:10B868002DD10123CDE903530523CDE901534FF42D
:10B878007A7303FB0BF300933946434646F2A8124A
:10B8880028466746B8472378DAF800200C214B434E
:10B8980094F90110D05800F0FDFDA18994F9010038
:10B8A800FFF75AFD0B9B217B1860D9F854302846C6
:10B8B80098470A9B01201E700DB0BDE8F08F01204B
:10B8C8000823CDE90350CDE901032A46CDF800B09D
:10B8D800654643463946A84701200546D3E700BFD9
:10B8E800580E0020101A01083C130108540E0020BD
:10B8F8001C1301082DE9F04F8FB0002405468A4635
:10B90800914698460494ADF81440ADF802400726D5
:10B918004FF0010B2B7AA34206D9686804A920448A
:10B9280000F014FC00285DD102238DF8083002A82D
:10B938006B7A8DF80A30FFF739FDAB7A8DF81D3038
:10B948009DF811308DF81E309DF812308DF81F309B
:10B958009DF810308DF82030EB7A8DF821302B7B54
:10B968008DF822306B7B8DF8233010238DF81C6006
:10B978008DF824303A4E8DF82C000DF102030A930D
:10B98800072332688DF82D30ADF834302B680C92CF
:10B9980006930DF1120204AB0DF1110106A800F097
:10B9A800EFFB072805460BD130680C22002100F573
:10B9B800587002F05FFE3368BDF80220A3F86023D8
:10B9C8009DF811308AF800309DF8123089F800305F
:10B9D8009DF8103088F80030189B28461C700FB06E
:10B9E800BDE8F08F9DF81330BDF81470ADF8027003
:10B9F8002044C4B2F3B917B3194A002011680726C6
:10BA080002464FF00C0C062B1BD10CFB00FE51F824
:10BA18000EE0BEF1000F04D00BFA00F23A4397B2E1
:10BA2800012201301028EED1002A3FF473AFADF89F
:10BA380002706FE75A1E042A01D9062BDCD00626AD
:10BA480068E747FA00FE1EF0010FEAD00CFB00FE83
:10BA580051F80EE0BEF1000F08BF0626E1E700BF6F
:10BA6800580E002038B505464068FFF761FC0722EC
:10BA7800841D002195F90000E4B200F003FA08B92A
:10BA880004F0FD0495F901000722002100F0FAF9FD
:10BA980008B904F0FB04204638BD002070470000B8
:10BAA80010B503780F2B044618D84068FFF740FC00
:10BAB80022780B4902EB42020968831C01EB8200E1
:10BAC80051F82220DBB21AB903F0FD0358B210BDB9
:10BAD800032B06BF626842600223F7E70020F6E7FF
:10BAE800580E0020022070472DE9F0413A4D0446D7
:10BAF800286896B00E46904600211F46012203236F
:10BB080000F55870CDE90411CDE906118DF80C1037
:10BB18008DF80D10ADF80E3000F0D6F930B92A685E
:10BB2800B2F8603343F00303A2F860332A68637AFB
:10BB38008DF8203002F55871CDE90912274A94F999
:10BB4800083012680B921022ADF830200DF10E0269
:10BB58000D9222680E9262680F92D4E90301A27ACC
:10BB68008DF8402001228DF8412011AA82E80300B7
:10BB7800227DE18A8DF8213018468DF84C20FFF798
:10BB8800EBFB08AB15930DF10D0314900093CDF862
:10BB9800048003AB04AA39460EA800F0E3FB044670
:10BBA80078B99DF80C10013902F034FD00F1580302
:10BBB8000DEB030010F8483C3370204616B0BDE882
:10BBC800F0810C2801BF2A68B2F8603343F0030300
:10BBD800A2F86033F1E700BF580E0020540E002091
:10BBE800F8B50679012E054648D90F2E48D80368BE
:10BBF800187A40F303000722002140B200F042F90E
:10BC08002B680446187A40F303100722002140B23B
:10BC180000F038F9B8B1B4FA84F4640929680B7AE9
:10BC2800086843F3030243F303135BB252B29A4228
:10BC3800C8BF0124FFF77CFB80F00103DBB224B10D
:10BC48000533D8B2F8BD0124E8E7DBB90E4F2968FF
:10BC58003B6806EB460003EB80000C2202F0F6FC82
:10BC68003A680C2303FB062320465C72B2F8601383
:10BC78000123B3400B43A2F86033E3E70620E1E772
:10BC88000320DFE70420DDE7580E002010B4017818
:10BC980001290ED9084B18680C234B43C4180022FD
:10BCA800C250C4E9012200F5587010BC102200F0FF
:10BCB800F2B8002010BC7047580E00202DE9F04162
:10BCC80086B050238DF81430037A102B074630D1F4
:10BCD8004368DD7B6DBB0224A8466426062C14D875
:10BCE8007A68535D03932A44517843EA0123039306
:10BCF800927843EA02437343CDE9033863B968464F
:10BD08008DF80040FFF7C2FF0DE0CDF80C808DF8EC
:10BD18001480CDF81080F2E703AB01A801938DF8E9
:10BD28000840FFF75DFF0134E4B2102C05F103056C
:10BD3800D4D106B0BDE8F0811FB502680379116857
:10BD480049B901A88DF80430FFF7A0FF78B10320A6
:10BD580005B05DF804FB02A802928DF80C30FFF7DD
:10BD68003FFF042805D0052805D00028EFD0002083
:10BD7800EEE70220ECE70120EAE70000C90020B95D
:10BD8800034B0B449856C0B27047024BF9E700BF0B
:10BD9800C1120108811201082DE9F3410023CDE900
:10BDA80000330E469046074618B9032002B0BDE896
:10BDB800F0810029F9D0002AF7D00C786308E00751
:10BDC80037F813104FF0000354BFC9B2090A1D46D3
:10BDD80041FA03F2D20706D505F108026A44013593
:10BDE80002F8083CEDB20133082BF1D16DB1691EA0
:10BDF800002002F00FFC00F108030DEB030010F81F
:10BE0800083C03EBC40388F800300134E4B2082C82
:10BE180028BF00241DB93378A342CFD1C5E73470B9
:10BE28000020C3E702FB00107047F0B59A42069D58
:10BE380003DB9DF914309A4220DD0020F0BD03EBAE
:10BE4800430331F814C005EB830300264CFA06F7C8
:10BE5800FF0707D51F7A07F00F0E964502DCB2EBF5
:10BE6800171F0DDD0136102E03F10C03EED101343E
:10BE7800E4B22301DBB29842E1D8DEE70024F8E718
:10BE88000120DBE7884204DB9042CCBF0020012080
:10BE980070470020704710B51409B4EB111F034612
:10BEA8004FEA11100ED391420CD202B201F00F01E9
:10BEB80033F81240012000FA01F124EA010123F8C5
:10BEC800121010BD0020FCE7F0B528B100EB4105C9
:10BED80001270020914200D3F0BD002435F802CBA1
:10BEE800234607FA04F636EA0C0608BF013304F1C4
:10BEF800010408BFDBB2102CF3D118440131C0B2E1
:10BF0800C9B2E7E710B500B149B910BD31F813401F
:10BF180020F813400133DCB2A242F7D8F5E700233A
:10BF2800F9E782B030B504880493D2B9B3F5616FEC
:10BF380015D349F6AF2542F21072AB4298BF4FF4C1
:10BF48007A72944238BF14466143BDE83040C368F2
:10BF58008B428CBF5B1A0023C36002B07047642217
:10BF6800EFE7012C38BF0124EEE700002DE9F04F80
:10BF78008FB01546199F03939DF8603007930C46C0
:10BF8800804604F009FB6A4A0590A7F5F633303B72
:10BF9800B3FBF2F3534303F5F63B0493182313FB67
:10BFA80005430BF1300B069300254FF0FF3A069B33
:10BFB8009C4207D1002D14BF50464FF0FF300FB000
:10BFC800BDE8F08FBDF96830ADF8243009991997AC
:10BFD8003846089704F070FA2688B8F1000F5FD148
:10BFE800B7F5616F5AD349F6AF2242F21073974200
:10BFF80098BF4FF47A739E4238BF1E46642E59D1BB
:10C00800DFF83091A060A1680CA804F077FA0D9BC6
:10C018000093DDE908120C9B0AA804F0CEF9039AF4
:10C028000A9B0AB9079A2AB122694A4502D1424AAB
:10C0380093420ED9414BC4F80C909F4209D9002372
:10C04800ADF82C300B99CDF828B0584604F034FAE6
:10C05800A060606808B9C4F80C90C4F81090B8F1F2
:10C06800000F04D004F0A2FAE3680344E360D4E9C3
:10C0780003329342059B88BFE26063601B9BE168C3
:10C088007343994204D20398E8B9B8F1000F1AD063
:10C0980001231D442375EDB2183488E76423AAE709
:10C0A800039B0BB9234BE360012EDFF8889038BF60
:10C0B8000126CEE7B6F57A7F0ABFDFF88490DFF86D
:10C0C8008490A0609FE700209342207506D85B1AF1
:10C0D8009A4505F1010528BF9A46EDB2B8F1000F5F
:10C0E800DAD1642E184AADF82C801DD049F6B02359
:10C0F800B6F57A7F18BF1346974281BF049A02F5B6
:10C10800A83202F5C0729B180A931A9B00930AAED4
:10C1180096E80600199B304604F04FF996E80300AC
:10C1280004F0CAF98246B7E74FF46163E4E700BF59
:10C138008051010040771B007F5101002FEC010066
:10C1480080A81201002E930230EC01000378032B23
:10C1580014D1437803F00F021B098A704B7083785F
:10C168008B80C27843EA02238B800379C3F30212DF
:10C1780003F00F03CA700B7005207047002070474A
:10C188002DE9F3479A464379057990F90760914676
:10C19800044690F906208846D3B190F90870002D1E
:10C1A80037D00F2A1BD194F909200F2E27D194F9E3
:10C1B8000A00072D02D1002F08BF012788F80020A8
:10C1C80089F8000028468AF8007002B0BDE8F087B8
:10C1D80090F90B7090F9092090F90A60DFE7A369DC
:10C1E800019394F91530009394F914302169207B58
:10C1F800FFF71BFE0028D8D105F0FD05D5E794F917
:10C208001D00B042D5DC94F91C30B34203DA05F0C6
:10C21800FB053046D2E73046CBE70000024B03FA75
:10C2280000F0B0FBF1F0704740420F004FF4FA53B2
:10C23800B3FBF0F0704730B54FF47A750C1F6A43C2
:10C2480000FB042252001EBF00F1FF341219B2FB9A
:10C25800F0F2914238BF1146039A116082004843B8
:10C268001CBF013040084FF47A71121A01FB1323E6
:10C27800002BCABF03F2E73393FBF1F1B3FBF1F1F3
:10C28800049B196030BD38B5400014460D46F4F7DC
:10C29800ABFC01462846F4F7F5FB2146F4F7F2FB20
:10C2A800F4F7D2F804F0F0FBF4F7C0FB40B238BD65
:10C2B8002DE9F74F019300239C469E46048A1E01F0
:10C2C800F6B2B44246D906EB46054FEA4309AD003B
:10C2D8000024476837F809702741FF0729D5876880
:10C2E80007EB050A7F5927B3077837B9476927B19C
:10C2F80037F809702741FF071BD59AF8087090F99D
:10C3080001B047F303084FFA88F8D84511DC47F322
:10C3180003177FB25F450CDB9AF8097007EB4708F3
:10C32800C76807EBC8073F7D5FB90CF1010C5FFADE
:10C338008CFC0134102C05F10C05CAD10133DBB299
:10C34800BCE70EF1010706EB040801F80E805FFA5E
:10C3580087FEEEE7019B82F800E083F800C003B097
:10C36800BDE8F08F2DE9FF4704464068DDE90C671A
:10C378001D468A46914604F019F923681B1A3B604A
:10C388004FF000080123337085F80080636813B10B
:10C398002368834224D8D4F81CC0CAF80080A36953
:10C3A8009CF800E00393D4E9030101AB83E80300A0
:10C3B800237D0093DCF80C10237A627A7046FFF72D
:10C3C800D5FD334638602A46E0694946FFF770FFD5
:10C3D8002B782BB1C7F80080002004B0BDE8F087A7
:10C3E8003378002B0CBF0C200B20F6E737B590F9FB
:10C3F800002090F90250954204460FD0013A52B2FB
:10C4080095420BD0A368019394F9013000936168B9
:10C41800E0782B46FFF709FD0028EFD0104603B05F
:10C4280030BD8842B8BF08467047000051F8200068
:10C43800054B984205D0054BC31A58425841400055
:10C4480070470120704700BF90D0030020A107006B
:10C4580005281FB50ED80C4B53F820300093CDE9B2
:10C4680001120A4B01220021022003F0ADFD05B0A4
:10C478005DF804FBCDE90012054B012200210220E2
:10C4880003F0A2FDF3E700BFAC1301084413010851
:10C498006313010807B5054BCDE90001012200210E
:10C4A800022003F091FD03B05DF804FB7F1301083F
:10C4B800F0B5114B85B00C4610491F560546FFF7DD
:10C4C800B5FF0F4BE4B25E6A072D4FF00103CDE9CB
:10C4D800024301460AD105220023CDE900234FF487
:10C4E8007A727A431846B04705B0F0BD082200209A
:10C4F800CDE900203A46F5E7F4130108D413010802
:10C50800101A010838B5194B1B6A04460D4698479E
:10C5180058B1174B174A2344934207D9164B174A69
:10C52800234493420CD800232B7038BD0223FBE729
:10C538000123F9E70523F7E70323F5E70423F3E7E6
:10C548000F4B104A23449342F2D90F4B0F4A23440E
:10C558009342EFD90E4B0F4A23449342ECD90E4B2A
:10C568000E4A23449342E9D90020DEE7101A010855
:10C5780040AA8FCC7F841E00C02571CCC0C62D0078
:10C58800FF5E43CCBF270900A0B038CC20A107002C
:10C5980040022ECC90D00300606E29CCE0930400BA
:10C5A8001FB50023009303780B3B2D2B68D8DFE8D9
:10C5B80003F02C2F31363A3C3F4245484B675367CE
:10C5C800555A5F616767646B17676767676767676F
:10C5D800676767676767536D7267675372677478D1
:10C5E80043788DF8043007238DF805304FF48053D5
:10C5F800ADF806302E4B1B6801A803F55872CDE93B
:10C608000223FFF7F3FE00903AE04023009337E05F
:10C618002023FBE790F90130264AD35CF6E790F92E
:10C628000130254AF9E70123F0E740F6B833EDE792
:10C638004FF47A73EAE74FF4FA63E7E741F2883395
:10C64800E4E741F27073E1E71C484FF47A7101F0B6
:10C65800E1FF00F5FA60D6E7194BD7E7144B1B68E2
:10C6680003F55873D2E7124B1B6803F55B73CDE7EC
:10C678001023CBE70E4B1B68C8E74FF083430093AA
:10C68800009805B05DF804FB0E4BF8E740F2111373
:10C69800ADF80030F4E70323B8E790F901300A4A0F
:10C6A800BBE70A4990F90100FFF7C0FEABE700BFFE
:10C6B800600E0020CC130108C413010818FCFFFF0A
:10C6C80008E6D3339A990940F4130108D4130108F2
:10C6D80037B50B4B02781B680C2101FB02335B7AE0
:10C6E80003EB4304074B1D6803690093C368427852
:10C6F800816805EBC400FFF714FC03B030BD00BF30
:10C70800600E00205C0E002030B5A5B004468E22D5
:10C7180000210DF1020004F089F94FF47A72ADF8A6
:10C728003020ADF87820227B64230A21012AADF855
:10C738000030ADF81830ADF84810ADF860302FD0A3
:10C74800022A38D052BB236843B3636833B31F4D02
:10C75800A0682B601E4B90226946186001F076FF96
:10C768001C4B2C6893E8070084E8070003F10C02CF
:10C7780007CA04F10C05183385E8070093E8070099
:10C7880004F11805072385E80700A4F86C33012293
:10C7980004F55B7104F55870FFF7B4FB25B030BDA4
:10C7A8000A4B1868002343600361C36100F55B719D
:10C7B80000F55870F0E7054B1B68B3F86023B3F831
:10C7C8006C130A43A3F86023E8E700BF600E00205B
:10C7D8005C0E0020F80B010807B50F291FD8DFE809
:10C7E80001F00C1E1E1E1E1C121C1E1C1C1E1E1ED2
:10C7F8001E08012003B05DF804FB0DF10701006875
:10C80800FFF780FEF6E7052290F900000021FFF708
:10C8180039FB003818BF0120ECE70722F4E70020B5
:10C82800E8E7000008B502791AB1012A0BD0002008
:10C8380008BD084B01681B68012203F55870FFF713
:10C8480061FB0120F4E7034B01681B6803F55B708B
:10C85800F5E700BF600E0020F7B50728144D1C4609
:10C86800A8BF072058700E4629461746FFF7DEFD79
:10C8780094F90130A070072B13D13220FFF7D6FCB2
:10C888000C4BDB6D0546984704F10C02083403464F
:10C89800019200943A4631462846FFF7CCFC03B093
:10C8A800F0BD054A55F82310D05CFFF7B7FCE7E761
:10C8B800D4130108101A0108F41301082DE9F04FE8
:10C8C800344F90F901607B68D0F804908BB004462F
:10C8D800884698470546002859D1E37C73B92E4A03
:10C8E8002378126803EB4303990002EB8303D3F820
:10C8F8000490B9F1000F01D152F80190274B484636
:10C9080013F906B0FB689847A37C2289D7F818A0CA
:10C918000993072E28D100230121CDE90223204ABB
:10C928000693CDE90431CDE907330521CDE900218E
:10C938004FF47A7202FB0BF24CF250311846D04792
:10C94800637C13B3174B995D7B6D0D31C9B22846D3
:10C958009847E07C32464946FFF77AFD88F8006040
:10C9680001200BB0BDE8F08F002101250823CDE997
:10C978000013CDE90715CDE90511CDE903110292A0
:10C98800A1782B465A462846D9E7074BDBE7002013
:10C99800E7E700BF101A0108600E0020F413010831
:10C9A80085450100C4130108CC1301082DE9F04F97
:10C9B8008DB090F90130DFF8FCA0DFF8FC90CDE9EC
:10C9C8000A123E4A12F903B00278DAF800300C2550
:10C9D80005FB02333A4A5B7A126803EB430302EB26
:10C9E800C303044693F9021090F90200FFF719FDFA
:10C9F8003449064694F90100FFF718FDA2686168FA
:10CA080080463046FFF73FFC2178DAF80020D9F855
:10CA18000C306943074650589847D9F81C309C4653
:10CA280094F901300025072B4FF47A63CDE90753B9
:10CA3800CDE905552DD10123CDE903530523CDE9D2
:10CA480001534FF47A7303FB0BF3009339464346C3
:10CA580046F2A81228466746B8472378DAF8002035
:10CA68000C214B4394F90110D058FFF713FDA1890D
:10CA780094F90100FFF71CFD0B9B217B1860D9F886
:10CA88005430284698470A9B01201E700DB0BDE817
:10CA9800F08F01200823CDE90350CDE901032A4690
:10CAA800CDF800B0654643463946A84701200546FB
:10CAB800D3E700BF600E0020101A0108F413010824
:10CAC8005C0E0020D41301082DE9F04F8DB000242E
:10CAD80005468A46914698460294ADF80C40ADF852
:10CAE800064007264FF0010B2B7AA34206D9686847
:10CAF80002A92044FFF72AFB002854D1AB7A8DF80D
:10CB080015309DF809308DF816309DF80A308DF8EB
:10CB180017309DF808308DF81830EB7A8DF81930F9
:10CB28002B7B8DF81A306B7B8DF81B3010238DF81A
:10CB380014608DF81C303A4E0DF1060308934FF43B
:10CB4800E063ADF8243033680A930723ADF82C303E
:10CB58002B6804930DF10A0202AB0DF1090104A838
:10CB6800FFF70EFB072805460BD130680C22002181
:10CB780000F5587001F07EFD3368BDF80620A3F873
:10CB880060239DF809308AF800309DF80A3089F84A
:10CB980000309DF8083088F80030169B28461C7035
:10CBA8000DB0BDE8F08F9DF80B30BDF80C70ADF8F6
:10CBB80006702044C4B2F3B917B3194A00201168AB
:10CBC800072602464FF00C0C062B1BD10CFB00FE6F
:10CBD80051F80EE0BEF1000F04D00BFA00F23A4310
:10CBE80097B2012201301028EED1002A3FF47CAF21
:10CBF800ADF8067078E75A1E042A01D9062BDCD056
:10CC0800062671E747FA00FE1EF0010FEAD00CFB7A
:10CC180000FE51F80EE0BEF1000F08BF0626E1E75E
:10CC2800600E002037B505460DF107014068FFF793
:10CC380069FC0722841D002195F90000E4B2FFF782
:10CC480021F908B904F0FD0495F901000522002135
:10CC5800FFF718F908B904F0FB04204603B030BD0B
:10CC68004FF0FF307047000013B5027800230F2AF9
:10CC780004468DF807301BD80DF107014068FFF70F
:10CC880041FC22780B4902EB42020968831C01EB44
:10CC9800820051F82220DBB222B903F0FD0358B21A
:10CCA80002B010BD032B06BF626842600223F6E79C
:10CCB8001846F5E7600E0020704700002DE9F041A6
:10CCC8003A4D0446286896B00E46904600211F4605
:10CCD8000122072300F55870CDE90411CDE90611AA
:10CCE8008DF80C108DF80D10ADF80E30FFF7ECF83C
:10CCF80030B92A68B2F8603343F00703A2F860330A
:10CD08002A68637A8DF8203002F55871CDE9091246
:10CD1800274A94F9083012680B921022ADF8302097
:10CD28000DF10E020D9222680E9262680F92D4E9FC
:10CD38000301A27A8DF8402006228DF8412011AA1D
:10CD480082E80300227DE18A8DF8213018468DF8AB
:10CD58004C20FFF7ADFB08AB15930DF10D031490B4
:10CD68000093CDF8048003AB04AA39460EA8FFF758
:10CD7800F9FA044678B99DF80C10013901F04AFC1B
:10CD880000F158030DEB030010F8483C33702046BF
:10CD980016B0BDE8F0810C2801BF2A68B2F86033EC
:10CDA80043F00703A2F86033F1E700BF600E0020EC
:10CDB8005C0E0020F7B506790027022E05468DF88F
:10CDC80007704DD90F2E4DD80368187A40F3030029
:10CDD8000722394640B2FFF755F82B680446187AFF
:10CDE80040F303100722394640B2FFF74BF8D0B1A1
:10CDF800B4FA84F464092868037A006843F30302E8
:10CE080043F303135BB252B20DF107019A42C8BF54
:10CE18000124FFF777FB80F00103DBB22CB1053367
:10CE2800D8B203B0F0BD0124E5E7EBB90F4F29688C
:10CE38003B6806EB460003EB80000C2201F006FC81
:10CE48003A689DF807100C2303FB06232046597205
:10CE5800B2F860130123B3400B43A2F86033E0E754
:10CE68000620DEE70320DCE70420DAE7600E002076
:10CE780010B4017802290ED9084B18680C234B43CB
:10CE8800C4180022C250C4E9012200F5587010BC31
:10CE98001022FFF700B8002010BC7047600E002079
:10CEA8002DE9F04186B050238DF81430037A102B09
:10CEB800074630D14368DD7B6DBB0324A846642652
:10CEC800072C14D87A68535D03932A44517843EAAF
:10CED80001230393927843EA02437343CDE903386D
:10CEE80063B968468DF80040FFF7C2FF0DE0CDF842
:10CEF8000C808DF81480CDF81080F2E703AB01A800
:10CF080001938DF80840FFF755FF0134E4B2102C67
:10CF180005F10305D4D106B0BDE8F0811FB502685C
:10CF28000379116849B901A88DF80430FFF7A0FF0B
:10CF380078B1032005B05DF804FB02A802928DF8D1
:10CF48000C30FFF737FF042805D0052805D0002846
:10CF5800EFD00020EEE70220ECE70120EAE7881A8C
:10CF680040B220EAE070C0B27047000030B50B4B09
:10CF780085B00C460A491D56FFF758FA08220146A3
:10CF88000020CDE90020074A0123E4B2029403936C
:10CF9800546A18462A46A04705B030BD70140108E7
:10CFA80030140108101A01080B4B10B51B6A04460F
:10CFB800984768B1094B0A4A2344934209D8094A59
:10CFC800534341F6F632B2EBB31F2CBF01200020C9
:10CFD80010BD0020FCE700BF101A0108608FF7C8D9
:10CFE800401640005FF743591FB5002300930378AC
:10CFF800013B372B6CD8DFE803F01C6B6B6B6B6B5A
:10D008006B6B6B6B3436383D6B4144474A4D506B04
:10D01800581C5A5F64666B6B696B1F6B6B6B6B6B31
:10D028006B6B6B6B6B6B6B6B6F751C1C6B6F1C1C72
:10D038007D81082300934BE043788DF80430042366
:10D048008DF805304FF49043ADF806302E4B1B6831
:10D0580001A803F55872CDE90223FFF7C7F900903C
:10D0680036E04023E6E72023E4E790F90130274A39
:10D07800D35CDFE790F90130254AF9E740F6B83389
:10D08800D8E74FF47A73D5E74FF4FA63D2E741F261
:10D098008833CFE741F27073CCE71E484FF47A71BA
:10D0A80001F0B8FA00F5FA60D9E71B4BC2E7164B56
:10D0B8001B6803F55873BDE7134B1B6803F55B73D7
:10D0C800B8E74823B6E7104B1B68B3E7134B009348
:10D0D800009805B05DF804FB114A0F490079FEF786
:10D0E800A1FEBCE740F21743ADF8003003238DF8EA
:10D0F8000230EDE790F901300A4AB9E70A4990F998
:10D108000100FFF793F9AAE7680E00200C14010844
:10D11800FC13010818FCFFFFA07008379A99004219
:10D12800C0270900701401083014010837B50B4BEB
:10D1380002781B680C2101FB02335B7A03EB430482
:10D14800074B1D6803690093C3684278816805EB43
:10D15800C400FEF7E6FE03B030BD00BF680E002035
:10D16800640E0020F0B587B00123047BADF80030D1
:10D178000023CDE90133CDE903338DF802308DF872
:10D18800143024B1013C012C4ED907B0F0BD03681E
:10D19800002BFAD04268002AF7D0304E80683260FF
:10D1A8002F4A304D10609C81182269462B6001F08F
:10D1B8004DFA30682C4B2D4F024601464FF0300C8B
:10D1C8000B6003F5433303F5A073BB4281F808C035
:10D1D8004C7201F10C01F3D1254B26494427002458
:10D1E800C2F8003303F5C31303F520638B4282F8BA
:10D1F800087382F8094302F10C02F1D14FF0FF33B2
:10D20800C0E9DB33FF23C0F8743300F55B710622F5
:10D2180000F55870FEF776FE31682868062201F599
:10D228005871FEF76FFEB0E70C4C2068062200F537
:10D238005B7100F55870FEF765FE0A4B21681B68A4
:10D2480001F25E319A1E0A3332F8020F31F8024FAA
:10D258009A4200EA04001080F6D196E7680E002092
:10D26800640E00206C0E00206001C83560518B36BA
:10D27800C0AFD235C0FF953608B50A291DD8DFE8FA
:10D2880001F0061C1C1C1C0B0E101C1A1A00BDE811
:10D2980008400068FFF788BE0422002103E0052249
:10D2A800FBE70D22082190F90000FEF7EBFD00389E
:10D2B80018BF012008BD0E22EFE70020FAE70000A2
:10D2C800F0B5037A102B22D14468E37B012B1ED1E1
:10D2D8000F4B1D680F4B196805F25E3002390022AA
:10D2E800671C14F8123020F8023F17F81260042A5D
:10D2F80043EA0623038004BFDBB2A5F8683331F89C
:10D30800023F068801323340052A0B80E9D1F0BD7F
:10D31800680E00206C0E002070B50422044600211F
:10D328000068FEF7D1FD012803D025791DB1012D34
:10D3380021D000201EE0144E21683068062200F536
:10D348005870FEF7DFFD336893F87423A3F874234D
:10D358000E4AA3F87653126803F25E33911E0A321E
:10D3680031F8020F33F8024F914200EA04000880B6
:10D37800F6D1012070BD044B21681868062200F51B
:10D388005B70FEF7BFFDF4E7680E00206C0E00200E
:10D39800F7B50D28114DA8BF0D201C460E46587034
:10D3A80029461746FFF742F894F901300C4A55F818
:10D3B8002310A070D05CFEF731FF0A4BDB6D0546E9
:10D3C800984704F10C0208340346019200943A4647
:10D3D80031462846FEF72FFF03B0F0BD3014010890
:10D3E80070140108101A01082DE9F047DFF894803D
:10D3F80090F90160D8F8043047688AB00446894635
:10D40800984700283CD1E37C33B923781E4A1F4F44
:10D4180003F0070302FB03771D4B384613F906A0F8
:10D42800D8F80C309847A37C099300250123CDE94F
:10D438000753CDE90555CDE9035522890292082203
:10D44800CDE900521846D8F81850A1785246A84796
:10D45800637C9BB10F4B9B5D03F10D01C9B2D8F8FA
:10D46800543001209847E07C32463946FEF7F0FFF9
:10D4780089F8006001200AB0BDE8F087064BEAE7AA
:10D488000020F8E7101A0108C0270900A070083723
:10D4980070140108FC1301080C1401082DE9F04F61
:10D4A8003E4B90F901B0DFF8F8A013F90B70DAF8E9
:10D4B8000090037890F9026090460C2202FB0393D7
:10D4C800384A5B7A126803EB43038FB002EBC3035D
:10D4D8000B91044693F902103046FEF7A2FFBBF108
:10D4E800040F05464CD1022E3546B8BF02252E49F9
:10D4F80094F90100DFF8B490FEF798FF2C490D90DD
:10D5080000222846FEF7BFFE26780C904FF00C0B41
:10D51800DAF80000D9F80C200BFB06F68059904782
:10D52800012600224FF47A630820CDE90723CDE9CC
:10D538000522DDE90C13CDE90326CDE9016000974A
:10D548003046D9F81C70B8472378DAF8002094F9E7
:10D5580001100BFB03F3D058FEF79CFFD9F85430A9
:10D56800217B30469847A18994F90100FFF7FEFC1A
:10D578000B9BC8F8000030461D700FB0BDE8F08F57
:10D588000422002109F55870FEF79EFC3128AED818
:10D59800052E3546B8BF0525A9E700BF7014010858
:10D5A800680E0020640E002030140108101A0108CB
:10D5B8000000F0412DE9F04F7A4F93B0CDE9011208
:10D5C8003968039307AE00240546062201F5587111
:10D5D8003046C6E901440594ADF818400794FEF7B3
:10D5E80091FCA0464FF0FF392B7AA34205D9686811
:10D5F80005A92044FEF7AAFD60B99DF91530032B53
:10D6080065DC0422002107A8FEF75EFC01285ED82D
:10D6180006235DE09DF81730BDF818102044062B4E
:10D62800C4B205D1CDE90799C9B2ADF82410DBE73A
:10D63800072B02D1CDE90788F6E7052B41D14FF03A
:10D64800000CC9B260464FF0010B12AB0BFA0CF29A
:10D6580003EB400E11423EF82C3C0CF0010A1CD0A2
:10D6680092B2BAF1000F0ED143F0FF032EF82C3C12
:10D67800BDF8243013430CF1010CBCF1080FADF8D0
:10D688002430E2D1B0E763F0FF032EF82C3CBDF85C
:10D69800243013430130C0B2EDE7D24392B2BAF15D
:10D6A800000F07D123F0FF032EF82C3CBDF82430DF
:10D6B8001340E0E7DBB22EF82C3CBDF824301340D1
:10D6C800E8E712AA02EB430323F82C1C8CE7072394
:10D6D8008DF82C30AB7A8DF82D309DF815308DF8FB
:10D6E8002E309DF816308DF82F309DF814308DF8B7
:10D6F8003030EB7A8DF831302B7B8DF832306B7B04
:10D708008DF8333048238DF834304FF48063ADF80A
:10D718003C303B6810930E23ADF844302B680A93D5
:10D728000DF1160205AB0DF115010AA80E96FEF7CC
:10D7380027FD0728054623D138680622314600F51B
:10D748005870FEF7DFFB184B3A681B68B2F86003A5
:10D75800198801401980B2F862035988014059803C
:10D76800B2F86403998801409980B2F86603D988B1
:10D778000140D980B2F86813B2F86A2319815A8136
:10D78800019A9DF815301370029A9DF8163013709F
:10D79800039A9DF8143013701C9B28461C7013B014
:10D7A800BDE8F08F680E00206C0E002038B50546E5
:10D7B8004068FFF7F9FB0D22841D082195F9000048
:10D7C800E4B2FEF75FFB08B904F0FD0495F9000028
:10D7D80007220521FEF756FB012803D095F90030F2
:10D7E8000D2B01DD04F0FD0495F901000322002151
:10D7F800FEF748FB08B904F0FB04204638BD4FF09B
:10D80800FF3070474FF0FF3070474FF0FF307047E0
:10D81800094B1B68587B69B90130C0B25873C0EB1B
:10D82800C00300EBC300C0B21C288CBF002001203D
:10D83800800070470138F0E76C0E00202DE9F047B2
:10D848000025A4B04A4E8DF80E5004460F46914666
:10D858002946442213A898468DF80F50129503F0D4
:10D86800E5F829463068DFF80CA10422FEF72CFB06
:10D87800054648B9DAF800103068042201F55871F5
:10D88800FEF740FB33681D7394F908303268DAF804
:10D898000010032B04DD107A10B9B1F86803108169
:10D8A800CDE90521344A607A126807924822ADF81A
:10D8B80020200022099222680A9262680B92A27ABA
:10D8C8008DF810008DF83020D4E9030101228DF87D
:10D8D800312004AA11920DAA82E80300227DE18A70
:10D8E8008DF8113018468DF83C20FFF73FFB0DF1FD
:10D8F8000F0310900093CDF804900DF10E0312AAB7
:10D9080041460AA8FEF72EFD054690B9637AA3B1F1
:10D918009DF80E10013900F07DFE00F190030DEB2B
:10D92800030010F8483C3B70397830684822FEF70D
:10D93800B2FA284624B0BDE8F08794F90830306878
:10D9480063B1007A2B46D9B240FA01F1C9071A46E9
:10D9580003F10103F7D502F14003E4E73A4600F189
:10D968000C01FEF719FA0328DED10546E1E700BFEE
:10D978006C0E0020680E0020640E0020034B03EBA1
:10D988008103985620EAE070C0B270471C14010861
:10D9980010B5102204460021F13000F06BFE002182
:10D9A800C4F814112046F022BDE8104000F062BE11
:10D9B80002460846102100F0A5B92DE9F0430446B7
:10D9C800D0F8140185B00E46154604F2011988B343
:10D9D800C0F110089045474628BF1746BAB24844D8
:10D9E80000F034FED4F814313B440F2BC4F8143142
:10D9F8002DD9A8452BD204F1F00304F5807113F852
:10DA0800012F187C8B4282EA00021A70F7D104F1C8
:10DA1800F10810224146684600F018FE2246694681
:10DA2800684600F0F1F910226946404600F00EFE03
:10DA38003E44ED1B04F5807804F1F107102D09D858
:10DA4800AAB23146484600F001FEC4F8145105B0A8
:10DA5800BDE8F08304F1F003711E13F8012F11F8EB
:10DA6800010F434582EA00021A70F6D110223946A6
:10DA7800684600F0EBFD22466946684600F0C4F9A6
:10DA880010226946384600F0E1FD1036103DD5E712
:10DA9800F0B589B00C46102200210546684600F012
:10DAA800E9FD22466946684600F0AEF99DF9003066
:10DAB800002B6A464FF0000143DA137812F8010F81
:10DAC80001315B0043EAD0130F2902F8013CF4D17D
:10DAD8009DF80F305B0083F08703D4F81401DBB2A4
:10DAE80010288DF80F303BD104F58073694604F592
:10DAF800887013F8016F11F8012B984282EA060228
:10DB08001A70F6D104F1F00304F5807113F8012FAF
:10DB1800187C8B4282EA00021A70F7D110220DEBB2
:10DB2800020004F1F10100F091FD2246294604A803
:10DB380000F06AF910220021684600F09BFD09B048
:10DB4800F0BD137812F8010F01315B0043EAD013DE
:10DB58000F2902F8013CF4D19DF80F305B00BCE7B7
:10DB68009DF90030002B6A464FF0000137DA137830
:10DB780012F8016F01315B0043EAD6130F2902F84E
:10DB8800013CF4D19DF80F305B0083F08703471CFC
:10DB9800DBB28DF80F30102F04EB0003C0F10F0635
:10DBA8004FF0800288BF002600F5817083F80121BC
:10DBB8000021324620443E4402F038FFC4F8146184
:10DBC80004F58073694604F5887013F8016F11F83D
:10DBD800012B984282EA06021A70F6D192E713786E
:10DBE80012F8016F01315B0043EAD6130F2902F8DE
:10DBF800013CF4D19DF80F305B00C8E70A78037840
:10DC0800534003704A784378534043708A78837846
:10DC180053408370CA78C3785340C3700A79037934
:10DC2800534003714A794379534043718A79837920
:10DC380053408371CA79C3795340C3710A7A037A0E
:10DC4800534003724A7A437A534043728A7A837AFA
:10DC580053408372CA7AC37A5340C3720A7B037BE8
:10DC6800534003734A7B437B534043738A7B837BD4
:10DC780053408373CA7BC37B5340C373704710B54B
:10DC88000B7814786340037054784B786340437082
:10DC980094788B7863408370D478CB786340C37072
:10DCA80014790B796340037154794B79634043715C
:10DCB80094798B7963408371D479CB796340C3714C
:10DCC800147A0B7A63400372547A4B7A6340437236
:10DCD8008B7A947A63408372D47ACB7A6340C37226
:10DCE800147B0B7B63400373547B4B7B6340437310
:10DCF800947B8B7B63408373CB7BD27B5340C37312
:10DD080010BD0000A1F11003DBB2102B2DE9F04784
:10DD1800044604D83A4820FA03F3DB0705D4002365
:10DD280082F8F030FF20BDE8F087561E254615F82A
:10DD3800013B06F8013F631B0B4413F0FF00F6D1CB
:10DD480001F11C039B005FFA83FCC3F30313013B3F
:10DD5800DFF8B09082F8F030884653184FF0010E83
:10DD6800B8FBF1FA01FB1A8A1AF0FF0A13F8047CCF
:10DD780013F8036C13F8025C13F8014C30D119F84E
:10DD880006A019F8056019F8045019F807404FEA79
:10DD9800DE1707EB47078EEA0A0A07EBC7074FEAC1
:10DDA8004E0EFFB25FFA8EFE87EA0E0E574692F8C5
:10DDB80000A087EA0A071F7057787E405E70967841
:10DDC80075409D70D57808F104085FFA88F86C40B2
:10DDD800C445DC7002F1040203F10403C0D8A2E7D1
:10DDE8001829E4D9BAF1100FE1D1DFF818A01AF810
:10DDF80007701AF806601AF805501AF80440D6E7B2
:10DE080001010100801601082DE9F04FA3B092F836
:10DE1800F0301D911B920193002B00F053810146B5
:10DE28001EA8FFF72CFF1B9BA74CA84DA84E10332C
:10DE38000293002303939DF87C0004909DF88600CC
:10DE48000590205C06909DF87B000790205C089068
:10DE580004989DF881C0205C099014F80C000A9081
:10DE68009DF880000B909DF885009DF878809DF8BE
:10DE78007DE09DF882A09DF887900C909DF87A002F
:10DE8800029B1C9314F80A2014F8093014F808109F
:10DE980014F80E700D90205C0E909DF87F000F9086
:10DEA800205C10900B98205C11900C98205C1290CC
:10DEB8009DF8840013909DF8790014909DF87E00D9
:10DEC8001590205C16909DF883001790205C1890A0
:10DED8001398205C19901498205C1A9003980130CC
:10DEE80003900298DDF804B0103002909DF80C0001
:10DEF800834536D88DF878108DF87A2009990E9ACE
:10DF08008DF87C108DF882201199069A8DF8801072
:10DF18008DF87E201999169A8DF884108DF8862030
:10DF28000A99189A8DF87D108DF887201299109A01
:10DF38008DF87B301B9B8DF881108DF883201A9902
:10DF4800089A1D988DF885108DF87F201EA903EB7F
:10DF58000B128DF87970FFF792FE002023B0BDE810
:10DF6800F08F15F808B082EA03008BEA000016F873
:10DF78000EB080EA0B008DF8780015F80E004B40C3
:10DF8800434016F80A0043408DF8793081EA0703C8
:10DF980015F80A10594016F80930594016F8083093
:10DFA8008DF87A107A40534015F8092053408DF8BF
:10DFB8007B30089A069B5340049AAA5C534016F893
:10DFC8000C2053408DF87C30DDE908325A4015F8B2
:10DFD8000C305340059AB25C53408DF87D30DDE932
:10DFE80009325A40059BEB5C5340079AB25C534098
:10DFF8008DF87E30069B0A9A5340049AB25C5A40C8
:10E00800079BEB5C5A408DF87F200E9B109A53407B
:10E018000B9AAA5C53400C9AB25C53408DF880303E
:10E02800DDE910325A400C9BEB5C53400D9AB25C10
:10E0380053408DF88130DDE911325A400D9BEB5C7D
:10E0480053400F9AB25C53408DF88230129A0E9B5F
:10E0580053400B9AB25C5A400F9BEB5C1C995A4098
:10E068008DF88320169B189A5340139AAA5C534044
:10E07800149AB25C53408DF88430DDE918325A4066
:10E08800149BEB5C5340159AB25C53408DF8853075
:10E09800DDE919325A40159BEB5C5340179AB25C84
:10E0A80053408DF886301A9A169B5340139AB25CE7
:10E0B8005340179AAA5C1EA853408DF88730FFF783
:10E0C8009DFDB8E6FF2049E7801601088015010884
:10E0D8008014010808B538B1044A05491060D822EF
:10E0E80000F0B4FA002008BD0220FCE7700E002002
:10E0F80000E503080A4B1A6870B5002302F11805F9
:10E1080003EB03142E5D864204D1183422440A60BE
:10E11800002070BD01330B2BF2D10320F9E700BFBB
:10E12800700E00202DE9F041CCB00646DDF848819C
:10E1380017461C460D4631B3B8F1000F23D006A888
:10E14800FFF726FC204601A9FFF7D4FF0446B0B923
:10E15800019906A80131FFF72BFC26B110223146A0
:10E1680006A8FFF72AFC3A46294606A8FFF725FC29
:10E1780006A902A8FFF78CFC029BC8F800302046CD
:10E188004CB0BDE8F0810224F9E7000030B595B045
:10E1980013A90446FFF7AEFF002830D11B4B0C2112
:10E1A80001FB00F2D5189A5CA2422AD1139B1A7C73
:10E1B8001092DA7B0F929A7B0E925A7B0D921A7B01
:10E1C8000C92DA7A0B929A7A0A925A7A09921A7A05
:10E1D8000892DA7907929A7906925A7905921A7909
:10E1E8000492DA7803929A7802925B78019300227B
:10E1F800AB6800931146064B022001F0E5FE15B00E
:10E2080030BD01300B28CBD1F9E700BFF818010861
:10E218008017010810B40B2B019C03D8019410BC83
:10E22800FFF780BF032010BC704730B50D4685B09E
:10E238001446014668B103AA002000922A460390BA
:10E24800FFF770FF18B90398001B18BF012005B02D
:10E2580030BD0220FBE72DE9F0430D46BFB0144660
:10E268009946804620B31BB311F00F0122D1F0224A
:10E2780001A800F0FFF920466946FFF73BFF044676
:10E2880048B9009801AA10210130FFF73BFD2E463E
:10E29800AF1BFFB21EB920463FB0BDE8F08301AA0C
:10E2A80009EB070108EB0700FFF7AEFD103EEFE7AB
:10E2B8000224F0E70524EEE7F0B5184E346802466C
:10E2C80085B00846002304F1180103EB03154F5DE0
:10E2D80097421ED10D2A05F1190513D10023CDE966
:10E2E8000033CDE902330C2210216B46FFF7B3FF50
:10E2F8000446306810226946284400F0A7F92046F1
:10E3080005B0F0BD01461022601900F09FF9002405
:10E31800F5E701330B2BD8D10324F0E7700E00206A
:10E3280009B1FFF7C9BF022070471FB51446A0B155
:10E338000C2A01D10B2912D10023CDE90033CDE9F4
:10E3480002330A466B461021FFF785FF18B9694664
:10E358002046FFF7B1FF04B010BD0220FBE7032001
:10E36800F9E7F8B51E46DDE907479DF818505BB395
:10E3780054B34FB3212D29D819462A46204600F018
:10E3880065F90122631C691EB018FFF764FFF8B92C
:10E39800E37ADB093B70EBB96319204613F8012CCB
:10E3A80013F8021C120642EA014213F8041C0A433D
:10E3B80013F8031C012342EA0122291FFFF735FF46
:10E3C800003818BF0120F8BD0220FCE70520FAE755
:10E3D8000720F8E70420F6E710B5044628B1044BF7
:10E3E8005B6998472060002010BD0220FCE700BF51
:10E3F800101A010808B5014630B1044B0822186804
:10E4080000F024F9002008BD0220FCE7700E00206F
:10E4180008B530B1044B0822196800F017F900203C
:10E4280008BD0220FCE700BF700E00207FB5124E29
:10E438000023044602A801930D46FFF7E9FF33685D
:10E448005B6901936CB102AA082312F8011B41B958
:10E45800013B13F0FF03F8D102A8A04702A8FFF779
:10E46800C9FF35B1019B23B901A8A8473368019AB0
:10E478005A61002004B070BD700E002008B5014636
:10E4880038B1054B18680822104400F0DFF8002066
:10E4980008BD0220FCE700BF700E002008B538B1A7
:10E4A800044B19680822114400F0D0F8002008BD78
:10E4B8000220FCE7700E0020034B1B6802280CBFEB
:10E4C8001961596100207047700E002049B1064B50
:10E4D8001B68D3E90423022808BF13460B600020F9
:10E4E80070470220704700BF700E002030B58FB013
:10E4F800002405460CA80994FFF78AFF9DF83730D9
:10E5080007939DF8363006939DF8353005939DF8AE
:10E51800343004939DF8333003939DF832300293DE
:10E528009DF8313001939DF8303000932246214602
:10E538001E4B022001F048FD0AA8FFF7AFFF9DF827
:10E548002F3007939DF82E3006939DF82D300593B4
:10E558009DF82C3004939DF82B3003939DF82A30B6
:10E5680002939DF8293001939DF8283000932246A4
:10E578000F4B2146022001F027FD09A92846FFF785
:10E58800A5FF9DF8243003939DF8253002939DF84C
:10E59800263001939DF8273000932246054B2146EB
:10E5A800022001F011FD0FB030BD00BFDC170108DB
:10E5B8001A1801085818010808B50020FFF7E6FDE9
:10E5C8000120FFF7E3FD0920FFF7E0FD0820FFF732
:10E5D800DDFD0020FFF78AFF002008BD10B50446C6
:10E5E8000B20FFF7D3FD0C20FFF7D0FD0920FFF724
:10E5F800CDFD0820FFF7CAFD0A20FFF7C7FD20461A
:10E60800FFF774FF002010BD014B1860704700BF72
:10E61800FC0000200B4A30B514680B4D43F2390357
:10E6280005FB04331360091A6FF00042B3FBF2F2E2
:10E63800C2EBC27201319B1A93FBF1F201FB123358
:10E64800184430BDFC0000206D4EC64101380A4414
:10E65800914200D1704711F8013B00F8013FF7E7FC
:10E6680010440A44914200D1704711F8013B00F868
:10E67800013DF7E702F0DAB930B530B10A4D01448F
:10E688004FF0FF33814201D1D84330BD10F8012B40
:10E698005340082243F30004013A2C4092B284EA22
:10E6A8005303002AF6D1EDE72083B8ED0120704727
:10E6B800054B4FF400529A62044B1B6813B15B6818
:10E6C80003B11847704700BF00040048000F00203E
:10E6D800054B4FF480529A62044B1B6813B1DB68F8
:10E6E80003B11847704700BF00040048000F00201E
:10E6F8004FF0FF3070474FF0FF30704701207047F0
:10E708000120704700F0FCBD10B501F0DFFA0E21C2
:10E71800044640F61F1000F0F3FD2046012101F0E9
:10E72800BFFABDE8104000F09DBF000070B50C4E68
:10E7380001EB40030D46B3654FF6FF710023044615
:10E748001A46084601F024F896F85600002101F010
:10E75800A7FA29462046BDE8704000F05BBF00BF1D
:10E76800A40E002010B5044601F06DFB01281CD151
:10E7780001F071FB34B11248214601F0D9FF10486D
:10E7880001F09CFF0F4C104B00214FF48052A16503
:10E798009A6194F8560001F083FA63786BB16FF0D0
:10E7A8007F40BDE8104000F019BF002340F262210D
:10E7B8001A46084600F0ECFFDCE7A0688001F0E7A5
:10E7C800740E0020A40E002000040048002000F071
:10E7D80085BE00F0A5BD000008B500F08BFD04382B
:10E7E800C0B2032896BF024B0020185C08BD00BFCA
:10E7F800DA19010808B501F07EFA033008BD00F007
:10E808000DBE00F0CDBD08B501F0C4F908BD00008B
:10E8180038B50D46144601F021F8284601F056FA9D
:10E828000E21054640F61F1000F06AFD284601211A
:10E83800074D01F035FA00F015FF4FF47A71614386
:10E84800284601F075FF2846BDE8384001F036BF7C
:10E858008C0E002001F002B808B5084B002193F88F
:10E86800560001F01DFA00234FF4C0711A460846FD
:10E8780000F08EFFBDE8084000F0E8BEA40E0020BE
:10E8880010B5044601F0DFFA01281CD101F0E3FAC3
:10E8980034B11248214601F04BFF104801F00EFF39
:10E8A8000F4C104B00214FF48052A1659A6194F8E7
:10E8B800560001F0F5F963786BB16FF07F40BDE861
:10E8C800104000F041BE002340F262211A4608467B
:10E8D80000F05EFFDCE7A0688001F0E7740E00201E
:10E8E800A40E00200004004808B54FF0040000F012
:10E8F800DBFDBDE808400220F3F76CBBF7B5002349
:10E908000D4640F201211A460646084600F040FF2F
:10E918002F4B304C4FF400529A6194F85600012165
:10E9280001F0BEF92378012B40F6890012D194F842
:10E938005130062B0ED100F0F3FC00F0FB0140F63D
:10E94800890000F0DDFC2378032B29D8DFE803F0E9
:10E958000F080F3C00F0E4FC40F00401C9B2EEE7F8
:10E96800E5771D4801F094F80022294615E001F0EA
:10E978006AFA0128074625D129460DF107023046D3
:10E9880001F066FA0546A0B99DF807301248A3754C
:10E9980001F07EF89DF807102A46304600F0CAFDBF
:10E9A80061680E4801F0C4FE0C4801F087FE0020A3
:10E9B80006E00B4B3A460021022001F005FB03203C
:10E9C80003B0F0BDA575CCE70223A373A576C8E70D
:10E9D80000040048A40E0020B20E00208C0E002077
:10E9E8007C19010808B500231A461946184600F094
:10E9F800CFFEBDE8084000F0BDBD00001D4B73B55B
:10EA08001D4D186000241D486C70C5E90144AC65B3
:10EA180000F0E8FEAC8100F053FE2146204601F0EC
:10EA28009BF821460422012000F04CFF144E154D9E
:10EA38004FF6FF7123462246084600F0A9FEFFF76D
:10EA480053FF2246104B00944FF0FF31304601F03F
:10EA580089FD0E4B009422464FF0FF31284601F005
:10EA680081FD304601F0DCFD284602B0BDE870406B
:10EA780001F0D6BD000F0020A40E0020EDF2000822
:10EA88008C0E0020740E0020B9E60008D9E60008B4
:10EA98000128084805D1084BC17719700E3000F0DD
:10EAA800F7BF437D012B03D1034B81751970F5E73F
:10EAB800704700BFA40E0020000100200D4B10B5C8
:10EAC800044618735873012000F016F85CB134211D
:10EAD8004FF4E86000F014FC4421BDE8104040F217
:10EAE800417000F00DBC14214FF4E86000F008FC00
:10EAF8002421F2E7A40E002038B5114D04462870F1
:10EB080001F0AEF9012C0DD0032C17D02CB1032045
:10EB180000F0C2FE00236B7303E0204600F0BCFE49
:10EB28006C7338BD204600F0B7FE287B6B7B8342B0
:10EB3800F7D06873BDE83840FFF7C0BF0220E7E7A9
:10EB4800A40E00202DE9F04F85B006460E9DBDF8B5
:10EB580040A09DF844709DF84890019388469346DC
:10EB6800494C01F06FF90198A6B1012E4CD04046EE
:10EB780001F0ACF80E2184F8560040F61F1000F0A2
:10EB8800BFFB94F8560001F062F9169B636005B06C
:10EB9800BDE8F08F0B2384F8443084F83860E563CF
:10EBA80001F0F6F8B9F1000F41F6040363820CBFD7
:10EBB8000123F223E3754FEACA0A012387F001070C
:10EBC800237684F84500C4F840B0A673A4F810A0D2
:10EBD80026756775FFF7FAFD3046FFF78DFF04F1DC
:10EBE800380000F0E9FE04F10E0000F051FF274A5A
:10EBF8001068516802AB03C302A800F0E1FB40F2C1
:10EC0800FF1000F0B1FBB2E7214A84F83860EBB29C
:10EC1800125C84F8503070BB0B3D012D8CBF002571
:10EC28000125053B012B04D8BAF10C0F38BF4FF072
:10EC38000C0A9DF83C3084F85230164B84F8535037
:10EC48001B78E37701259DF8543084F8512084F827
:10EC58002130A573A4F81CA0A77784F82090FFF7AB
:10EC6800B5FD2846FFF748FF0B4800F0A5FE0B4806
:10EC780000F00EFF7BE7012804D1A5F10C014D42FD
:10EC88004D41CEE70025CCE7A40E00201C0C01085E
:10EC98000C1A010800010020DC0E0020B20E002032
:10ECA8002DE9F04F87B0DFF8C4A19DF864B09DF856
:10ECB8004C8002930F469DF854309DF85010BDF8D3
:10ECC800489003918AF801B0BDF844600193054665
:10ECD800144601F0B7F8BBF1000F18BF4FF0000958
:10ECE800DFF88CB10399B8F1000F08BFFF218BF84A
:10ECF800001025B1012D50D007B0BDE8F08F28468F
:10ED080000F0BAFC0B2138468AF844108AF83850CB
:10ED1800CAF83C4001F03CF8019B9BF800208AF8B7
:10ED28001620002B0CBF0122F22241F604018AF8BA
:10ED38001720F600012288F00108AAF812108AF8B4
:10ED480018208AF845008AF80E50AAF810608AF848
:10ED580014508AF81580FFF739FD2846FFF7CCFED6
:10ED68000AF1380000F028FE0AF10E0000F090FECB
:10ED780040490868496804AA03C204A800F020FBB7
:10ED880040F2FF1000F0F0FA4FF4FA5202FB09F2D9
:10ED9800B2FBF4F2CAF80820AEE7002000F06CFCE1
:10EDA80035488AF83850E1B2C05D8AF85010002F13
:10EDB8004DD10B3C012C8CBF0024012405390129BD
:10EDC80002D80C2E38BF0C26029B9BF800208AF82C
:10EDD80052308AF85340019B8AF81F2001249DF87D
:10EDE80060208AF821208AF820308AF851008AF8B1
:10EDF8000E40AAF81C608AF81E80FFF7E7FC204640
:10EE0800FFF77AFE1D4800F0D7FD1D4800F040FED0
:10EE18005FFA89F000F03CFC40F6A30000F080FAAD
:10EE280000EA040140F6A30000F06AFA9AF82120EB
:10EE3800A24240F2367013D100F072FA00F0FB01E2
:10EE480040F2367000F05CFA4FF6FF72A2E7012F2D
:10EE580004D1A4F10C035C425C41AFE70024ADE7A8
:10EE680000F05EFA40F00401C9B2E9E7A40E002000
:10EE7800000100201C0C01080C1A0108DC0E0020FF
:10EE8800B20E0020F0B58BB00D46044617461E465C
:10EE9800FFF79CFC0020FFF72FFE204600F0DEFC69
:10EEA80000240123CDE9084303234FF416722946B1
:10EEB8002046CDE90644CDE90444CDE90244CDE934
:10EEC80000532346FFF7ECFE2046FFF7D9FCFFF777
:10EED80091FCF3F77FF801F05FFB0446204601F050
:10EEE80065FBB04205D30124FFF770FC20460BB048
:10EEF800F0BD00F04FFE8742F0DA0024F4E700008E
:10EF0800F0B5BDF814409DF818709DF81CE09DF808
:10EF1800205040B1012814D001220023981801384C
:10EF2800B0FBF2F0F0BD87F00107E30003EBC70385
:10EF380018330EEB450503EBC5034FF47A714B43C9
:10EF4800ECE7501F012803F1040302D80C2C38BF4A
:10EF58000C24D1B9A2F10B0CBCF1010F8CBF4FF0FE
:10EF6800000C4FF0010C2801002F00EBCE000CBF65
:10EF780014250025A0EB8200062A4FEA82062844C1
:10EF8800A2F102070DD8354610E0012906D1A2F1F9
:10EF98000C00D0F1000C4CEB000CE4E74FF0000C37
:10EFA800E1E70830BCF1000FEDD0BD000028ACBF90
:10EFB8002E182E1C701E90FBF5F003FB0044094B25
:10EFC800062A5A5C8CBF0C340E340A2A09D8A300CE
:10EFD80001334FF47A71BB404B43034951F8222067
:10EFE8009CE7FFDE0C1A0108E019010808B5094B77
:10EFF800012193F8560000F053FE4FF4D7602D21FD
:10F0080000F07EF900F033FBBDE80840024800F04C
:10F018007BBA00BFA40E0020FFFF0F0073B5A44CFD
:10F02800B4F854300025202B8DF80350019500F0DA
:10F038001B8114D8082B0DD87BB1013B072B0CD8AA
:10F04800DFE813F042005B000B00CD000B000B0063
:10F058000B00FD00102B00F0008102B070BDB3F56D
:10F06800807F00F0988011D8402B00F01081802B11
:10F07800F3D1284600F032FA8E4B1B68002BECD0F7
:10F088009B69002BE9D028469847E6E7B3F5007F4F
:10F09800E3D1894B01222946022000F095FF00F0B8
:10F0A80029F9042840F08580844B85484FF40052A4
:10F0B8009A6201F0B5FA284600F010FA7D4B1B68F9
:10F0C800002BCAD05B6814E07C4B7D484FF400529B
:10F0D8009A6201F0A5FA002000F000FA00F0B5FEEF
:10F0E800012801D100F0BAFE724B1B68002BB4D086
:10F0F8001B68002BB1D09847AFE7704B71484FF4AD
:10F1080080529A6201F08CFA657895B9284600F029
:10F11800E5F9294640F6021000F0F2F840F64410EE
:10F1280000F0FEF840F00201C9B240F6441000F0C9
:10F13800E7F8FF220DF1030163485E4D00F05AFD28
:10F14800624800F071FD2B68002B86D09E68002E67
:10F1580083D094F82430012B08D194F9313094F9F4
:10F1680030209DF803105848B04776E7E06B01A9B6
:10F1780000F022FE019B9DF8031053484FF47A7269
:10F1880003F5FA7393FBF2F32A685BB2956894F976
:10F198002920A84761E7284600F0A0F9454B1B68DD
:10F1A800002B3FF45AAF9B69002B3FF456AF012068
:10F1B8006AE700F09FF805287FF44FAF3F4B4148BE
:10F1C8004FF480529A6201F02BFA284600F086F933
:10F1D800384B1B68002B3FF440AFDB6889E7002100
:10F1E8003B4B0122022000F0EFFEA16D00293FF405
:10F1F80034AFC1F3074140F6031000F081F894F8EA
:10F20800591040F6041000F07BF894F8581040F6B6
:10F21800051000F075F840F6021000F081F840F093
:10F228000101C9B240F6021000F06AF8002340F26A
:10F2380062211A460846A36500F0AAFA0DE7254B95
:10F2480001220021022000F0BFFE00F0FCFD012891
:10F258007FF403AF00F003FEFFE61F4B01220021FD
:10F26800022000F0B1FEF8E6164801F0D9F96078FE
:10F2780008B900F033F90F4B1B68002B3FF4EDAED3
:10F28800DB68002B3FF4E9AE9847144BE6E7144BD4
:10F2980001222946022000F097FE607808B900F0A4
:10F2A8001DF9044B1B68002B3FF4D7AE1B6920E700
:10F2B800A40E0020000F0020911901080004004846
:10F2C8008C0E0020740E0020040F0020C80E0020B1
:10F2D800A5190108AE190108B8190108C1190108D2
:10F2E800CA190108024BA3F85400FFF797BE00BFE4
:10F2F800A40E0020014B1878704700BF12100020A0
:10F3080007B501238DF807100DF1070201460348E0
:10F31800F6F7BEF803B05DF804FB00BFE00100207B
:10F3280007B5012301460DF107020448F6F7E9F88D
:10F338009DF8070003B05DF804FB00BFE001002062
:10F3480010B50446F3F75EFD01280CD140F62310F2
:10F35800FFF7E6FF00F0F901214340F62310BDE86E
:10F368001040FFF7CDBF10BD10B50C4B1B780446FD
:10F378009BB94FF4D760FFF7D3FFC4F3002100F027
:10F38800FE0001434FF4D760FFF7BAFFE1B240F245
:10F39800B960BDE81040FFF7B3BF10BD11100020E1
:10F3A80010B51346EFF3108472B60A4601460348B7
:10F3B800F6F76EF884F3108810BD00BFE001002056
:10F3C80008B5014608224FF4D860FFF7E9FF00208E
:10F3D80008BD000007B5074B1B7840BAADF804001C
:10F3E8002BB9022201A940F2BC60FFF7D9FF03B094
:10F3F8005DF804FB1110002007B5074B1B7840BAD5
:10F40800ADF804002BB9022201A940F2BE60FFF753
:10F41800C7FF03B05DF804FB1110002010B51346B8
:10F42800EFF3108472B60A4601460348F6F769F806
:10F4380084F3108810BD00BFE001002010B513460A
:10F44800EFF3108472B60A4601460348F6F74BF903
:10F4580084F3108810BD00BFE00100200A46014671
:10F468000020FFF7EBBF000010B51346EFF3108440
:10F4780072B60A4601460348F6F768F984F310881D
:10F4880010BD00BFE001002010B51346EFF3108453
:10F4980072B60A4601460348F6F76EF884F31088F8
:10F4A80010BD00BFE001002013B504460020F3F7AB
:10F4B800A3FC0220FFF744FF04F0070401220DF12A
:10F4C800070184208DF80740FFF7DEFF024B00227A
:10F4D8001A7002B010BD00BF1210002007B501223B
:10F4E8008DF807000DF107018020FFF7CDFF9DF88B
:10F4F8000730002B034B14BF022201221A7003B0FD
:10F508005DF804FB1210002007B5094B8DF80600C2
:10F5180004221A70030C8DF804300322030A01A98F
:10F5280083208DF80530FFF7AFFF03B05DF804FBCB
:10F538001210002010B51446FFF790FF2046BDE8D2
:10F548001040FFF7E1BF000007B5094B8DF8060032
:10F5580005221A70030C8DF804300322030A01A94E
:10F5680082208DF80530FFF78FFF03B05DF804FBAC
:10F578001210002073B5002640F6E2000196FFF74E
:10F58800CFFE00F0FE01054640F6E200FFF7B8FEA8
:10F5980040F6E500FFF7C4FE00F07F01044640F6A0
:10F5A800E500FFF7ADFE6FF07F40FFF7CDFF0422C7
:10F5B8000DEB020140F61900FFF730FF3046FFF768
:10F5C8008DFF294640F6E200FFF79AFE214640F6F5
:10F5D800E500FFF795FE019802B070BD13B50C4B1E
:10F5E80004460522972140F6AC001A70FFF788FE02
:10F5F800230C8DF804300322230A01A982208DF8F8
:10F6080005308DF80640FFF73FFF02B010BD00BF80
:10F618001210002007B5030C8DF80030030A8DF88E
:10F6280001300B0C49BA8DF80200ADF8041006221F
:10F63800694694208DF80330FFF726FF024B062217
:10F648001A7003B05DF804FB12100020002208B500
:10F658001146C520FFF718FF014B07221A7008BD95
:10F668001210002000221146D120FFF70DBF002202
:10F678001146D220FFF708BF07B501228DF8070011
:10F688000DF107019F20FFF7FFFE03B05DF804FBB3
:10F6980007B501228DF807000DF10701A020FFF73B
:10F6A800F3FE9DF807103F2907D901F0F801013151
:10F6B800C9B240F20670FFF723FE03B05DF804FB01
:10F6C80007B5F3F79FFB431E584258418DF80700D2
:10F6D80001220DF107019620FFF7D6FE03B05DF871
:10F6E80004FB07B500F07F008DF8070001220DF13B
:10F6F80007018920FFF7C8FE03B05DF804FB00008E
:10F70800154B984207B51BD8144B98421BD8144B7D
:10F7180098421BD8134B98421BD8134B98428BBF67
:10F728006B2229226F232B238DF8042001A90222A2
:10F7380098208DF80530FFF7A7FE03B05DF804FBAD
:10F74800E122E923F0E7D722DB23EDE7C122C52335
:10F75800EAE775228123E7E700E9A43580F8A932B2
:10F768008044E52D000B6B1B40FC541907B58DF840
:10F77800062004228DF804008DF8051095200DEB65
:10F7880002018DF80730FFF77FFE03B05DF804FB38
:10F7980007B552BAADF8042040BA082249BAADF804
:10F7A8000000ADF802105BBA69461046ADF80630A5
:10F7B800FFF76AFE03B05DF804FB07B50B0C0422E3
:10F7C80000F0070049BA8DF80400ADF8061097203C
:10F7D8000DEB02018DF80530FFF756FE03B05DF81A
:10F7E80004FB000010B508B1194B1860F2F7EEFAE7
:10F7F8000220FFF7A5FD0024164B20461C70FFF7DA
:10F808006DFEF3F7FDFA012816D14021FFF7D5FF69
:10F8180040F611102146FFF773FD4FF07F00FFF708
:10F8280060FF0E2140F61F10FFF76AFDF3F7E2FABA
:10F83800094B01221A7010BD202140F61110FFF764
:10F848005FFD202140F61210FFF75AFDE9E700BFDF
:10F8580004100020081000201210002037B50C4DAD
:10F868002B7804461BB9FFF74BFF01232B700023AD
:10F87800084A6006E109F1F7A5FB042200BA0190E5
:10F888000DEB02018620FFF7FFFD03B030BD00BF7E
:10F89800081000200048E80107B5094B8DF807005B
:10F8A8000146187018B940F2AC60FFF729FD012233
:10F8B8000DF107018A20FFF7E7FD03B05DF804FBAF
:10F8C80011100020012873B50C46164637D10020C8
:10F8D800F3F79AFAA042B8BF44B20E2805461AD1E7
:10F8E80001231A4600210420FFF740FF6FF01003A0
:10F8F8009C42B8BF1C46182140F6E700FFF700FD00
:10F90800022201A98E208DF804408DF80560FFF7CA
:10F91800BBFD02B070BD01230A28E4B21A464FF0BD
:10F92800000105D11846FFF721FF033464B2DDE773
:10F938000720C5F10E05FFF719FF2C44F6E740F63E
:10F94800D800FFF7EDFC40F01E01C9B240F6D80020
:10F95800FFF7D6FC0120F3F757FAA042B8BF44B22C
:10F96800142805464FF001034FF000020CD1052181
:10F978000320FFF7FBFE023464B26FF008039C42D9
:10F98800B8BF1C463821B7E7112805D1032102204A
:10F99800FFF7ECFE0534EFE70E2804D102210846F4
:10F9A800FFF7E4FEE9E7C5F1160507210420254421
:10F9B800FFF7DCFE6CB2E0E713B5314A0446516844
:10F9C80010686B4603C32F4B20781B78834201D005
:10F9D800FFF762FF2378032B27D8DFE803F002390B
:10F9E800283C6268284BB3FBF2F31A0CA1688DF827
:10F9F80000208DF802301A0A237B8DF80330637BD0
:10FA08008DF801208DF80430204A00234806C909E2
:10FA1800F1F7D8FA030C40BA8DF80530ADF80600B6
:10FA2800082269468B20FFF72FFD02B010BD22691E
:10FA3800154BB3FBF2F31A0C8DF800208DF8023049
:10FA48001A0A237D8DF801208DF803300422E8E797
:10FA5800A3690093FAE762680B4BB3FBF2F31A0C45
:10FA68008DF800208DF802301A0A237B8DF80330B8
:10FA7800637B8DF801208DF804300522D1E700BFA3
:10FA8800240C0108111000200000093D0048E8017D
:10FA98001FB52E4A0446D1689068127C01AB03C397
:10FAA8001A702B4B20781B78834201D0FFF7F4FEA5
:10FAB8002378032B26D8DFE803F002383302637A71
:10FAC800F12B21D14FF6FF70FFF784FC48F20500B7
:10FAD800FFF792FC02236288A188ADF8061052BA9B
:10FAE800E188ADF804208DF80B30227AA37A8DF8DE
:10FAF8000A20ADF808108DF80C30092201A98C20D5
:10FB0800FFF7C2FC04B010BDF22BE4D141F60F5050
:10FB1800FFF760FC41F22100FFF76EFC0623DAE7ED
:10FB2800237B8DF804300122E8E7E389094A5BBAB0
:10FB3800ADF80430237C13708DF80630637C8DF8A3
:10FB48000730638AADF808300622D7E7240C01088D
:10FB5800111000201010002007B502228DF80400B3
:10FB68008DF805108F2001A9FFF78EFC03B05DF812
:10FB780004FB000010B51346EFF3108472B60A4672
:10FB880001460348F5F730FD84F3108810BD00BF27
:10FB9800E001002007B5012201A91520FFF7EAFFBF
:10FBA8009DF804004042401003B05DF804FB0000DB
:10FBB80037B505460C46022201A91320FFF7DAFFE4
:10FBC8000A4B1B78012B0DD1094B1B78012B09D14E
:10FBD80040F20270FFF7A4FB9DF8053028702370EF
:10FBE80003B030BD9DF80400F6E700BF11100020F7
:10FBF80010100020F7B50D46064600240DF1070148
:10FC0800284617468DF80740FFF7D2FF2A78BA42F0
:10FC180007D89DF807003146FFF726FC204603B0B9
:10FC2800F0BD0120FBE7000013B50322044601A93B
:10FC38001420FFF79FFF184B1A7822704AB1012A47
:10FC480017D014220021204600F0CEFA0F2323708B
:10FC58000DE09DF8043023719DF80530A2605B42E9
:10FC68005B10A3719DF806305B425B10637102B0B4
:10FC780010BD9DF804305B425B1023739DF905307D
:10FC880002339B1063739DF806305B425B10A373CD
:10FC9800024B1B682361EAE7111000200C100020BA
:10FCA800012908B5034608460ED1012B07D10420C7
:10FCB800FFF746FB0220BDE80840F3F79DB8022B8A
:10FCC80014BF08460320F6E70120F4E738B50446D8
:10FCD800F3F794F850B102280CBF022501252846F5
:10FCE80002222146FFF7EEFD284638BD102CB4BF8E
:10FCF80001250225F3E7012070470000014B012090
:10FD08001B68184704100020014B02201B68184785
:10FD180004100020014B40201B68184704100020E5
:10FD280011B1012904D07047044B1B688020184783
:10FD3800024B4FF480701B68F9E700BF04100020E5
:10FD4800024B4FF400701B68184700BF04100020D6
:10FD5800014B20201B68184704100020014B042089
:10FD68001B68184704100020014B08201B6818471F
:10FD780004100020014B10201B68184704100020B5
:10FD8800024B4FF480401B68184700BF0410002046
:10FD980010B568B1074A002352F83340844202EB99
:10FDA800C30101D9087910BD0133162BF4D1FEE740
:10FDB8001F20F8E79C1A010873B51D4B01930446F0
:10FDC80040F607000D46FFF7ABFAC0F3C10308334E
:10FDD8006B4413F8042C00F00703013302FA03F311
:10FDE800144AB2FBF3F2B2FBF4F007281ED8400025
:10FDF800042834BF042302234FF4D66002FB03F423
:10FE0800FFF78EFA060240F2B160FFF789FA06F4AE
:10FE180070663043030544BF6FEA00506FEA105024
:10FE280063094343DB112B6002B070BD0123E3E794
:10FE380004080A0C0048E8014FF0FF3070474FF003
:10FE4800FF307047704700207047002070477047A8
:10FE58004FF0FF3070474FF0FF30704770477047E2
:10FE68007047000070B5EFF3108672B6144B5C8AC9
:10FE78001A8A944213D1C4F5806292B2904206D392
:10FE8800844218D901229A7000221C805A825A8A08
:10FE98000A800244C2F309025A8200200DE006D902
:10FEA800C4F58065ADB28542F1D88242E9E7121BFC
:10FEB80092B28242EBD84FF0FF3086F3108870BDC3
:10FEC80014160020EFF3108172B6034AD38A013367
:10FED800D38281F31088704714160020EFF3108145
:10FEE80072B6034AD38A013BD38281F310887047E4
:10FEF8001416002010B508481822002100F074F9E3
:10FF080006484FF48062002100F06EF9044B054862
:10FF18001B68BDE810401847141600201312002073
:10FF2800F40C010899000108014B5860704700BFA4
:10FF380014160020014B1872704700BF14160020D9
:10FF480073B5EFF3108572B61C4CE08A00282FD1E8
:10FF5800FFF7B8FF218A628A914227D0A378012B44
:10FF680012D1238820805B1A9BB20221A382A17040
:10FF780063B9A3702382238A9A428BBFD21AC3F52E
:10FF88008063A282A38201E0002BF4D0268A0C4B66
:10FF98001E4485F31088F2F70BF80A4BA18ADB6838
:10FFA8000193304602B0BDE870401847FFF796FF4E
:10FFB80085F31088002002B070BD00BF1416002021
:10FFC80013120020F40C010808B4F0B586B0002321
:10FFD800ADF800302B4B0B9C1D7A85424CD3D8686A
:10FFE80081434CD15B681BB112B1694602A898479E
:08FFF8000CAB22464FF400712E
:020000040801F1
:100000002348019300F0F4FBFFF760FFBDF80030D8
:1000100018440DF1020180B2FFF728FF01302AD009
:100020000023BDF80020BDF802601A480DF1080C4D
:100030001F4699B216FA83F58A42ADB215D817B1A8
:100040003244ADF80220BDF80250019B22464FF425
:100050000071284400F0CCFBFFF744FFFFF774FF6A
:1000600006B0BDE8F04001B070471CF8011B4155D7
:1000700001330127DDE7FFF735FF6FF00200EFE7FF
:100080006FF00400ECE76FF00500E9E714160020BC
:10009000131000201312002013B5EFF3108472B672
:1000A000204B9A78588A022A1DBF1A8A998A5218B8
:1000B000002214BFC2F309029A7090421A8228D01B
:1000C000D98A012925D19978012913D119888A1A49
:1000D000022192B2997000219A82198062B99A70B5
:1000E0001A821A8A90428BBF801AC2F58062988267
:1000F0009A8201E00029F4D0188A0B4A104484F354
:1001000010880A4A998AD368019302B0BDE810406A
:10011000184784F31088F1F753FF02B0BDE8104090
:10012000FFF7E0BE1416002013120020F40C0108A3
:10013000024A00231360024A136070473016002001
:100140002C16002010B5EFF3108472B641B10129CE
:1001500003D1064A13680343136084F3108810BD6B
:10016000024A136823EA0003F6E700BF30160020B6
:1001700010B5EFF3108472B641B1012903D1064ADC
:1001800013680343136084F3108810BD024A136898
:1001900023EA0003F6E700BF2C16002038B5EFF382
:1001A000108572B60A4B0B4C1B6833B12368984715
:1001B0006368984785F3108838BD074B1B681BB1EF
:1001C000A3689847E368F4E7236998476369F0E711
:1001D00030160020380C01082C16002001380A4483
:1001E000914200D1704711F8013B00F8013FF7E759
:1001F00000F020BC10B5EFF3108472B6064A136805
:1002000003431360054A52F83130034342F831305A
:1002100084F3108810BD00BF58160020341600204B
:1002200070477047B0F5803F3ABF000410230023A9
:10023000B0F1807F3EBF08330002DBB2B0F1805FD7
:1002400038BF00014FEA1070054A38BF0433125C12
:1002500038BFDBB2C3F11F03981AC0B2704700BFAA
:100260004C1B01082DE9F84F384D394ED5F8008068
:10027000DFF8E0B0DFF8E0A0DFF8E090D6F800C0EB
:10028000374FDBF80010374CDAF80020D9F800308F
:1002900008EA00002860286800EA020E1EEA0C0F37
:1002A00001D019421ED04FF0FF333B60FFF7B8FF7B
:1002B000EFF3108472B63368DBF80020DAF8001030
:1002C0000B4029680B4205D1D9F80030134201D107
:1002D000F1F700FE84F31088FFF7A3FFC5F8008054
:1002E000BDE8F88F236823680340134062681A4210
:1002F00004BF4FF0FF32626060681840FFF792FF62
:1003000062683860012303FA00F022EA00026260AA
:10031000EFF3108172B63A689340326822EA030222
:100320003260226822EA0303236081F310880E4AB8
:100330003B6852F823309847D6F800C0DBF800102D
:10034000DAF80020D9F80030A5E700BF040100204A
:1003500058160020541600200801002050160020D6
:100360004C160020341600203C16002010B5114613
:10037000EFF3108472B6FFF755FF034B43F82010DC
:1003800084F3108810BD00BF3C16002082B082B0FC
:100390000DF1080C0CE90600BDF8042003930B4492
:1003A000BDF810100A4491B212B2B2F57A7FA2BF22
:1003B000A1F57A72013312B20360828002B002B0FA
:1003C000704782B082B00DF1080C0CE90600BDF850
:1003D00004200393CB1ABDF81010521A91B212B236
:1003E000002ABEBF01F57A7203F1FF3312B2036037
:1003F000828002B002B0704730B585B0114D6B46B7
:1004000083E8030000230293ADF80C3003A82B69A6
:100410009847009BBDF804400290181ABDF80C30B4
:10042000E41AA3B224B2002CBEBF03F57A731CB247
:1004300000F1FF302B689847AB682046984705B01D
:1004400030BD00BFB40C010873B5114E0023054642
:100450000093ADF8043001A833699847F368009021
:100460009847736804469847009B1844BDF80430C9
:1004700023449AB21BB2B3F57A7FA2BF0130A2F532
:100480007A731BB228602846AB8002B070BD00BFF3
:10049000B40C010837B500230093ADF80430074BC6
:1004A00004461B6901A898476D46009095E8030033
:1004B00084E80300204603B030BD00BFB40C01083F
:1004C00037B50F4D02AB03E90300EB6898476B6843
:1004D00004469847BDF80430009A1B1B99B21BB222
:1004E000002BA2EB0002BEBF01F57A7102F1FF32D0
:1004F0000BB24FF47A7000FB023003B030BD00BF86
:10050000B40C01082DE9F0414FF47A75B1FBF5F513
:10051000C5EB4513DFF83C8005EB8303A1EBC30378
:100520009CB2D8F80C3006469847D8F804300746F5
:100530009847E31999B21BB2B3F57A7F2844A2BF5A
:10054000A1F57A7301301BB23060B3803046BDE84C
:10055000F08100BFB40C0108024B00221A60024B6C
:100560001B6818475C160020C80C0108F8B5044643
:10057000174608461E467CB173B1084B00255B6ADE
:1005800025609847069B60602581A572E66023611F
:10059000E77265612846F8BD0120FCE7C80C010838
:1005A00010B5034CE3699847A36ABDE810401847AB
:1005B000C80C010870B5064DEB69064698476B6A92
:1005C000044630469847AB6A201ABDE87040184789
:1005D000C80C0108054B1B680BB9184670478342CD
:1005E00001D05B69F8E70120704700BF5C1600206E
:1005F0002DE9F3410B4E336A044698470123B7694E
:100600002372D4F800800546B8472844804502D2BA
:10061000B84728442060B3682068019302B0BDE861
:10062000F0411847C80C010870B520B3EFF31086ED
:1006300072B6124D2B680122827253B100224272AF
:1006400098425C690ED102723CB120462C60FFF7E3
:10065000CFFF86F31088002070BD094BDB689847F8
:100660002C60F6E71A465B69002BF2D09842F9D16C
:1006700043695361EDE70120EEE700BF5C160020FF
:10068000C80C0108084B10B51A685369516911B9B3
:100690005061416110BD046819688C4202D91A4644
:1006A0005B69F3E71946F3E75C160020044A136818
:1006B0000BB10021197243611060FFF799BF00BFB1
:1006C0005C1600202DE9F041044600282DD0FFF7EC
:1006D00081FF50BB657A45BBEFF3108872B6144EAC
:1006E0006768336A984787422CBF27602060114FA4
:1006F000A5724FF4807323813B684BB933699847E7
:100700002046FFF7D3FF88F310882846BDE8F08124
:10071000B3699847236818443B6820601B68984277
:100720002046EED3FFF7AEFFEDE70125EDE700BF72
:10073000C80C01085C16002010B5044608467CB1C0
:10074000084B5B6A984760602046FFF743FF40B163
:100750002046FFF769FF2046BDE81040FFF7B2BF13
:10076000012010BDC80C01082DE9F041EFF31087FE
:1007700072B61D4E1D4D73699847336904469847FC
:100780002B684BB94FF000082B688BB9286828BB41
:1007900087F31088BDE8F081011B241A1A688A4289
:1007A0008CBF121900221A605B69002BF6D1E9E7B1
:1007B0001C681CB1B36998478442E7D22C6863690E
:1007C0002B60A4F80880D4E9033098476389B3F517
:1007D000807FD9D12046FFF775FFD5E7037A002B3C
:1007E000D6D1FFF705FFD3E7C80C01085C1600203F
:1007F0002DE9F04F002997B081461E4640F3118144
:1008000004464F1E1378A4EB090023B9002323707C
:1008100017B0BDE8F08FB842F8DA252B05D004F800
:10082000013B904608F10102ECE792F801E0AEF1DD
:10083000300102F10108AEF130034A424A41092B6E
:100840002BD8414600250A20884611F8013BA3F128
:10085000300CBCF1090F1BD998F80030692B00F05F
:100860009E801DD8632B29D0642B00F09880582BD4
:100870005AD0252B1AD198F80030002B00F0938025
:1008800004F8013BA4EB0903BB4280F28A80C9E76C
:1008900000FB0533A3F13005D6E74FF0FF35DBE76A
:1008A000752B7ED0782B41D0732B1CD0252304F8D8
:1008B000013BA4EB0903BB4273DADCE7002D05F131
:1008C000FF3AD8BF4FF0000A52462046202100F0E0
:1008D000B1F8A244002D56F8043B8AF80030D8BF86
:1008E00001252C449EE7504B56F804BBBBF1000F8A
:1008F00008BF9B465846EFF73FFC2A1A8542B8BF0F
:100900000022824620212046019200F093F8019AAD
:1009100000232244534502DB02EB0A0482E71BF862
:100920000310D1540133F5E742F040021021DFF803
:10093000FCB0DFF8FCA056F804CB12F0400F18BF53
:10094000DA46BEF1300FCDF808A0A4EB09030CBFC6
:100950004FF0300A4FF0200A9207A7EB03036046DE
:10096000CDF80CA022D5002820DA4042013D4FF0FE
:100970002D0C05AA019200228246B0FBF1F001FB8A
:1009800010AB029810F80BB0019800F801BB51456C
:10099000019002F10102BAFBF1F0EDD910E042F052
:1009A00002020A21C3E708F1FF386BE7BCF1000F30
:1009B00002D04FF0000CDCE730228DF81420012229
:1009C000BEF1300FA5EB020504D02020002D05F16B
:1009D000FF350ADCBCF1000F05D02D21013B04F8E6
:1009E000011B3FF41FAF25440AE0013B04F8010B53
:1009F000ECD117E7039904F8011B013B3FF412AF58
:100A0000291B0029F6DC05A9114423442244A242F3
:100A10003FF408AF11F8010D04F8010B9C42F6D128
:100A200000E70020F4E600BF5C1B0108881B0108FA
:100A3000631B010802440346934200D1704703F848
:100A4000011BF9E770B50D4D0D4C641BA410002679
:100A5000A64209D10B4D0C4C00F09AF8641BA4106F
:100A60000026A64205D170BD55F8043B98470136D3
:100A7000EEE755F8043B98470136F2E7B81B01084A
:100A8000B81B0108B81B0108BC1B010800000000CE
:100A90002DE9F041C1F30A57A7F2FF36132E0246A3
:100AA0000B460C460546804635DC002E17DA34A38B
:100AB000D3E90023EFF76EFB00220023EFF7B0FF2E
:100AC00050B1002C57DA24F000442C430025AC42EE
:100AD0002D4C08BF4FF0004423462A4624E02B4FFC
:100AE000374101EA070C5CEA000C1DD024A3D3E9CE
:100AF0000023EFF74FFB00220023EFF791FF0028C0
:100B0000EAD0002CBEBF4FF480133341E41824EA2E
:100B100007040025E0E7332E0ADDB6F5806F03D128
:100B2000EFF738FB02460B4610461946BDE8F08148
:100B3000A7F213474FF0FF3C2CFA07F70742F3D018
:100B40000FA3D3E90023EFF725FB00220023EFF7E3
:100B500067FF0028C0D0002C0ADA142E01D101341E
:100B600006E0C6F134060123B3401D444545F6D3E3
:100B700025EA0705B0E700252C46ADE7AFF3008076
:100B80009C7500883CE4377E0000F0BFFFFF0F003B
:100B9000F8B500BFF8BC08BC9E467047F8B500BF6A
:080BA000F8BC08BC9E4670473A
:100BA800000000000100000002000000000000003A
:100BB8008813000010270000204E00003075000048
:100BC800409C000050C3000060EA0000C0D401004F
:100BD80080A903000053070000EA06370000000060
:100BE8005000000040F709370000000050000000E6
:100BF800A027BE330000000050010000E034C133DC
:100C080000000000500100002042C4330000000032
:100C180050010000C194C100000000000000000065
:100C280000000000000000000000000000000000BC
:100C38008B1A0008791A00085D1A00087D1A000846
:100C4800591A00089D1A00080D0A2023232323237C
:100C5800202047726F737320576569676874203D59
:100C680025642020203C3C3C3C3C3C200D0A000DE7
:100C78000A20232323232320204E657420576569E7
:100C8800676874203D25642020200D0A004E657495
:100C980020576569676874203D20256420206720F7
:100CA8000D0A00256473253033643A005D2100087D
:100CB800FD2100086D21000809220008CD21000847
:100CC80015220008000000007D21000835210008D9
:100CD80001210008B9200008112100082521000879
:100CE800C5200008C9200008DD2000088D24000860
:100CF800B5240008392400082524000853776974AE
:100D0800636820746F20436C6173732025632064CB
:100D18006F6E650D0A00414243000D0A2323232309
:100D28002323203D204A4F494E4544203D20004181
:100D38004250203D3D3D3D3D3D3D3D3D3D3D3D3DE0
:100D48003D3D3D3D3D3D3D3D3D0D0A004F5441413A
:100D5800203D3D3D3D3D3D3D3D3D3D3D3D3D3D3DD8
:100D68003D3D3D3D3D3D0D0A000D0A232323232330
:100D780023203D204A4F494E204641494C45440DC9
:100D88000A0023232323232320552F4C2046524196
:100D98004D453A4A4F494E207C2044523A2564201A
:100DA8007C205057523A25640D0A004C6D48616EFC
:100DB800646C65722053746F70206F6E20676F6962
:100DC8006E67202E2E2E0D0A004C6D48616E646CE5
:100DD80065722053746F707065640D0A004C6D481D
:100DE800616E646C65722073776974636820746FD0
:100DF80020414250206D6F64650D0A005765696790
:100E08006874205363616C65203A2025640D0A00DC
:100E1800564444413A2025640D0A0074656D703AC1
:100E28002025640D0A0053454E442052455155452E
:100E380053540D0A004E65787420547820696E204A
:100E4800203A207E2564207365636F6E64287329B9
:100E58000D0A000D0A23232323232320424541435F
:100E68004F4E204C4F53540D0A000D0A23232323C1
:100E7800232320424541434F4E205245434549567E
:100E88004544207C2044523A2564207C2052535308
:100E9800493A2564207C20534E523A2564207C2010
:100EA80046513A2564207C2054494D453A25642012
:100EB8007C20444553433A2564207C20494E464FC4
:100EC8003A303258253032582530325820253032C1
:100ED8005825303258253032580D0A000D0A232380
:100EE8002323232320424541434F4E204E4F542075
:100EF80052454345495645440D0A004E564D204437
:100F08004154412053544F5245440D0A004E564D0A
:100F1800204441544120524553544F5245440D0AF0
:100F2800004E41434B000D0A232323232323203D56
:100F38003D3D3D3D3D3D3D3D3D204D4350532D43C1
:100F48006F6E6669726D203D3D3D3D3D3D3D3D3DC9
:100F58003D3D3D3D0D0A0023232323232320552F08
:100F68004C204652414D453A25303464207C20506F
:100F78004F52543A2564207C2044523A2564207C00
:100F8800205057523A256400207C204D5347205466
:100F98005950453A00434F4E4649524D4544205B0F
:100FA80025735D0D0A00554E434F4E4649524D4537
:100FB800440D0A004C4544204F46460D0A004C4556
:100FC80044204F4E0D0A0023232323232320442F9C
:100FD8004C204652414D453A25303464207C2050FF
:100FE8004F52543A2564207C2044523A2564207C90
:100FF80020534C4F543A2573207C20525353493A7E
:101008002564207C20534E523A25640D0A004E5622
:101018004D204441544120555020544F20444154C0
:10102800450D0A004E564D20444154412053544F1B
:101038005245204641494C45440D0A004150504C08
:1010480049434154494F4E5F56455253494F4E3AD2
:10105800205625582E25582E25580D0A004D575F25
:101068004C4F524157414E5F56455253494F4E3AA5
:1010780020205625582E25582E25580D0A004D5744
:101088005F524144494F5F56455253494F4E3A20AB
:101098002020205625582E25582E25580D0A004C5C
:1010A800325F535045435F56455253494F4E3A209D
:1010B800202020205625582E25582E25580D0A0068
:1010C80052505F535045435F56455253494F4E3A2D
:1010D80020202020205625582D25582E25582E25ED
:1010E800580D0A0031003200435F4D4300505F4DF8
:1010F80043000000EC100108EE100108200D010863
:10110800F0100108A9130108F5100108A0860100D4
:10111800400D0300801A060000350C0040420F0005
:1011280080841E0000093D0000127A000024F400AB
:1011380000366E010048E801006CDC020000000087
:101148000000000000000000000000000000000097
:101158000000000000000000000000000100000086
:10116800020000000300000004000000010000006D
:10117800030000000500000001000000010000005D
:10118800060000000A000000200000000200000025
:1011980004000000080000001000000040000000EB
:1011A80080000000000100000002000001000200B1
:1011B8000400060008000A000C001000200040008F
:1011C8008000000108040204080101010101010373
:1011D800070100006572726F723A20526567696F85
:1011E8006E206973206E6F7420646566696E65642D
:1011F80020696E20746865204D573A207365742005
:101208006C6F726177616E5F636F6E662E682061C6
:1012180063636F7264696E676C790D0A004D4143B0
:1012280020727854696D654F75740D0A004D4143FD
:1012380020747854696D654F75740D0A004D4143EB
:10124800207278446F6E650D0A004D414320747812
:10125800446F6E650D0A00080A0C0D0E1012141565
:10126800181A1B1D1E21240305020501060202058A
:101278000000060000010504040202020202020244
:101288000202020202020202030202020202020334
:101298000403020202020204050403020202020518
:1012A80006050403020202060706050403020207F4
:1012B80007070605040302070700000000000001F5
:1012C8000201000000000002030201000000000308
:1012D80004030201000000040504030201000005E4
:1012E80006050403020100060706050403020107B8
:1012F80007070605040302070700000B357DF2F215
:10130800F233337373DEDEDEDE33337373F2F2F2FD
:10131800F200000048E8010048E8010048E8010040
:1013280048E8010048E8010048E8010090D00300BF
:10133800000000000C0B0A090807073252585F2505
:1013480073206F6E206672657120256420487A20AC
:1013580061742044522025640D0A005258206F6E93
:10136800206672657120256420487A2061742044C3
:10137800522025640D0A005458206F6E206672654D
:101388007120256420487A20617420445220256405
:101398000D0A004D756C74695F43004D756C746976
:1013A8005F500000EC100108EE100108200D010844
:1013B8009B130108A9130108A313010833333373DE
:1013C800DEDEDEDE33333373F2F2F2F248E8010098
:1013D80048E8010048E8010048E8010048E8010041
:1013E80048E8010090D00300000000000C0B0A0937
:1013F800080707320B357DF2F2000000216DDEDEB2
:10140800DEDE00000B357DF2F20000003581F2F2DD
:10141800F2F200000A0908080B0A09080C0B0A096D
:101428000D0C0B0A0D0D0C0B48E8010048E80100F3
:1014380048E8010048E8010020A10700000000007A
:10144800000000000000000020A1070020A1070004
:1014580020A1070020A1070020A1070020A1070064
:1014680000000000000000000A090807080000004A
:101478000C0B0A0908070000A584998D0DBDB1540D
:101488005003A97D1962E69A459D408715EBC90B63
:10149800EC67FDEABFF7965BC21CAE6A5A41024F81
:1014A8005CF434089373533F0C52655E28A10FB562
:1014B80009369B3D2669CD9F1B9E742E2DB2EEFBEF
:1014C800F64D61CE7B3E7197F568002C601FC8ED24
:1014D800BE46D94BDED4E84A6B2AE516C5D75594E3
:1014E800CF100681F044BAE3F3FEC08AADBC4804CD
:1014F800DFC17563301A0E6D4C14352FE1A2CC395B
:1015080057F28247ACE72B95A098D17F667EAB83D4
:10151800CA29D33C79E21D763B564E1EDB0A6CE4A1
:101528005D6EEFA6A8A4378B324359B78C64D2E01E
:10153800B4FA0725AF8EE918D5886F7224F1C75120
:10154800237C9C21DDDC86859042C4AAD805011243
:10155800A35FF9D0915827B93813B333BB7089A763
:10156800B622922049FF787A8FF88017DA31C6B808
:10157800C3B07711CBFCD63AC6F8EEF6FFD6DE91AB
:101588006002CE56E7B54DEC8F1F89FAEFB28EFB9D
:1015980041B35F452353E49B75E13D4C6C7EF58375
:1015A8006851D1F9E2AB622A0895469D30370A2F77
:1015B8000E241BDFCD4E7FEA121D583436DCB45B97
:1015C800A476B77D52DD5E13A6B900C140E379B6B3
:1015D800D48D67729498B085BBC54FED869A661115
:1015E8008AE904FEA078254BA25D80053F2170F1B1
:1015F8006377AF4220E5FDBF811826C3BE35882E2C
:101608009355FC7AC8BA32E6C0199EA344543B0BE2
:101618008CC76B28A7BC16ADDB647414920C48B851
:101628009FBD43C43931D3F2D58B6EDA01B19C49E1
:10163800D8ACF3CFCAF447106FF04A5C38577397A9
:10164800CBA1E83E96610D0FE07C71CC9006F71CAB
:10165800C26AAE6917993A27D9EB2B22D2A9073368
:101668002D3C15C987AA50A50359091A65D784D0F6
:1016780082295A1E7BA86D2C637C777BF26B6FC521
:101688003001672BFED7AB76CA82C97DFA5947F07D
:10169800ADD4A2AF9CA472C0B7FD9326363FF7CC59
:1016A80034A5E5F171D8311504C723C31896059AF6
:1016B800071280E2EB27B27509832C1A1B6E5AA019
:1016C800523BD6B329E32F8453D100ED20FCB15B04
:1016D8006ACBBE394A4C58CFD0EFAAFB434D33856D
:1016E80045F9027F503C9FA851A3408F929D38F541
:1016F800BCB6DA2110FFF3D2CD0C13EC5F97441778
:10170800C4A77E3D645D197360814FDC222A9088EE
:1017180046EEB814DE5E0BDBE0323A0A4906245C7A
:10172800C2D3AC629195E479E7C8376D8DD54EA9DF
:101738006C56F4EA657AAE08BA78252E1CA6B4C6AB
:10174800E8DD741F4BBD8B8A703EB5664803F60E04
:10175800613557B986C11D9EE1F8981169D98E94F3
:101768009B1E87E9CE5528DF8CA1890DBFE642680C
:1017780041992D0FB054BB1623232323232320255F
:101788007320253032583A253032583A25303258AD
:101798003A253032583A253032583A253032583ABC
:1017A800253032583A253032583A253032583A25C1
:1017B8003032583A253032583A253032583A2530A6
:1017C80032583A253032583A253032583A25303294
:1017D800580D0A00232323232323204465764555E7
:1017E800493A202020202020253032583A2530320E
:1017F800583A253032583A253032583A253032583E
:101808003A253032583A253032583A253032580D78
:101818000A00232323232323204170704555493A86
:10182800202020202020253032583A253032583ABE
:10183800253032583A253032583A253032583A2530
:101848003032583A253032583A253032580D0A008D
:1018580023232323232320446576416464723A209A
:1018680020202020253032583A253032583A253069
:1018780032583A253032580D0A004170704B65795C
:101888003A2020202020004E776B4B65793A2020A3
:10189800202020004E776B534B65793A202020207A
:1018A80000417070534B65793A2020202000444253
:1018B800496E744B65793A202020004D43526F6F72
:1018C800744B65793A2020004D434B454B65793A76
:1018D80020202020004D43417070534B65795F30C4
:1018E8003A004D434E776B534B65795F303A0000B1
:1018F800000000004150505F8218010801000000FC
:101908004E574B5F8F180108080000004E574B5385
:101918009C1801080900000041505053A9180108FB
:101928000A0000004442495FB61801080B00000095
:101938004D435254C31801080C0000004D434B4559
:10194800D01801080D0000004D434B30DD18010888
:101958000E0000004D415330DD1801080F00000053
:101968004D4E5330EA180108100000005A45524FF6
:10197800940C0108526164696F53656E64204F7658
:10198800657273697A650D0A004952515F52585F52
:1019980054585F54494D454F55540D0A005052450F
:1019A800204F4B0D0A0053594E43204F4B0D0A0050
:1019B800484452204F4B0D0A00484452204B4F0DCB
:1019C8000A004952515F4352435F4552524F520DEC
:1019D8000A00020100030000841E0000093D000007
:1019E800127A000024F4000048E8010090D00300B7
:1019F80020A1070000000000B1280000615100008C
:101A0800C3A200000405060005EA0008E1E7000893
:101A180001EB00085DE800088DEE0008EDE900081C
:101A2800A9EC00084DEB0008B5E6000809EF00082E
:101A380005E90008F1E80008D5E7000889E800088A
:101A480061E8000819E800080FE800080DE7000839
:101A5800DBE700080BE8000807E8000899EA000837
:101A6800C5EA0008FDE7000825F000086DE7000852
:101A780035E70008F5EF000811E70008F9E6000867
:101A8800FFE6000841FE000847FE000805E70008D9
:101A980009E70008C01200001F000000A816000097
:101AA80017000000841C00000F000000E42500005F
:101AB8001E000000B42D00001600000008390000C8
:101AC8000E0000002C4C00001D000000685B0000A8
:101AD80015000000747200000D0000005898000006
:101AE8001C00000034B7000014000000E8E4000007
:101AF8000C000000783101001B000000686E010036
:101B08001300000034CA01000B0000002862020024
:101B18001A00000040DB0200120000003C930300A2
:101B28000A000000C0C204001900000060B30500EC
:101B380011000000382007000900000020A107005C
:101B4800000000000403020201010101000000007E
:101B5800000000003C4E554C4C3E003031323334CE
:101B680035363738396162636465666768696A6BF8
:101B78006C6D6E6F707172737475767778797A00A0
:101B880030313233343536373839414243444546AB
:101B98004748494A4B4C4D4E4F5051525354555655
:081BA8005758595A00000000D3
:081BB000C8E5FE7F0100000002
:081BB8005D01000800000000BF
:081BC0003901000800000000DB
:101BC8000000204100000000410300201027000011
:101BD80000000100000000000000000000000000FC
:101BE80004000000401F0000D91E0008091F00085B
